:020000040800F2
:1000000000000110DDE903082FA50308CD14010845
:10001000E1EA0308E1EA0308E1EA0308000000005E
:1000200000000000000000000000000071AB0308A9
:100030006FAB0308000000006DAB0308E5DF0008AC
:10004000E1EA0308E1EA0308E1EA0308E1EA030858
:10005000E1EA0308E1EA030845E8000871E900085D
:1000600035E90008F9E80008BDE8000801B000081B
:10007000F1AF0008E1AF0008D1AF0008C1AF000840
:10008000ADAF000899AF0008E1EA0308E1EA030810
:10009000E1EA0308E1EA0308E1EA030881E800086D
:1000A000E1EA030861D60008F1D5000889D6000806
:1000B00051D6000841D6000831D6000879C10008A1
:1000C00081C100086DC1000875C10008E1EA03089C
:1000D000E1EA030859E10008B9E0000819E0000866
:1000E00009E80008E1EA030881AC0308E1D500084B
:1000F00001D60008E1EA030811D6000885AF000820
:10010000E1EA0308E1EA030821D60008E1EA03086E
:10011000E1EA0308E1EA030865C1010849C10108F1
:1001200071AF00085DAF000849AF000835AF0008A7
:1001300021AF0008E1EA0308E1EA0308E1EA030865
:10014000E1EA0308E1EA0308E1EA030831A503084C
:100150000DAF0008F9AE0008E5AE0008E1EA0308BB
:1001600061C1000869C10008E1EA0308E1EA030887
:10017000E1EA0308E1EA0308E1EA0308E1EA030827
:08018000E1EA0308E1EA0308CB
:0801880074E503000100000012
:1001900002020300541F0020501F00200000000036
:1001A000000000000E020200441F0020581F002023
:1001B0000000000018060008160008007C2300203C
:1001C00094230020000000001A0600081D00010012
:1001D00058250020E4250020000000002206000829
:1001E0002700040078250020E825002000000000FA
:1001F00024060008010104002C2600206C35002094
:1002000000000000000000000802090094340020F3
:10021000703500200000000015C4000806020C0024
:100220000C3500207C35002000000000C18A000849
:100230000702020040350020883500200000000041
:100240002806000802000C00183500208C3500201C
:100250000000000000000000F701060088340020C4
:1002600098350020000000002A0600080A020A0053
:10027000B0260020A0350020000000003006000855
:1002800003123300633800203038002000000000E3
:100290003C06000825005A007C370020D637002095
:1002A0000000000000000000F6110C007037002074
:1002B0006437002000000000700600081500700080
:1002C00084360020F436002000000000000000000A
:1002D0002A006000C4350020243600200000000001
:1002E000B58803082C001000003E0020F03D0020DF
:1002F00000000000B12102082B002400343E002041
:10030000103E00200000000081210208290050005A
:10031000283D0020583E00200000000000000000A2
:1003200005100600E03F00202C41002000000000E6
:100330007C0600080E20EA00C03E00203441002068
:1003400000000000E557020813000400F43F0020FD
:100350002042002000000000840600080201030083
:10036000AB3E0020244200200000000041B80108FC
:1003700001200800544300208043002000000000BA
:10038000880600081A00080038430020884300202F
:10039000000000009006000812200C00B843002066
:1003A0005C44002000000000980600080C002400B7
:1003B000C4430020684400200000000019B8010870
:1003C00000020500904300208C4400200000000043
:1003D000000000001E000400344B00201C4D0020D3
:1003E00000000000A406000822000C00A04A002023
:1003F000204D002000000000A80600081F000E008D
:100400008C4E00206050002000000000B406000860
:1004100005020100744E0020705000200000000012
:10042000C2060008140002001053002014530020DC
:1004300000000000C4060008100003000053002064
:100440001853002000000000C60600082800100015
:10045000F05200201C53002000000000FD8C020818
:1004600023001000E05200202C5300200000000068
:10047000218D020819000500D85200203C530020AD
:1004800000000000CA060008F8110100D452002044
:100490004453002000000000D006000800010400C2
:1004A000D05200204853002000000000D20600086F
:1004B0002F001100BC5200204C530020000000000F
:1004C000D606000834001000C85B0020985C0020AD
:1004D00000000000DD88030818102C00645B002079
:1004E000A85C002000000000912802080D003400E4
:1004F000905B0020D45C002000000000312703083E
:10050000FA010200D0530020085D00200000000026
:1005100049C200081B00F400F4640020147300209A
:100520000000000035B1020826000E0018740020FB
:100530000874002000000000853703080B2010001D
:10054000D06200202874002000000000E8060008A7
:100550000902010099740020DC74002000000000F2
:10056000F806000803010A00107500201C75002021
:1005700000000000FA060008FD012400AC82002003
:10058000D08200200000000095C30008060016007D
:10059000287F0020F4820020000000000558020897
:1005A000FB010100647E00200C830020000000009D
:1005B00041C20008FC010900307D002010830020AA
:1005C000000000000DC200080A101200287500206B
:1005D0001C83002000000000040700080300010045
:1005E000E4840020C089002000000000000000001A
:1005F00004008000589D002094A600200000000008
:1006000000000000F90104003C92002014A7002023
:080610000000000005C4000811
:100618000000C40900001901282800002003000078
:10062800013C35000100000000004A01B400D60179
:1006380000000000000000000000000000000000B2
:1006480000000000000000000000000000000000A2
:100658000000000000000000000000000000000092
:100668000000000000000100000000000000000081
:100678000000000020000101000000000800000048
:10068800E8036400040A00017E05EA05B4053200A7
:10069800000000010005434F4C4900000000010024
:1006A800C800141E010064002C012800000000008E
:1006B8000000010000000005000000000300000128
:1006C800050000002801000004009001000000005F
:1006D8000000000000000000000000000000000012
:1006E8002B21231E64000200000001000A012900DA
:1006F8001A00040101006C1600000000003001001F
:0E070800005A0000000090012C01C80064009F
:100716005001000007000000020000000000000079
:10072600000000000102030406070809FF0000009C
:1007360001010000C4350408D86804080000000060
:1007460000000000D4350408DC3504080000000071
:1007560001200000E0350408E83504080000000028
:1007660001400000EC350408EC4F040800000000CE
:1007760001200000F83504080436040800000000D3
:1007860004000000083604081436040800000000BF
:100796000400000018360408206004080000000069
:1007A60001000000020100000000803F0000803FC1
:1007B6000000000000000000000000000000803F74
:1007C600F40704080508040000000000D02B040804
:1007D60004240408BC2B04080000000020080408B8
:1007E60005080A0000000000D02B040804240408B1
:1007F600DC1E040800000000FFFFFFFF0101D60118
:10080600591B0208000000000000000020700020B4
:10081600702D72000000000000000000A40E0020F1
:10082600FFFFFFFFFA0000000100000001000000CA
:10083600C060040800000000000000000000000086
:1008460000000000AE600408040000009F52030888
:100856000000000000000000C8600408010000005D
:100866000000000000000000000000000000000082
:100876000D00000000000000000000000000000065
:100886000A9E00200100C40900000000089E002006
:100896000100C40900000000069E00200100C409F2
:1008A60000000000049E00200100C40900000000B2
:1008B600009E00200100C40900000000029E0020E6
:1008C6000100C40900000000FE9D00200100C409CB
:1008D60000000000FC9D00200100C409000000008B
:1008E600000000000000000020010020304E002023
:1008F6009CFF2C0100000000241500200A000000C7
:10090600DC1E04083C740020E0150C1700000000F3
:1009160026150020080000000424040825150020E0
:1009260005000000D02B04083E74002002000000E1
:10093600F41E0408E63F00200100FF7F01000000CE
:10094600DF3F002002000000001F0408B43E002024
:1009560003000000101F0408B33E0020030000003F
:10096600101F0408B23F00200000F401010000003F
:10097600B03F00200000F40101000000AE3F00205F
:100986000000F40101000000AC3F00200000F4016B
:1009960001000000AA3F002000FF0100CA3F00201E
:1009A600E803D0070A000000C83F002000640100E9
:1009B6000A000000C43F002000640100C33F00207D
:1009C60000640100C93F0020006401000A00000025
:1009D600C23F0020006401000A000000C73F00205B
:1009E600006401000A000000C63F00200064010008
:1009F6000A000000C53F0020006401000A00000054
:100A0600C13F002000FF01000A000000C03F002097
:100A160000FF01000A000000BC3E00200000F401B7
:100A260001000000BA3E00200000F40101000000B1
:100A3600B83E00200000F40101000000B63E002090
:100A46000000F40101000000BC3F00201400E80390
:100A560001000000BA3F0020E803307501000000E5
:100A6600B93F002000C80100B83F002000C80100BF
:100A7600B73F002000C80100B63F00200064010017
:100A86000A000000B53F002000FF01000A00000038
:100A9600D53F002000C80100D43F002000C8010057
:100AA600D33F002000C80100D23F002000C801004B
:100AB600D13F002000C80100D03F002000C801003F
:100AC600CF3F002000C80100CE3F002000C8010033
:100AD600CD3F002000C80100FC60040800000000B3
:100AE6000000000000000000000000000C61040887
:100AF6000900000000000000C401002004000000FE
:100B0600146104080900000000000000B80100207C
:100B160004000000FC640408090000000000000056
:100B2600AC010020040000001C610408090000005C
:100B360000000000A001002004000000206104085D
:100B460009000000000000009401002004000000DD
:100B56002861040809000000000000008801002048
:100B660004000000306104080900000000000000D5
:100B76007C01002004000000386104080900000020
:100B8600000000007001002004000000C860040896
:100B9600010000000000000000000000000000004E
:100BA600000000000D000000000000000000000032
:100BB600000000004C620408000000000000000075
:100BC60000000000000000005C6204080500000050
:100BD60000000000B23E002000000000C8600408CB
:100BE60001000000000000000000000000000000FE
:100BF600000000000D0000000000000000000000E2
:100C0600000000006462040800000000000000000C
:100C16000000000000000000D86804080000000082
:100C260000000000C30F00200400000070620408EA
:100C36000C00000001530308180200200000000009
:100C4600DC6E04080C000000094D03080C020020AD
:100C560000000000746204080C000000ED4C03085C
:100C660000020020000000007C620408080000006A
:100C760000000000F4010020040000008462040863
:100C86000C000000394C0308E801002000000000B9
:100C96008C6204080900000000000000DC0100204E
:100CA600040000009462040803000000794702086B
:100CB600D001002000000000C86004080100000008
:100CC600000000000000000000000000000000001E
:100CD6000D00000000000000000000000000000001
:100CE60098620408000000000000000000000000F8
:100CF60000000000A86204080C00000000000000CC
:100D06003002002000000000B06204080A00000063
:100D1600000000005040002000000000BC620408F3
:100D26000A000000000000005840002000000000FB
:100D3600C46204080A0000000000000060400020B1
:100D460000000000CC62040808000000000000005B
:100D56002402002000000000D46204080400000001
:100D6600AD4802080000000000000000C86004084A
:100D7600010000000000000000000000000000006C
:100D8600000000000D000000000000000000000050
:100D960000000000E06204080000000000000000FF
:100DA6000000000000000000F46204080C000000CF
:100DB6000000000048020020000000000463040850
:100DC60004000000C1450208000000000000000009
:100DD6000C6304080C000000000000003C02002028
:100DE600000000002063040804000000A14502087A
:100DF6000000000000000000C860040801000000B8
:100E060000000000000000000000000000000000DC
:100E16000D000000000000000000000000000000BF
:100E26002863040800000000000000000000000025
:100E3600000000003C6304080700000000000000FA
:100E46008402002000000000486304080800000037
:100E5600000000007802002000000000546304082F
:100E660008000000000000006C02002000000000E6
:100E76006063040808000000000000006002002013
:100E8600000000006C630408080000000000000079
:100E96005402002000000000C860040801000000A1
:100EA600000000000000000000000000000000003C
:100EB6000D0000000000000000000000000000001F
:100EC600786304080000000000000000FF00002016
:100ED60000000000846304080B000000000000000E
:100EE600FC020020000000008C6304080B000000D8
:100EF60000000000F00200200000000098630408D3
:100F06000B00000000000000E402002000000000CA
:100F1600A46304080B00000000000000D8020020B3
:100F260000000000B06304080B0000000000000091
:100F3600CC02002000000000BC6304080B00000087
:100F460000000000C002002000000000C463040886
:100F56000B00000000000000B402002000000000AA
:100F6600D06304080700000000000000AC02002067
:100F760000000000D863040807000000000000001D
:100F8600A402002000000000E46304080B00000037
:100F9600000000009802002000000000F063040832
:100FA60008000000000000008C0200200000000085
:100FB600C8600408010000000000000000000000F6
:100FC60000000000000000000D000000000000000E
:100FD6000000000000000000FC63040800000000A0
:100FE600000000000000000000000000106404087B
:100FF60008000000000000002C0300200000000094
:101006001C64040808000000000000002003002003
:10101600000000002864040808000000000000002A
:1010260014030020000000003464040808000000D7
:10103600000000000803002000000000C86004084B
:101046000100000000000000000000000000000099
:10105600000000000D00000000000000000000007D
:10106600000000003C6404080000000000000000CE
:10107600FC000020000000004C6404080B00000087
:1010860000000000740300200000000058640408FB
:101096000B000000000000006803002000000000B4
:1010A60064640408070000000000000060030020DC
:1010B6000000000070640408070000000000000043
:1010C60058030020000000007C64040807000000AC
:1010D600000000005003002000000000886404089F
:1010E600080000000000000044030020000000008B
:1010F6009064040808000000000000003803002087
:1011060000000000C86004080100000000000000A4
:101116000000000000000000000000000D000000BC
:1011260000000000000000000000000098640408B1
:101136000000000000000000FC000020000000008D
:10114600A46404080700000000000000C00300209B
:1011560000000000AC640408070000000000000066
:10116600B803002000000000B46404080700000073
:1011760000000000B003002000000000BC6404086A
:101186000700000000000000A80300200000000087
:10119600C46404080700000000000000A00300204B
:1011A60000000000CC6404080700000000000000F6
:1011B6009803002000000000D46404080700000023
:1011C600000000009003002000000000DC6404081A
:1011D6000700000000000000880300200000000057
:1011E600E4640408070000000000000080030020FB
:1011F60000000000C86004080100000000000000B4
:101206000000000000000000000000000D000000CB
:1012160000000000000000000000000000000000C8
:1012260099410208C8030020B03E00201B000000C0
:10123600201F0408AF3E00200A320100AE3E002007
:1012460001FA0100AA3E002000C80100A83E0020C5
:10125600E803D00701000000434F4C4942524900C1
:10126600AF41020875450208A4040020754C030826
:1012760000000000F40400208D480208F54302082F
:10128600D0050020D141020800000000840600209D
:10129600594202082942020810070020E1420208CA
:1012A60025430208B0070020BE3F002001030100CD
:1012B60005420208E1410208C808002089420208E6
:1012C600E145020854090020554302083946020840
:1012D6001C0A0020B43F002001030100EC6404084E
:1012E60000000000000000000000000000000000F8
:1012F600F864040808000000000000003C0B002011
:10130600000000000065040807000000000000005F
:10131600340B0020000000001065040807000000E0
:10132600000000002C0B0020000000001C650408D3
:101336000700000000000000240B00200000000051
:10134600286504080C00000000000000180B0020AF
:101356000000000034650408030000007947020815
:101366000C0B002000000000C8600408010000000B
:101376000000000000000000000000000000000067
:101386000D0000000000000000000000000000004A
:101396003C6504080000000000000000000000009A
:1013A600000000004C6504080A0000000000000070
:1013B6002436040800000000546504080A000000F2
:1013C60000000000A4350408000000005C65040865
:1013D6000A00000000000000D63F002000000000C8
:1013E600646504080A00000000000000480B0020A5
:1013F60000000000C86004080100000000000000B2
:101406000000000000000000000000000D000000C9
:101416000000000000000000000000006C650408E9
:1014260000000000000000000000000000000000B6
:10143600806504080300000079470208680B002055
:10144600000000008C6504080300000079470208CC
:101456002815002000000000946504080300000021
:10146600794702085C0B0020000000009C65040818
:101476000300000079470208500B0020000000001E
:10148600C860040801000000000000000000000021
:1014960000000000000000000D0000000000000039
:1014A6000000000000000000A8650408000000001D
:1014B600000000000000000000000000B465040801
:1014C6000700000085460208C40B0020000000004B
:1014D600486A04080300000079470208B80B002098
:1014E60000000000C06504080300000079470208F8
:1014F600AC0B002000000000C865040803000000D3
:1015060079470208A00B002000000000D0650408FF
:101516000700000069460208980B00200000000042
:10152600F86E040803000000794702088C0B0020BF
:1015360000000000DC65040803000000794702088B
:10154600800B002000000000E8650408030000008E
:1015560079470208740B002000000000C8600408E8
:101566000100000000000000000000000000000074
:10157600000000000D000000000000000000000058
:10158600000000006141020829410208CC0B00203E
:10159600C143020800000000800C0020000000008B
:1015A600000000000C0D002099430208A146020825
:1015B600980D0020F46504080000000000000000FB
:1015C60000000000000000000066040803000000A0
:1015D60079470208980E00200000000008660408FB
:1015E60003000000794702088C0E0020000000006E
:1015F600146604080300000079470208800E0020E4
:101606000000000020660408030000007947020875
:10161600740E002000000000286604080200000086
:101626005D49020800000000000000003066040862
:10163600020000005D4902080100000000000000F1
:101646003C660408020000005D4902080200000032
:1016560000000000000000000D0000000000000077
:1016660000000000000000000000803F00000000B5
:1016760000000000000000000000803F00000000A5
:101686000000000000000000000000000000000054
:101696000000000000000000000000000000000044
:1016A6000000803F00000000000000000000000075
:1016B600010000000001010101000000000001011D
:1016C600FFFF000000FFFF0000000000AA55050113
:1016D6000000012D202D2D202D2D2D2D202D2D2DE1
:1016E6002D000000000000000000000000000000C7
:1016F6000000AA550B010000AA5507010000AA55D3
:10170600090200000000000001000000C012AA55F6
:1017160003009F0000000001000000000000000020
:101726000000000047A4030801A40308AFAB0308A8
:101736000000000069A0030875A20308F1A20308CF
:10174600DDA1030800000000000000005DA0030802
:1017560041A003083FA003083DA0030837A00308E3
:1017660035A003083BA0030839A0030851A00308CD
:1017760043A00308B5A10308C9A10308A1A1030852
:101786008DA1030879A10308D856040800000000BB
:101796000000000055B80108A08601000400000002
:1017A6000000000000000000000000000000000033
:1017B600000000000000000000000000486A040865
:1017C6002C56040800000000E56401087D000000B6
:1017D60006000000000000000000000000000000FD
:1017E60000000000000000000000000000000000F3
:1017F600546D040800000000000000009D0D010863
:10180600E8030000030000000000000000000000E4
:1018160000000000000000000000000000000000C2
:10182600000000005C6D04080000000000000000DD
:1018360049590208102700000300000000000000BC
:101846000000000000000000000000000000000092
:101856000000000000000000C0670408000000004F
:101866000920020875EA0008204E00000500000065
:101876000000000000000000000000000000000062
:10188600000000000000000000000000645804088A
:1018960000000000000000002D15010810270000C0
:1018A6000100000000000000000000000000000031
:1018B6000000000000000000000000000000000022
:1018C600686D0408000000000000000041EA0008FE
:1018D600E803000005000000000000000000000012
:1018E60000000000000000000000000000000000F2
:1018F60000000000746D04080000000000000000F5
:1019060055BA0108204E0000030000000000000048
:1019160000000000000000000000000000000000C1
:101926000000000000000000846D040800000000B4
:101936000000000085B80108204E000003000000EA
:101946000000000000000000000000000000000091
:10195600000000000000000000000000946D040874
:10196600000000000000000009120108400D0300FD
:10197600030000000000000000000000000000005E
:101986000000000000000000000000000000000051
:101996009C5704080000000000000000D132030834
:1019A60010270000010000000000000000000000F9
:1019B6000000000000000000000000000000000021
:1019C6000000000048560408000000000000000067
:1019D600017B020810270000030000000000000041
:1019E60000000000000000000000000000000000F1
:1019F6000000000000000000A46D040800000000C4
:101A060000000000ADDA0308A08601000100000016
:101A160000000000000000000000000000000000C0
:101A26000000000000000000000000003856040816
:101A36000000000000000000CDD9030850C30000DC
:101A4600010000000000000000000000000000008F
:101A56000000000000000000000000000000000080
:101A6600E4610408000000000000000035D503080A
:101A7600A861000001000000000000000000000056
:101A86000000000000000000000000000000000050
:101A960000000000AC6D040800000000000000001B
:101AA6006D8B0208A0860100010000000000000006
:101AB6000000000000000000000000000000000020
:101AC60000000000000000006C5804080000000040
:101AD60000000000851A0108A00F000001000000A8
:101AE60000000000000000000000000000000000F0
:101AF600000000000000000000000000B86D0408AF
:101B0600000000000000000041AB020810270000A2
:101B160001000000000000000000000000000000BE
:101B260000000000000000000000000000000000AF
:101B3600D058040800000000000000005DC502083F
:101B46001027000001000000000000000000000057
:101B5600000000000000000000000000000000007F
:101B660000000000145604080000000000000000F9
:101B7600F14A02081A4100000100000000000000BE
:101B8600000000000000000000000000000000004F
:101B96000000000000000000C46D04080000000002
:101BA60000000000A1D00308400D03000000000063
:101BB600000000000000000000000000000000001F
:101BC600000000000000000000000000CC6D0408CA
:101BD60000000000000000005DD00308400D030077
:101BE60000000000000000000000000000000000EF
:101BF60000000000000000000000000000000000DF
:101C0600D46D040800000000000000009D88020852
:101C1600A086010003000000000000000000000094
:101C260000000000000000000000000000000000AE
:101C36000000000001010100254D0308000000001E
:101C46009C160020306F0408000000000000000011
:101C56000000000000000000D86804080000000032
:101C660000000000DC1A002004000000DC6E0408FE
:101C76000C0000004D450208C41A002000000000B8
:101C8600746204080C00000025450208B81A0020FA
:101C9600000000007C62040808000000000000004C
:101CA600AC1A002004000000846204080C00000046
:101CB60005410208A01A00200000000094620408F2
:101CC6000300000079470208941A00200000000073
:101CD600406F04080300000079470208881A0020B4
:101CE60000000000C86004080100000000000000B9
:101CF6000000000000000000000000000D000000D1
:101D0600000000000000000000000000306F040822
:101D160000000000000000000000000000000000BD
:101D2600D86804080000000000000000DC1A00204B
:101D360004000000846E0408030000002553030815
:101D46007C1A002008000000846204080C000000D1
:101D560005410208A01A0020000000009462040851
:101D66000300000079470208941A002000000000D2
:101D7600406F04080300000079470208881A002013
:101D860000000000C8600408010000000000000018
:101D96000000000000000000000000000D00000030
:101DA600000000000000000000000000486F04086A
:101DB600000000000000000000000000000000001D
:101DC600D86804080000000000000000DC1A0020AB
:101DD600040000008C6E0408030000007947020826
:101DE600D01A002000000000C860040801000000AE
:101DF60000000000000000000000000000000000DD
:101E06000D000000000000000000000000000000BF
:101E16004274002088136F170100000044740020EC
:101E260088136F1700000000E06D04080000000032
:101E3600000000000000000000000000F06D040833
:101E460008000000000000000C170020040000003D
:101E5600FC6D0408080000000000000000170020C8
:101E660000000000946204080400000065530308A3
:101E76000000000000000000C86004080100000027
:101E8600000000000000000000000000000000004C
:101E96000D0000000000000000000000000000002F
:101EA6004074002088136F17010000006C4E00205C
:101EB60088136F1700000000854D0308000000001E
:101EC600181700209874002001000000902B0408C9
:101ED6006E4E0020010000009C2B0408644E00207A
:101EE60002000000A42B0408529E002000000000FF
:101EF60000000000509E00200000000000000000CE
:101F06004E9E002000000000000000004C9E0020B5
:101F160000000000000000004A9E002000000000B3
:101F260000000000489E00200000000000000000A5
:101F3600FC0F002000000000000000003F7400209D
:101F460002000000B02B04083C6E040800000000EC
:101F5600000000000000000000000000F06D040812
:101F660008000000000000009C170020040000008C
:101F7600FC6D040808000000000000009017002017
:101F8600000000009462040804000000594D030894
:101F96000000000000000000C86004080100000006
:101FA600000000000000000000000000000000002B
:101FB6000D0000000000000000000000000000000E
:101FC6004C6E040800000000000000000000000045
:101FD600000000005C6E04080C000000CD440208FE
:101FE600CC17002004000000686E04080C000000F6
:101FF60075440208C017002004000000746E04082F
:102006000C00000099440208B417002000000000EC
:10201600806E04080300000045530308A81700203B
:10202600080000008C6E04080300000079470208CF
:10203600D01A002000000000C8600408010000005B
:10204600000000000000000000000000000000008A
:102056000D0000000000000000000000000000006D
:10206600C06004080000000000000000000000003E
:1020760000000000946E0408040000008153030869
:102086000000000000000000C86004080100000015
:10209600000000000000000000000000000000003A
:1020A6000D0000000000000000000000000000001D
:1020B600E46E0408000000000000000000000000BC
:1020C60000000000645904080C0000000000000035
:1020D6002C18002004000000F46E0408080000001C
:1020E600000000002018002004000000006F040813
:1020F6000800000000000000141800200400000082
:10210600086F0408080000000000000008180020FE
:1021160004000000106F0408080000000000000022
:10212600FC17002004000000186F040808000000D7
:1021360000000000F017002004000000206F0408D3
:102146000800000000000000E41700200400000062
:10215600286F04080800000000000000D8170020BF
:1021660004000000C8600408010000000000000030
:102176000000000000000000000000000D0000004C
:10218600000000000000000000000000714D030880
:1021960000000000381800200000000000000000C9
:1021A600B0180020000000000000000050190020B8
:1021B6006A4E002004000000BC2B0408684E002074
:1021C600E0150C1700000000674E00200800000014
:1021D60004240408664E002005000000D02B0408E5
:1021E6000000000000000000A01900202D202D2D69
:1021F600202D2D2D2D202D2D2D000000000000005E
:1022060000000000000000000000000000000000C8
:102216000102030401020304060708090100000085
:10222600006002401060024000000000000B000049
:1022360000002000000000000000000000600240D6
:102246002860024000000000060C0000000020008C
:1022560000000000000000000060024040600240F4
:1022660000000000100D000000002000000000002B
:1022760000000000006002405860024000000000BC
:10228600160E000000002000000000000000000004
:10229600006002407060024000000000200F000055
:1022A6000000200000000000000000000060024066
:1022B6008860024000000000261000000000200098
:1022C600000000000000000000600240A060024024
:1022D6000000000030110000000020000000000097
:1022E6000000000000600240B860024000000000EC
:1022F600362F000000002000000000000000000053
:102306000064024010640240000000000038000033
:1023160000004000000000000000000000640240D1
:10232600286402400000000006390000000040005A
:10233600000000000000000000640240406402400B
:1023460000000000103A00000000400000000000FD
:1023560000000000006402405864024000000000D3
:10236600163B0000000040000000000000000000D6
:10237600006402407064024000000000203C00003F
:102386000000400000000000000000000064024061
:10239600886402400000000026440000000040005F
:1023A600000000000000000000640240A06402403B
:1023B6000000000030450000000040000000000062
:1023C6000000000000640240B86402400000000003
:1023D600364600000000400000000000000000003B
:1023E600040309041201000202020040830440575C
:1023F600000201020301000009024300020100C0BD
:102406003209040000010202010005240010010542
:1024160024010001042402020524060001070582A6
:10242600030800FF09040100020A00000007050175
:10243600024000000705810240000000FF00000086
:102446005D6803081DA3030815630308A9A0030814
:10245600DDA40308B9A00308D5A003089BA00308C0
:102466008DA0030800000000000000000000803F6F
:10247600685E0C00681D00200000000000000000DF
:102486000000000000000000000000000000000046
:102496000000000000000000000000000000000036
:1024A6000000000000000000000000000000000026
:1024B6000000000000000000000000000000000016
:1024C6000000000000000000000000000000000006
:1024D60000000000000000004300000000000000B3
:1024E60000000000000000000000000000000000E6
:1024F6000000000000000000430000000000000093
:1025060000000000000000000000000000000000C5
:102516000000000000000000430000000000000072
:1025260000000000000000000000000000000000A5
:102536000000000000000000430000000000000052
:102546000000000000000000000000000000000085
:102556000000000000000000430000000000000032
:102566000000000000000000000000000000000065
:102576000000000000000000430000000000000012
:102586000000000000000000000000000000000045
:1025960000000000000000004300000000000000F2
:1025A6000000000000000000000000000000000025
:1025B600000000000000000023ED0308FFEC030804
:1025C60000000000BB6F0408AA600408AA400408C3
:1025D600AA400408AA400408AA400408AA4004081D
:1025E600AA400408AA400408AA400408AA4004080D
:1025F600FFFFFFFFFFFFFFFFFFFFFFFFFFFF0000E3
:10260600010041534349490000000000000000005A
:1026160000000000000000000000000000000000B4
:10262600000041534349490000000000000000003B
:102636000000000000000000000000000000000094
:0826460000000000010000008B
:10800000002870B51EDB0928044620DD012303EBA0
:1080100083035B00B0FBF3F2092AF8D87BB10E4E64
:10802000B4FBF3F00928CCBF57223022A6FB03E5AE
:10803000024403FB1044EB0801F8012BF0D10023AC
:108040000B7070BD2D230B7040420131DBE73030E7
:1080500001F8010BF3E700BFCDCCCCCC884230B4A3
:108060004FF001042ED301FB04F4B0FBF4F58D4274
:10807000F9D284B1AAB901E0B0FBF4F5092DCCBF67
:10808000572230222A4404FB150003F8012BB4FBCD
:10809000F1F4002CF0D100221A7030BC7047B0FB14
:1080A000F4F5092DCCBF372230222A4404FB1500F9
:1080B00003F8012BB4FBF1F4002CF0D100221A706C
:1080C00030BC70470546002AEBD1D7E72DE9F047D1
:1080D00014461D46064600234FF47A722046294670
:1080E00036F0A8FADFF840814B4A4C4F88FB00314C
:1080F0000144C31782FB002EC3EB611188FB0128EA
:1081000087FB00278644464AC3EBEE2EC1EB011CD9
:1081100082FB0E29A0EB8C0C0744424A86F806C06D
:10812000C3EB27474FEAEE7C08EB010ACCEBA90C26
:1081300082FB07824FEAE1780CEB4C0CC8EB6A1823
:10814000AEEBCC0EC8EB0818DFF8E0C086F804E010
:10815000A1EB880171718CFB0010F917C1EBE212E1
:1081600040F2B55101FB1272C3EBE050B2F5896FDA
:108170004FEA80073CDA40F2DA239A4242DCB2F559
:10818000B77FB4BF4FF0000C4FF0010C4FEA4C0921
:10819000DFF89C8009EB0C0308EBC3031FFA8CFE8D
:1081A000D88A09EB0C0108EBC10116310B2301E061
:1081B00031F8020D824218DA013BF9D1CC44012397
:1081C00038F83C00B37007F2B2770132121ABE449D
:1081D000F270A6F800E0204629464FF47A72002398
:1081E00036F028FA3281BDE8F0870133DBB2E9E7E7
:1081F0004FF0030EF44640F29650DFF834804FF013
:108200000609CEE74FF0020EDFF82480F44640F274
:1082100029404FF00409C4E7C5B3A29107452EC217
:10822000ABAAAA2A73B06D1689888888792D0311A4
:1082300030FE030803685A1C02601970704700BFC3
:108240002DE9F047089C2578002B804689460CBF15
:108250004FF0200A4FF0300A661C35B3002A29DDA2
:10826000334601E0024698B113F8011B501E002965
:10827000F8D1971E60B13D46013D51464046C84782
:108280006B1C002BF8DC257827EAE770013055B12C
:10829000041B29464046C847301916F8015B002DDB
:1082A000F7D1BDE8F087BDE8F087002A04DC284656
:1082B000BDE8F0870020EBE7571EDCE783684268E3
:1082C000D0ED037A00EB83010133934281ED040A80
:1082D000836004BF0023836000EB830393ED047A83
:1082E000036870EE277A9A42C0ED037A77EEC77A78
:1082F000C0ED037A0CDA013307EE103AF8EEC76AE4
:10830000B7EE007A87EEA60A036030EE070A7047E0
:1083100007EE102AB8EEC77A87EE870A704700BFCB
:1083200090ED057A90ED004AD0ED066AD0ED014A55
:10833000D0ED047A90ED035AD0ED025AA4EE007A03
:10834000B0EE406AB0EE470AB0EE667AA6EE247A46
:1083500067EEC07AA0EE457AE6EE257A80ED057AE2
:10836000C0ED067A704700BFD0ED057A90ED013A76
:10837000D0ED003AD0ED064A90ED024A90ED077A32
:1083800090ED035A90ED086AD0ED045AC0ED067ADC
:10839000F0EE406A27EE830AC0ED056AA3EEA60A56
:1083A00080ED087AA4EE240AA5EE470AA5EEC60AD7
:1083B00080ED070A704700BFD0ED007A90ED017A9A
:1083C00030EE670AE7EE007AB0EE670AC0ED007A99
:1083D000704700BF704700BF0A44914214D030B4C8
:1083E0000139551E41F2210211F8014F082380EA9C
:1083F000042004044CBF82EA40004000013B80B2EC
:10840000F7D18D42F0D130BC704770470378407887
:1084100040EA032010FB01F04FF4807190FBF1F073
:1084200000F30F0000B270472DE9F04F654B664E28
:10843000B3F80AC03468B3F8048087B04FEA0C2A56
:1084400005901889B4EB0A0A4FF000024FF00005BE
:1084500065EB020BA0FB0A4500FB0B55E00940EA67
:1084600045604FEA084407198E46D8884FEAE5115F
:1084700041EB0208A0FB0A45CDE90278B3F802807F
:1084800000FB0B55200A40EA05604FEAC83410EBA8
:1084900004084FEA252141EB02099A89A2FB0A014F
:1084A00002FB0B11C20D42EA412212F5FA604FEABB
:1084B000E15343F10001B0F5FA6FCDE9000171F12C
:1084C0000001B4465EDA0524A2FB040104FB03119B
:1084D00000FB03F402FB0144DDE90267A0FB02019B
:1084E00021444D104FEA3004361B4FEA900444EA11
:1084F000817467EB05078D10B8EB040869EB05097B
:10850000DDE9004531484FF0FF31844275EB010150
:10851000CDE9026723DA40F6AC5012184FF00001A3
:108520004B4102FB03F1A2FB022303EB4103D90001
:10853000D000101A41EA527163EB0101341847EB85
:108540000105CDE902450B24A2FB040104FB031144
:1085500049104FEA3000B8EB000869EB01090AFB4B
:108560000BF3DDE90001AAFB0AAB0BEB430B4FEA6F
:10857000DA7242EA4B02801A4FEAEB7361EB0301B5
:10858000CDE90001DCF80410A1FB082301FB09334D
:10859000540D5D1544EAC324DDE90223A21A65EBFC
:1085A00003031D46D30B059A43EA454302B113600A
:1085B000BEF1000F02D0009BCEF8003007B0BDE83E
:1085C000F08F00BF3C490020381F002024FAFFFF35
:1085D0004FF4805383827047012380F84530704701
:1085E000BFF34F8F0549064BCA6802F4E06213439C
:1085F000CB60BFF34F8F00BFFDE700BF00ED00E091
:108600000400FA0570B4037B04681F2B08D9203BD3
:108610002021626801FA03F31A421CD170BC704732
:108620002021226801FA03F31A42F7D04269144963
:108630005C2000FB021251685689CD6808682968E1
:1086400021F001012960828992B222EA0602828128
:10865000A36070BC7047426909495C2000FB0212AC
:1086600051685689CD680868296821F001012960A0
:10867000828992B222EA06028281E36070BC70476E
:10868000507F00202B4B1978002951D02A4B30B451
:108690001C68988800226262A5899A80284380B26B
:1086A0000129A08143D09C6898896262A5892843EA
:1086B00080B20229A0819A8139D01C69988A6262AD
:1086C000A589284380B20329A0819A822FD09C6972
:1086D000988B6262A589284380B20429A0819A837D
:1086E00025D01C6A988C6262A589284380B205292E
:1086F000A0819A841BD09C6A988D6262A5892843C8
:1087000080B20629A0819A8511D01C6B988E626276
:10871000A589284380B20729A0819A8607D0986B43
:10872000998F42628489214389B281819A8730BCC2
:10873000704700BF308200203482002010B4037BD9
:1087400001681F2B09D9203B20224C6802FA03F351
:108750001C4214D15DF8044B704720220C6802FAC9
:1087600003F31C42F6D00C4A4068002414700268DF
:108770005DF8044B22F0010202608B607047064AEC
:1087800040680024147002685DF8044B22F0010276
:108790000260CB60704700BFB5490020F0B5C4004F
:1087A00022189200AE498B585B689D8AADB2EEB23A
:1087B000F7070A445CD4B70732D5BFF35F8F167E44
:1087C000F6B2012E00F0C780A64D1A8BBFF35F8F63
:1087D000221801EB8202167E022E00F0D5802218AC
:1087E00001EB8202167E032E00F088809A8895F9AC
:1087F000086092B242F480629A80221801EB8202F1
:10880000127E013296425BD1AA7A00266E72002A4D
:1088100040F09580204401EB800000234375F0BDBB
:1088200077074ED416F0400600F0C9808D4D1E8AA1
:1088300095F908E0176AF6B207F80E605FFA8EFE47
:108840000EF1010C4FFA8CFC177E85F808C00CF174
:1088500003029742664600F01C81221801EB820257
:10886000127E9445C9D10EF1020676B22E72C4E78B
:108870001E887C4D26F400663604360C1E801E8849
:10888000B6B246F480661E80967E00272F72002EB8
:1088900048D06E7A002E42D0221801EB82020126C7
:1088A000127E6E72022A00F0B980221801EB820259
:1088B000927D42F001021A82204401EB8000037E87
:1088C000F0BD684D967E0127AF72002E73D06E7A90
:1088D000002E7BD1221801EB8202527E002A00F08A
:1088E000A3801A882E7A92B2013642F4007276B2D0
:1088F0001A802E721A88D205FCD47EE7927E002A56
:108900003FF474AF6A7A002A3FF470AF9A8895F901
:10891000086022F480621204120C9A806DE7D27D06
:10892000FF2AB9D0221801EB8202967D06F0FE06DE
:108930001E82D37DFF2BBFD0FF232B72BCE79A880A
:1089400022F4407212042044120C01EB80009A8041
:1089500000234375F0BD927E424D002A3FF435AFAF
:108960006A7A002A3FF431AF1A8822F48062120436
:10897000120C1A80BFF35F8F1A8B1A88AE7292B2F4
:1089800042F400721A8031E7927E002A3FF427AF4A
:108990006A7A002A3FF423AF1A8895F9086022F416
:1089A00080621204120C1A809A8822F480621204E7
:1089B000120C9A8021E76A7A002A8BD091E715F091
:1089C000800F284D3AD195F9086016E7167ED2F847
:1089D00020E01F88022E95F9086045D927F48067AA
:1089E0003F043F0C1F801F8AFFB20EF806701F88DD
:1089F000D2F820E0BFB247F400771F80F2B21F8A9E
:108A0000561C76B2FFB20EF806709F88961CBAB25A
:108A100076B242F480622E729A806BE71A8892B224
:108A200042F400621A8040E71A8895F9086092B211
:108A300042F4807201271A806F725BE795F9087023
:108A4000B7F1FF3F2CD0D669F65D1E8292F818E090
:108A500001377AB2964516462A727FF4CEAEA3E766
:108A6000A0340020381F0020BFB247F400771F80D9
:108A70001F8AFFB20EF80670F6B21F8AD2F820E005
:108A8000721C52B20336FFB276B20EF802702E722A
:108A900030E79A8822F480621204120C9A80DCE695
:108AA000D77D1F822E72957E1DB9127E002A7FF41B
:108AB00003AF9A8822F480621204120C9A80FBE6BB
:108AC0000023182203608270392243604271012220
:108AD00083600272C3727047F8B50468C4F30D0472
:108AE00005460E4604B32F682EF02CF9092840F0F5
:108AF0008880454C236923F440732361236943F440
:108B000000732361236943F0010323613E602EF06B
:108B100019F92369092823F00103236171D12B6816
:108B200004332B600020F8BD384B394A93422BD9CF
:108B300002F58042934226D902F5804293422AD917
:108B400002F58042934228D902F58032934226D919
:108B500002F50032934224D902F50032934222D921
:108B600002F50032934220D902F5003293421ED919
:108B700002F5802293421CD9B3F1016F1BD305206B
:108B800003F09AFDFBE708242EF0DCF8092814D046
:108B90004FF0FF30F8BD1024F6E71824F4E7202446
:108BA000F2E72824F0E73024EEE73824ECE740240D
:108BB000EAE74824E8E75824E6E7134F3B6923F443
:108BC00040733B613B6943F400733B613B6923F0B5
:108BD000F8033B613B6943F002031C433C613B6982
:108BE00043F480333B612EF0ADF83B6923F0020380
:108BF0003B613B69092823F0F8033B613FF473AF05
:108C0000C6E76FF00100F8BD003C024000400008DC
:108C1000FF3F0008F8B504460D468E180027B54200
:108C200001D12069F8BDE368591CE160234415F8BF
:108C3000012B1A720429F2D1206918B9A1682046C3
:108C4000FFF74AFF2061E760E9E700BF014B1868C2
:108C500005F046BB58200020F8B5057B466903683F
:108C60001F2D29D9A5F120045F682021A1400F42C2
:108C70002A4613D01022A240D960DA605A68E24036
:108C8000D10703D5012202FA04F4DC600446304621
:108C900005F0B2FA227B23681F2A20D9A2F1200016
:108CA00008215A688140114200D0D96004225968D5
:108CB00082400A4221D1F8BD20211C68A9400C4203
:108CC0002A460CD01022AA4099609A601A68EA409D
:108CD000D207DBD5012202FA05F59D60D6E708210F
:108CE00018689140014200D099600421186801FA87
:108CF00002F2024203D09A60F8BDDA60F8BDF8BD16
:108D000008B504F047FC40B12D2282710022C271E7
:108D10002021BDE8084005F05DBC08BD0B4B984222
:108D200006D0A3F5784398420DD04FF0FF3070473E
:108D30000022074B03EB02135A89013292B25A8187
:108D4000588980B270470122F3E700BF003001402C
:108D5000D453002008B540F2E93300E0A3B1028902
:108D6000013B12F0020F9BB2F8D089B2818140F230
:108D7000E93300E043B10289013B12F0010F9BB2DD
:108D8000F8D08089C0B208BDFFF7C8FFC0B208BDE7
:108D900070B583680446164613B11A689B885383DE
:108DA000606840F2E93301E0002B30D00589013BD7
:108DB00015F0020F9BB2F7D089B2818140F2E933FE
:108DC00000E023B30289013B12F0010F9BB2F8D0FF
:108DD000838940F2E93300E0EBB10189013B11F0F6
:108DE000020F9BB2F8D0B6B2868140F2E93300E0C0
:108DF0008BB10289013B12F0010F9BB2F8D083893D
:108E0000A36813B11A689B881383012070BDFFF714
:108E100085FF6068DDE7FFF781FFF1E7F0B587695F
:108E200083B0064617B13B68BA885A837069DFF889
:108E3000A4E08389C3244FF47A734FF0060C6D4687
:108E40004FF6FF710EF1010E03E0013B9BB28B4226
:108E500020D002899207F8D5A3B283814FF47A73A8
:108E600002E0A3B28B4215D00289D20703F1FF348E
:108E7000F7D5828992B20DB12A700135BCF1000F8D
:108E80000BD00CF1FF3CFF24BEF1000FE1D09EF8A7
:108E90000040D7E7FFF742FFB76917B13B68BA88D0
:108EA0001A839DF805009DF801509DF802109DF869
:108EB00003409DF804209DF8063041EA052143EA6D
:108EC000002342EA0422012031877287B38703B06E
:108ED000F0BD00BF90FE0308F8B584894FF6FF7619
:108EE0004FF47A7433B319B30F78013101E0B4420F
:108EF00018D00589013CAD07A4B2F8D5BCB2848175
:108F00004FF47A7402E0BCB2B4420BD00589ED078D
:108F100004F1FF37F7D58589ADB20AB1157001327A
:108F2000013BDFE7FFF7FAFE003018BF0120F8BD74
:108F3000FF27DEE70120F8BD427A02B9704710B57D
:108F400004460368406804F10A01984700236372ED
:108F500010BD00BF437A5A1C0344D2B242729972C8
:108F6000037A934200D802B9704710B504460368EB
:108F7000406804F10A0198470023637210BD70B580
:108F8000448806460D46C4F30B04224600212846B9
:108F900036F0DFFE33690A4A934209D3094A934205
:108FA00006D2224628461946BDE8704035F0D6BDA7
:108FB00023B121462846BDE87040184770BD00BF68
:108FC0001806000816070008064B07498B4202D313
:108FD0000023184670471A88C2F30B029042F8D05B
:108FE0001433F3E79001000818060008024A1368DA
:108FF00023EA000010607047F43F0020F8B5174DD9
:109000002B78A52B28D16B78BE2B25D1022229469F
:109010004FF6FF70FFF7E0F9114FAC1C22884AB100
:10902000A618BE4218D2052A16D92146FFF7D4F950
:109030003446F3E721460222FFF7CEF90222A118B7
:10904000FFF7CAF90634074B641B1C8041F60F5327
:10905000C31A58425841F8BD0020F8BD004000082E
:1090600000800008BE3500202DE9F04FDFF84C915C
:109070004D4F8BB00326A7EB09071822002104A847
:1090800036F067FE494BCDF8109005971A69002A13
:1090900004DA474A5A6002F188325A6001228DF898
:1090A0002420F322DA60434B434C1B88ADF8003098
:1090B0000222694604A8FFF7ADFD022269464FF679
:1090C000FF70FFF789F9DFF8F8A080464FF0000B3A
:1090D000544539D30AAC002524F8245D02222146E8
:1090E00004A8FFF797FD022221464046FFF774F9D6
:1090F00040BAC043ADF80800022202A904A8FFF755
:1091000089FD079878B106ABC0F1040229461844DE
:1091100036F01FFE089818B9069904A8FFF7DCFC82
:109120000023089007939DF82430089A23B11F4923
:109130000B6943F000430B61013E2DD0002A9CD106
:10914000FFF75CFF50B32CE065888DF80DB0C5F3D8
:109150000B05AB1DADF808302388C3F30B02ADF847
:109160000A201B0B062202A904A88DF80C30FFF779
:1091700051FD062202A94046FFF72EF9616880469C
:109180002A4604A8FFF746FD616840462A46FFF7D5
:1091900023F9143480469BE7002AD1D0052003F040
:1091A0008BFA0BB0BDE8F08F00800008003C024055
:1091B0002301674597FE030890010008004000085E
:1091C000180600080378202B024600F10100F9D0B0
:1091D000092BF7D02D2B2CD02B2B03BF5378B7EEB8
:1091E000000A0246B7EE000AA3F13001C8B209280E
:1091F0009FED467A10D8F2EE046A07EE901AF8EE68
:10920000E77A12F8013FE7EE267AA3F13001C8B2FF
:109210000928B0EE677AF0D92E2B4CD003F0DF038B
:10922000452B0BD0F7EE007A67EE276A20EE260A70
:1092300070475378BFEE000A0246D5E710B4517864
:109240002D2959D02B290ABF9178501C901C00243D
:10925000A1F13003092B53D8002303EB830301EB67
:10926000430310F8011FA1F13002092AA3F13003D2
:10927000F3D9B3F59A7F28BF4FF49A73072B42D9DD
:10928000DFED236A1A46F7EE007A083A072A67EEFE
:10929000A67AFAD803F007032BB1F2EE046A013B79
:1092A00067EEA67AFBD124B3C7EE276A5DF8044BBC
:1092B00020EE260A70475378A3F13001C8B209287E
:1092C00002F10102AAD8F2EE046AF0EE665A07EE45
:1092D000901AF8EEE77A12F8013F87EEA66AA3F13A
:1092E0003001C8B2092866EEA56A37EE067AEED9D3
:1092F00094E767EE276AD9E7901C91780124A7E7E5
:10930000F7EE007ACFE7F7EE007AC5E7000000003D
:1093100020BCBE4CB5EEC00ADFED317AF1EE10FA9A
:10932000CCBF30EE270A30EE670ADFED2E7A20EE52
:10933000270A30B5FDEEC07A87B017EE904A054691
:1093400084EAE470002303A9A0EBE4700193009386
:10935000029331F022FF002CACBF20232D2303A861
:109360008DF8003034F0BCFC012803A924D0022879
:109370002DD0032805BF3023684668468DF801309C
:1093800036F0EFFC684634F0ABFC0338C4B222463A
:109390006946284636F01CFD00232B55284634F03C
:1093A0009FFC2E22431C2A540DEB0401E81836F0D2
:1093B000F5FC284607B030BD302368468DF80130F3
:1093C0008DF802308DF8033036F0CBFCDAE730232D
:1093D00068468DF801308DF8023036F0C2FCD1E7D6
:1093E0006F12033A00007A442DE9F0410646154613
:1093F0000846B6FBF2F43CB905FB1464124B1B5D46
:1094000000F8013BBDE8F081B4FBF2F767B90E4B01
:1094100005FB174705FB1464DA5D00F8012B1B5DA3
:1094200000F8013BBDE8F081B7FBF2F8B8F1000F9E
:1094300002D04046FFF7D8FF05FB1878024B13F81F
:10944000082000F8012BE3E7BC340408104B2DE999
:109450003048D3E9004554EA05020BD10346012206
:1094600000201871587198719A70DA7018801881FC
:10947000BDE83088074B1A6814EB020B45F1000C6D
:109480005A466346FEF722FE0120BDE8308800BF41
:109490008823002098A90020F0B402888578154F11
:1094A000C37804794179A2F2B27202F0030606EBA6
:1094B0004606013D05EB8605013B37F815608579C9
:1094C000008940F2B557920807FB0232931903EB6B
:1094D000430304EBC303C3EB031301EB8303C3EBAD
:1094E000031305EB830300214FF47A72C2FB0301DF
:1094F000F0BC704730FE0308FAB170B48E18044611
:1095000003E0101A14D1B14214D014F8012BA2F1C7
:109510004103192B11F8013BA3F1410598BF2032FB
:10952000192D03F12000ECD9D01A01D1002BEAD17A
:1095300070BC7047002070BC70471046704700BF79
:109540004FF0FF32FFF7D8BFA0F16103192B98BF8E
:1095500020387047A0F14103192B98BF2030704785
:10956000202805D0093804288CBF0020012070472E
:1095700001207047613819288CBF002001207047F6
:10958000413819288CBF0020012070473038092845
:109590008CBF002001207047A0F13003092B07D9B0
:1095A00020F02000413819288CBF0020012070478E
:1095B0000120704730B402681146531C036011F853
:1095C000024B0160D31C517803609378151D056030
:1095D0001B0443EA0123D078234343EA006030BCF4
:1095E000704700BF0368591C1A46016012F8021B3D
:1095F0000260587841EA0020704700BF03685A1C97
:1096000002601878704700BF38B5044600681546F8
:1096100035F0A4FA22682A44226038BD036810B4E9
:109620000A0E5C1C04601A7003680A0C5C1C04605F
:109630001A7003680A0A5C1C04601A7003685A1CDA
:10964000026019705DF8044B704700BF036810B4E6
:109650000A0A5C1C04601A7003685A1C02601970C4
:109660005DF8044B704700BF03685A1C026010B4D9
:10967000197003680A0A5C1C04601A7003680A0CFB
:109680005C1C04601A700368090E5A1C0260197091
:109690005DF8044B704700BF03685A1C02601970E4
:1096A0000368090A5A1C0260197070472DE9F047D7
:1096B000002488B080460F461E46A14605AD531CC7
:1096C0000393117839B3252933D1931CCDF8109029
:1096D0000393507830284ED04FF0000AA0F13003A9
:1096E000DBB2092B42D96C2819D0642800F0938092
:1096F00024D825281CD063D9582876D063281BD1BC
:1097000031784046B847039A531C039311780436C6
:1097100001340029D7D1204608B0BDE8F087039B6B
:109720005A1C03921B78642B7CD02AD8252B54D149
:10973000252140460134B847039AC0E7732833D047
:1097400044D975284FD106F1040E30682B4600220B
:109750000A217646FEF782FC049A00955346394664
:109760004046FEF76DFD039A0444A8E704AA03A946
:1097700031F0F0FCB7E7D31C039390784FF0010A67
:10978000ACE7732B10D05BD9752B3AD0782B96D1E0
:10979000A3F15802B2FA82F2306852092B46102126
:1097A0000436FEF75BFCD7E73368049A009339462A
:1097B00000234046FEF744FD04360444039A7EE746
:1097C0000028B9D1204608B0BDE8F0876E28B3D193
:1097D000039A336804361C6071E72AD9582BD7D016
:1097E000632B8DD06BE77828A6D1A0F15802B2FA8E
:1097F00082F2306852092B461021FEF72FFC043606
:10980000AAE706F1040E30682B4600220A217646AC
:10981000FEF724FCA0E7331D306829461E46FEF7FC
:10982000EFFB99E7331D306829461E46FEF7E8FB3B
:1098300092E7002B7FF443AF204608B0BDE8F087E5
:109840006E2BC6D03BE700BF0EB400B584B005ABAD
:10985000019053F8042B0649039301A8FFF726FF54
:10986000019B00221A7004B05DF804EB03B070474E
:10987000358200082DE9F047484BB3F90C708CB0E5
:109880000646002F56D13D463C460A8840F2B17349
:109890009A4203D98B78581E0B282FD90023012018
:1098A0001946ADF824308DF828308DF829308DF820
:1098B0002A30ADF82C309C469A4699461A4698466E
:1098C00086468DF826008DF827000346002CACBF95
:1098D0002B242D24049107950697CDF80CC0CDF8C4
:1098E00008A0CDF80490CDF800E0304605942C494E
:1098F000FFF7AAFF40460CB0BDE8F08791F803E0FF
:109900000EF1FF301E28C9D891F80490B9F1170F55
:10991000C4D891F805A0BAF13B0FBFD891F806C0A2
:10992000BCF13B0FBAD80989B1F57A7FB6D24FF0B6
:109930000108CBE71B4C84FB0734E319FC17C4EB8D
:109940006314C4EB0415A7EB85052DB2002D084662
:10995000B8BF6D42FFF7A0FD4FF47A720023804636
:10996000894634F067FE3C2307FB03074FF47A7205
:1099700000234046494634F05DFE24B24FF47A712C
:1099800092B20023C1FB072309A884EAE477FEF71B
:109990009DFBA7EBE47709A977E700BF381F0020FC
:1099A000E4340408898888880FB430B583B006ABE6
:1099B0000A490B4853F8042B096800680193FFF724
:1099C00075FE084C0546206804F076FC0028FAD0A5
:1099D000284603B0BDE8304004B07047643400202E
:1099E0006834002058200020DFED2B7AB4EEE70A1F
:1099F000F1EE10FA4ADDDFED296A9FED297A01E0E8
:109A0000B0EE670AB4EEC70AF1EE10FA70EE667AAD
:109A1000F6DC9FED247AF4EEC77AF1EE10FA38D531
:109A2000DFED1E6A9FED207A01E0F0EE407AF4EE61
:109A3000C77AF1EE10FA37EEA60AF6D4DFED1B7AFC
:109A4000B4EEE70AF1EE10FA14DDDFED137A37EE2B
:109A5000C00A60EE006A9FED166A9FED167ADFED90
:109A6000167AA6EE867A20EE266AE6EE877AA6EECB
:109A7000270A7047DFED117AB4EEE70AF1EE10FA2B
:109A800044BFDFED087A37EEC00AE2E7F0EE407A35
:109A9000BFE7B0EE670AD1E7DB0F4940DB0FC940F3
:109AA000E4CB1641DB0F49C0E4CB16C1DB0FC93F45
:109AB00092E741B99730083C15A82ABEDB0FC9BF11
:109AC00080EAE073A3EBE0738B4205DB002801DD45
:109AD000401A704702D17047002070470844704711
:109AE00009B909E0194690FBF1F301FB130308469D
:109AF000002BF7D1084670470146FBE7F0EEC07A2D
:109B0000B0EEE07AB4EEE77AF1EE10FAB4BFB0EE60
:109B1000676AB0EE476AB5EE406AF1EE10FA46D0D9
:109B2000B4EEE77AF1EE10FA8CBFF0EE675AF0EE81
:109B3000475AC5EE866A9FED1F3A9FED1F6A9FED5B
:109B40001F4A9FED1F5ADFED1F3ADFED1F4ADFED81
:109B50001F5AA6EEC36AE6EEA34AA6EE864AB7EE01
:109B6000006AA6EE845AA6EEA46AE6EE855AC5EE11
:109B7000866AB4EEE77AF1EE10FA48BFDFED147AA8
:109B8000F5EEC00A48BF77EEE66AF1EE10FA48BF7C
:109B9000DFED107AB5EEC00A48BF77EEE66AF1EE67
:109BA00010FA48BFF1EE666AB0EE660A7047DFED64
:109BB000076ADEE739094E3DE3B59E3E88FA163E58
:109BC00045FE7F3F99FB243F69A2163EA7DFA834DC
:109BD000DB0FC93FDB0F4940DFED317A30EE277AEA
:109BE000FDEEC76A16EE903A2033402B02D99FED66
:109BF0002D0A7047B4EEE70AF1EE10FA4DDD9FED45
:109C00002A6ADFED2A6A01E0B0EE677AB4EEE67AFE
:109C1000F1EE10FA77EE467AF6DC9FED257AF4EE57
:109C2000C77AF1EE10FA35D5DFED1F6A9FED217A84
:109C300001E0F0EE407AF4EEC77AF1EE10FA37EE7A
:109C4000A60AF6D4DFED167AB4EEE70AF1EE10FAC2
:109C50001BDCDFED197AB4EEE70AF1EE10FA44BF2F
:109C6000DFED137A37EEC00A60EE006A9FED136AEB
:109C70009FED137ADFED137AA6EE867A20EE266A40
:109C8000E6EE877AA6EE270A7047DFED0F7A37EE09
:109C9000C00AE9E7B0EE670AD4E7F0EE477ABCE71E
:109CA000DB0FC93F00000000DB0FC940E4CB1641C9
:109CB000DB0F49C0E4CB16C1DB0FC9BF92E741B946
:109CC0009730083C15A82ABEDB0F4940FDEEC07A4C
:109CD00017EE903A2033402B51D8DFED2D7AB4EEB9
:109CE000E70AF1EE10FA50DDDFED2A6A9FED2A7ADD
:109CF00001E0B0EE670AB4EEC70AF1EE10FA70EEBA
:109D0000667AF6DC9FED257AF4EEC77AF1EE10FA6A
:109D100038D5DFED206A9FED227A01E0F0EE407A3F
:109D2000F4EEC77AF1EE10FA37EEA60AF6D4DFEDBC
:109D30001D7AB4EEE70AF1EE10FA1BDCDFED1A7AB9
:109D4000B4EEE70AF1EE10FA44BFDFED147A37EE15
:109D5000C00A60EE006A9FED156A9FED157ADFED8F
:109D6000157AA6EE867A20EE266AE6EE877AA6EEC9
:109D7000270A7047DFED067A37EEC00AE9E79FED64
:109D80000E0A7047B0EE670AD1E7F0EE407AB9E705
:109D9000DB0F4940DB0FC940E4CB1641DB0F49C064
:109DA000E4CB16C1DB0FC93FDB0FC9BF92E741B956
:109DB0009730083C15A82ABE0000000007EE901A54
:109DC000F8EE677A9FED837A27EE800A20EE070A85
:109DD000FDEEC07A17EE903A2033402B00F28C80D3
:109DE000DFED7D7AB4EEE70AF1EE10FA40F3E88099
:109DF000B0EE407A9FED796ADFED796A01E0B0EE6E
:109E0000677AB4EEE67AF1EE10FA77EE467AF6DC8F
:109E10009FED747AF4EEC77AF1EE10FA40F1CD803E
:109E20009FED6E6ADFED706A01E0F0EE477AF4EEC6
:109E3000E67AF1EE10FA37EE867AF6D4DFED6B7A39
:109E4000B4EEE77AF1EE10FA51DCDFED697AB4EEA8
:109E5000E77AF1EE10FA44BFDFED627A37EEC77AA7
:109E600027EE076ADFED635ADFED637ADFED636AA1
:109E70009FED635AE6EE257A67EE065AE6EE276A0C
:109E8000F7EE007AA5EEA67AF0EE675AE7EE055AED
:109E9000E7EE457A87EEA55ADFED547A30EE277A61
:109EA000FDEEC76A16EE903A2033402B29D99FED7C
:109EB000557AF6EE006AB7EE006AF7EE004AC4EE95
:109EC000A57A0023836143610362C36180ED045A74
:109ED00067EEA66A27EE866A27EE877AC0ED006AEB
:109EE000C0ED026A80ED016A80ED037A7047DFED14
:109EF0003A7A37EEC77AB3E7B7EE005AF0EE455A32
:109F0000CAE7B4EEE70AF1EE10FA5FDD9FED336ABF
:109F1000DFED336A01E0B0EE677AB4EEE67AF1EE97
:109F200010FA77EE467AF6DC9FED2E7AF4EEC77AD9
:109F3000F1EE10FA47D59FED296ADFED2B6A01E0BB
:109F4000F0EE477AF4EEE67AF1EE10FA37EE867A22
:109F5000F6D4DFED267AB4EEE77AF1EE10FA27DCDC
:109F6000DFED237AB4EEE77AF1EE10FA44BFDFEDCD
:109F70001D7A37EEC77A27EE076ADFED1E4ADFED5E
:109F80001E6ADFED1E7AE6EE246A67EE064AE6EE0A
:109F9000267AB7EE006AA4EEA77AF6EE006A36EEED
:109FA000476AF8EE007A27EE277A66EE266A84E79B
:109FB000DFED097A37EEC77ADDE7B0EE677A3DE785
:109FC000F0EE407A24E7B0EE677AC2E7F0EE477A27
:109FD000AAE700BF27D4D236DB0F4940DB0FC940C8
:109FE000E4CB1641DB0F49C0E4CB16C1DB0FC93F00
:109FF000DB0FC9BF92E741B99730083C15A82ABECC
:10A00000F304353F0000008070B406688E4217D913
:10A010000139751E002311F8014F0822634013F027
:10A02000800F4FEA430318BF83F0D503013ADBB238
:10A03000F5D18D42EFD1721C0260337070BC704755
:10A040000023F8E710B44C09012250F8243001F045
:10A050001F0102FA01F10B4340F824305DF8044B74
:10A06000704700BF4B0901F01F0150F82320012366
:10A0700003FA01F1114214BF18460020704700BFD7
:10A08000F0B4114E114F12481249134B134D144C9A
:10A090000A2232707A60022640F22E424FF4FA67AA
:10A0A0000E7202822D2140F2A462012647824020D6
:10A0B000EE7020821972197583F820105A81DA82A5
:10A0C0005A84F0BC704700BF1053002018350020A0
:10A0D000287F0020645B0020C4430020F052002051
:10A0E000905B0020074A084B10781B78074A834290
:10A0F00096BFC31AC3F180030020126818441044AD
:10A10000704700BF28410020A54000200C530020CC
:10A11000064A074B10781B7883428ABFC3F180033D
:10A12000C01AC018C0F17F00704700BF284100204E
:10A13000A540002030B5134C237883B01BB9012013
:10A14000237003B030BD1049052200230D688DF83F
:10A1500004208DF8053000BFA86804F0F3FA6A46C1
:10A1600001A902236868FEF7B7FEA86804F0F0FAB8
:10A1700000BF9DF8013003F0010383F0010023705C
:10A1800003B030BD05540020C053002070B5064C0C
:10A190000646256803E023685B1BB34203D8FFF73C
:10A1A000C9FF0028F7D070BD98A90020F0B51F4C5A
:10A1B00083B0277800234FF0030E00930E46154618
:10A1C0008DF804308DF800E06FB3030E8DF8013088
:10A1D0000DF10203010C020A9870197006205A70E2
:10A1E000FFF7D4FFE8B100BF114F3B68986804F057
:10A1F000A9FA23783A68002B14BF05230423694683
:10A2000050680022FEF768FE3B683246002158681D
:10A210002B46FEF761FE3B68986804F099FA00BF90
:10A22000284603B0F0BD0DF10103D3E7045400202C
:10A23000C053002038B504460D4600BF806804F0C6
:10A2400081FA29466068FEF785FDA06804F080FA6F
:10A2500000BF38BD2DE9F04F89B0B2F1000A02907D
:10A260000491039340F3C5800B46002201EB8A0161
:10A2700053F8040B8B420244FAD1039B0592002B46
:10A2800000F0AF80059B002B7CD05E4B059A1B68CD
:10A29000DFF8889100920099DAB25118B1F5807F09
:10A2A0008CBFC2F58072009A0192574A92689A4216
:10A2B00040F28280554A1178002206928DF81C20C7
:10A2C00002228DF81820002960D01A0E8DF819206E
:10A2D0000DF11A021C0C190A9370147051700620AB
:10A2E000FFF754FF0621D9F80000FFF7A3FF484A03
:10A2F0000123137000BFD9F80030986804F022FAE7
:10A30000424BD9F800201B785068002B06A90CBFDF
:10A31000042305230022FEF7DFFD0024049D029E96
:10A32000019FA34629684FEA840800220B460134A6
:10A3300071B1B9422DD2D9F8000031684068FEF7FA
:10A34000CBFD2A68336813443360BF1AC5F800B0E8
:10A35000A24505F1040506F10406E3D1D9F8003061
:10A36000986804F0F5F900BF264B019900981B6826
:10A37000421A0092234A0B441360039A4AB3009A8C
:10A38000002A88D1059809B0BDE8F08F0DF11902B7
:10A39000A0E7029CD9F8003054F808105868002251
:10A3A0003B46FEF799FD54F808202B683A44DF1B22
:10A3B00044F808202F60D1E70598009C1549164AFB
:10A3C000001B0590059800230B70137009B0BDE8C1
:10A3D000F08F059B009A9B1A0593059809B0BDE87C
:10A3E000F08FFFF7A7FE00287FF44CAF039B059387
:10A3F000C8E7039C1CB9FFF79DFE0594C2E7002344
:10A400000593BFE70C5300200410002004540020E3
:10A410000554002028410020A5400020C053002002
:10A4200070B5104D104E2B7831788B4284B016D019
:10A430000E4A03921A4402928CBF0C46CA1A04A90F
:10A440008CBFC3F180020024012341F8102D02A823
:10A4500002220194FFF7FEFE002333702B7004B03C
:10A4600070BD00BFA540002028410020A84000206A
:10A47000F0B5124B9D6885B00DB905B0F0BDED0A81
:10A4800014D0002704AE7C196410E0021022694643
:10A49000FFF78CFE0F2809DD6B4653F8042B0132C1
:10A4A0000AD1B342F9D12546AF42ECDBFFF7B8FF42
:10A4B000034BED021D60E0E7671CF5E70410002088
:10A4C0000C53002070B5194C194D23782978994206
:10A4D00084B027D0174A03921A44029234BF0E4622
:10A4E000CA1A04A934BFC3F180020026002341F830
:10A4F000102D02A802220196FFF7ACFE2378184423
:10A50000C0B203062B7848BF80F0800083422070E1
:10A5100002D0002004B070BD002301202B702370F6
:10A5200004B070BD012004B070BD00BFA540002084
:10A5300028410020A840002010B50C4C45F208200E
:10A54000FFF724FE20680621FFF774FE084B206801
:10A550000122C7211A70FFF76DFE06480649074A17
:10A56000002303700B70136010BD00BFC0530020A8
:10A570000554002028410020A54000200C53002055
:10A58000F0B55FEA930E33D000F1100601F110052B
:10A5900002F11004774616ED046A55ED044A56EDB3
:10A5A000026A15ED025A16ED037A55ED035A56ED7F
:10A5B000017A26EE246A66EE856A04ED046A15EDDA
:10A5C000016A44ED026A27EE257A67EE867A013F3A
:10A5D00004ED037A44ED017A06F1100605F1100549
:10A5E00004F11004D7D14FEA0E1420442144224430
:10A5F00013F003030BD000EB8303F0EC017AB1EC12
:10A60000017A67EE877A8342E2EC017AF5D1F0BDF8
:10A61000144B984224D003F58063984220D00388DD
:10A6200023F040031B041B0C0380038823F0380332
:10A630001B041B0C59B141F48071002991FAA1F25D
:10A64000B2FA82F108BF4FF0FF310139C900194356
:10A6500089B2018003889BB243F0400303807047B6
:10A660004908DCE7003800400C4B984213D0A3F5B2
:10A67000806398420FD003F5804398420BD003F5D6
:10A680008063984207D003F58063984203D0044B5F
:10A69000186840087047024B186870470004014072
:10A6A00074820020F0B5774B774A87B019689142E1
:10A6B00000AF00F0DB800023744A3B607B601368CE
:10A6C00043F48033136003E03B68B3F5A04F09D037
:10A6D000136803F400337B603B6801333B607B68A5
:10A6E000002BF1D0694B1B6813F4003318BF012312
:10A6F0007B607B68012B7BD0654D644B654AEA60CB
:10A700006549586F654A0860AA605E6B644C654A8B
:10A71000654826F080065E635E6F46F080765E6771
:10A72000196B0C431C63596B5963996B9963196CD2
:10A7300041F05B5141F47B1141F41F6141F00F0185
:10A740001964596C07F118040A4348F2FF715A64FE
:10A7500044F8101D002621460123FB733E737E73CF
:10A76000BE732CF0B1FB21464FF6FF734F48BB6020
:10A770002CF0AAFB4FF6FF7321464D48BB602CF02E
:10A78000A3FB21464B482CF09FFB21464A482CF066
:10A790009BFB214649482CF097FB214648482CF06A
:10A7A00093FB214647482CF08FFB214646482CF06E
:10A7B0008BFB20462CF060F9444B454C1B68BA6873
:10A7C00044484549A4FB03439B09A0FB0202013B0B
:10A7D000920CB3F1807F0A6007D2404AF020072133
:10A7E000536085F82300966011601C37BD46F0BDAC
:10A7F000264B3B4D1A6C3B4842F080521A642C6841
:10A800004268816844F440442C609C689C609C6869
:10A8100044F400449C609C6844F4A0549C6000682C
:10A82000120642EA801242F48002490842F0100205
:10A83000013942EA01425A601A6842F080721A6095
:10A840001A689201FCD52849104A40F20570086048
:10A85000996821F003019960996841F002019960BB
:10A86000936803F00C03082BFAD145E700221A6025
:10A8700062B61E4B1B6883F308881D4B1B68984704
:10A88000FEE700BFFCFF0120EFBEADDE0038024056
:10A8900000ED00E00005FA053892002000000008F5
:10A8A000FF916700335F0700000002400004024090
:10A8B00000080240000C0240001002400014024058
:10A8C00000180240001C0240002002407482002058
:10A8D000D34D621083DE1B439CA9002010E000E0F2
:10A8E0000070004000000020003C02400000FF1FFC
:10A8F0000400FF1F08B5054B1B6803B19847044BC4
:10A90000044A1A6072B6FDF76BFE00BF9045002046
:10A91000FCFF0120EFBEADDE08B5034B1B6803B1A1
:10A92000984772B6FDF75CFE904500202DE9F04F88
:10A930007A4C54F8204083B0002C00F0EA80D4F820
:10A940006090B9F1000F00F0E680D9F81050D9F806
:10A950000470734EA16004F166012660616104F227
:10A9600066264FF40071A661E1602161A765A046EB
:10A970004DB3DFF8B4C14FF0000E61464E68B542EA
:10A9800001F11C0106D00EF1010EBEF1100FF5D140
:10A990004FF0000ECEEBCE0E0CEB8E01DFF884C133
:10A9A0000E69DCF830E04FF00C0A4EEA060E461C49
:10A9B000CCF830E081F818A04E76D9F80810E163A1
:10A9C0000437676565630546D9F80C001F461646CF
:10A9D00000283CD0DFF850C1002163465A689042FD
:10A9E00003F11C0303D001311029F7D10021C1EB81
:10A9F000C1010CEB81014B4B0A69186BDFF82CE1AC
:10AA0000104318630B200876681C4876186B0243C5
:10AA100099F81F001A63830991F80DC08DF805306D
:10AA2000002201234C61C1F808E001A88DF806203E
:10AA30008DF807308DF804C02BF0D6FFA36DD9F840
:10AA40000810D9F80C20A26304332164236594F81C
:10AA5000650002F09FFD824694F8640002F09AFDC2
:10AA6000834699F81C00002850D1380739D4B20722
:10AA70000ED5BAF1000F0BD00B226B1C8AF8062002
:10AA80008AF80730504699F81D20222102F0EAFB8F
:10AA9000F30716D4E36B83B999F81E208DF80420D0
:10AAA00099F820208DF8063001A8930901228DF82D
:10AAB00005308DF807202BF097FF404603B0BDE826
:10AAC000F08FBBF1000FE5D001350C238BF8075058
:10AAD0008BF80630584699F81D20222102F0C2FB5F
:10AAE000D8E70135EDB2BAF1000F04D00B238AF894
:10AAF00007508AF8063017F0100F50460CBF12218D
:10AB0000022199F81D2002F0ADFBC3E731F0F6FEFB
:10AB1000ABE7A046D1E7C846CFE700BF70340020BE
:10AB20009CFE030800380240101B0020598C0008CE
:10AB300000B97047F0B595B0054626F0FBF8B24E67
:10AB4000C368026832600446002B00F03781284653
:10AB500002F020FDAD4B186118B12922002382714B
:10AB6000C371227A2A2102F07DFB306802F070FF67
:10AB700031F0C4FE3268138823F001031B041B0C60
:10AB800013801046FFF770FDA14B984200F2188128
:10AB90000025DFF8B4E29F4F13889F4905F1010CAF
:10ABA000B0FBFCF04FF0030CB0FBF1F081B2B1FB55
:10ABB000FCF1AEF800104900398098498A429BB2F6
:10ABC00000F0088101F580618A4200F00381B2F152
:10ABD000804F00F0FF80A1F580318A4200F0FA80BA
:10ABE00001F580618A4200F0F58001F580618A42BA
:10ABF00000F0F0808A498A4200F0018101F580610D
:10AC00008A4200F0FC8023F44071844B89B29A425E
:10AC10001180D062158500F0EF80824B9A4200F0DF
:10AC2000EB8001219182E27960200023ADF80000E1
:10AC30009007ADF80230ADF804300293ADF80C3057
:10AC4000ADF80E30ADF81030ADF8123040F1C680DE
:10AC500012F0010F0CBF1A4608220423ADF80E2093
:10AC6000ADF8043000233068617902936A4602F03F
:10AC7000C1F8607933680C2816D8DFE810F0F900C5
:10AC80001500150015000D00150015001500F00049
:10AC9000150015001500E7001A8B22F4006212045B
:10ACA000120C42F400621A83B3F844205E4D5F4FE9
:10ACB0006FEA42426FEA524292B2A3F844201A88E5
:10ACC00092B242F080021A80E279198C92074CBF4E
:10ACD00004220122824092B289B221EA020119843F
:10ACE000198C89B20A431A841A88514992B242F0E7
:10ACF00001021A80237D086B1C2202FB03534FF0D4
:10AD0000290E1A6900251043086383F818E05D7660
:10AD1000086B02430A635A7B5D619F6005A80123AB
:10AD20008DF814208DF816508DF815308DF81730E9
:10AD30002BF05AFEE3683F4F18463B602BF06AFF4A
:10AD40003868036823F0010303602BF063FF336866
:10AD5000627938680A9534331344069340F22A33F3
:10AD600009934FF4806322690B93334B0592079349
:10AD700040224FF4805305A908920C934FF480426F
:10AD80004FF440330E9510951195129513950D9231
:10AD90000F932BF013FF6379316828480C2B9CBF6D
:10ADA000274A32F813508B893A689BB21D438D8134
:10ADB0001368012143F010031360017015B0F0BD5A
:10ADC00000F1B77303F558531E49B3FBF1F3013B90
:10ADD0009DB2DEE623F070039BB20BE712F0010F89
:10ADE0000CBF002202224FF48073ADF80210ADF8C0
:10ADF0000C20ADF8103035E70023138611E71380DF
:10AE0000D06215850DE700BFC4740020381F0020F4
:10AE1000FF6BDC02BA74002000350C00000001401A
:10AE20000010004000040140101B00203D87000876
:10AE300000380240C0740020EC650020BC74002083
:10AE4000042C0408006CDC02B87400209A8B22F4F5
:10AE500000621204120C42F400629A8324E79A8B77
:10AE600022F008021204120C42F008029A831BE737
:10AE70001A8B22F008021204120C42F008021A8304
:10AE800012E7094B10B507281B68C8BF14381844CF
:10AE90000C46007E02F07EFB20B12146BDE810404A
:10AEA00003F05CBC10BD00BF9034002038B50C4BE3
:10AEB00007281B68CCBFA0F11404044623440546B0
:10AEC000187E02F067FB50B128220134C4718271F0
:10AED00031F032FD28460021BDE83840D1E738BDC9
:10AEE000903400200348D0F8AC3113B100F5D27093
:10AEF00018477047101B00200348D0F8903113B159
:10AF000000F5C47018477047101B00200348D0F8A4
:10AF1000743113B100F5B67018477047101B00204C
:10AF20000348D0F8583113B100F5A870184770479E
:10AF3000101B00200348D0F83C3113B100F59A7083
:10AF400018477047101B00200348D0F8203113B178
:10AF500000F58C7018477047101B00200348D0F88C
:10AF600004310BB1FC301847704700BF101B0020A4
:10AF70000348D0F8E8300BB1E0301847704700BF05
:10AF8000101B00200348D0F8CC300BB1C430184758
:10AF9000704700BF101B00200348D0F8B0300BB141
:10AFA000A8301847704700BF101B00200348D0F896
:10AFB00094300BB18C301847704700BF101B002035
:10AFC0000248836F0BB1703018477047101B002088
:10AFD0000248C36D0BB1543018477047101B002056
:10AFE0000248036C0BB1383018477047101B002023
:10AFF0000248436A0BB11C3018477047101B0020F1
:10B000000248836803B11847704700BF101B002037
:10B01000F8B5654C0601A7190546387A31F06EFC83
:10B020003B7A03F01F015B090122032B02FA01F2B4
:10B030006DD0042B66D0022B5CD0A3190135187992
:10B0400002F0A8FAEDB2074610B11223C571837160
:10B05000A319587902F09EFA10B11323C5718371B8
:10B06000A319987902F096FA10B11423C57183716F
:10B07000A5190A21EA79384602F0F4F8687902F055
:10B0800089FAEA790A2102F0EDF8A87902F082FA49
:10B09000EA790A2102F0E6F8A359444A934247D0DC
:10B0A000434A934250D0434A934259D0424A934232
:10B0B00062D0424A93426BD0414A93422CD03444EE
:10B0C000227BE2B901200222198801F4415141F4A6
:10B0D00045710A4302431A809A8B22F400621204DB
:10B0E000120C07219A8319821A8892B242F0400208
:10B0F0001A80F8BD334B596A0A435A629DE7002013
:10B100000246E1E72F4B19690A431A6195E72D4B77
:10B11000196A0A431A6290E702F564424FF400107C
:10B12000536A43F4001353622BF096FCA359C6E70D
:10B1300002F584324FF48050536A43F480535362D3
:10B140002BF08AFCA359BAE702F500324FF4804095
:10B15000136A43F4804313622BF086FCA359AEE7D5
:10B1600002F5FE324FF40040136A43F400431362C9
:10B170002BF07AFCA359A2E702F582324FF400507B
:10B18000536A43F4005353622BF066FCA35996E7CD
:10B1900002F568424FF48010536A43F480135362FF
:10B1A0002BF05AFCA3598AE7D45300200030014009
:10B1B00000380040003C0040003401400050014095
:10B1C0000054014000380240431C00F014812DE976
:10B1D000F04F4FEAC00808EB00039B00DFF8F4A231
:10B1E0005AF803B087B00AEB0304BBF1000F00F07C
:10B1F000FF8014330AEB03010022DBF804704AF8E5
:10B2000003204A608A60CA600346A5680190013342
:10B21000D4F80C90DBB2002D00F0EE801522EB711B
:10B22000AA71B9F1000F00F00081162289F80620FA
:10B2300089F807309BF80E0031F060FBBB8823F4DF
:10B2400040731B041B0CBB80284603F081FA484660
:10B2500003F07EFA1121284603F066F811214846D2
:10B2600003F062F80826642404E00A203CB102F0EE
:10B27000C1FD013C284603F0BDFA0028F5D0284660
:10B2800003F060FA0A2002F0B5FD284603F060FAE8
:10B290000A2002F0AFFD013EECD1484603F052FA1D
:10B2A0000A2002F0A7FD284603F04CFA0A2002F01B
:10B2B000A1FD284603F04CFA0A2002F09BFD484607
:10B2C00003F046FA019B08EB03040AEB84042846CA
:10B2D000637C002B0CBF12213221042201F0C2FF3B
:10B2E000637C002B0CBF122132214846042201F05E
:10B2F000B9FF704B9F4200F0B7806F4B9F4200F048
:10B30000BD806E4B9F4200F0A580BB8801996C4ABE
:10B310006C4C23F440731B041B0CBB803B8888449B
:10B320000AEB880A9BB243F001039AF810103B80A5
:10B33000BD8802A8002918BF14462BF09DFB049A73
:10B340006148B2FBF4F325F03F05A0FB02122D0487
:10B35000900C2D0C0543BD805C4C39884FF49672DF
:10B3600002FB00F284FB02409BB2D217002BC2EB1F
:10B37000A01221F0010108BF01230904013243F4A6
:10B380000043090C92B239803A84BB833B889BB25C
:10B3900043F001033B803B8823F4816323F00203E5
:10B3A0001B041B0C43F480634FF480423B803A81C2
:10B3B0003B8823F080031B041B0C3B809BF8103060
:10B3C0008DF808300024012302A88DF80B308DF889
:10B3D00009408DF80A402BF007FB9BF80F308DF8E1
:10B3E000083002A88DF809408DF80A402BF022FBA6
:10B3F00007B0BDE8F08F7047B9F1000F48D01622B2
:10B4000089F8073089F806209BF80E0031F076FAAB
:10B41000BB8823F440731B041B0C2846BB8003F03D
:10B4200097F9484603F094F918E79BF80E0031F0BD
:10B4300065FABB8823F440731B041B0CBB802846B1
:10B4400003F086F9484603F083F91121284602F0FB
:10B450006BFF07E71E4A136A43F4000313624FF4BD
:10B4600000002BF001FB50E7194A136A43F4001364
:10B4700013624FF400102BF0F7FA46E7144A136AF0
:10B4800043F4800313624FF480002BF0EDFA3CE7A5
:10B490009BF80E0031F032FABB8823F440731B0492
:10B4A0001B0C4846BB8003F053F9484603F050F9A3
:10B4B000D8E600BF0054004000580040005C004047
:10B4C000009F2400804F120083DE1B43D34D621087
:10B4D00000380240A03400202DE9F0410678012E0A
:10B4E00082B005464CD0022E52D1806841F08001D6
:10B4F00010B1046880886083686840F2E93402E033
:10B50000002C00F099800689013C16F0020FA4B2CD
:10B51000F6D089B2818140F2E93102E0002900F0E1
:10B520008B800489013914F0010F89B2F6D081892A
:10B5300081894FF0000C4FF47A714FF6FF764FF08F
:10B54000FF0E634502D129E0B14225D004890139BB
:10B55000A70789B2F8D5A0F80CE04FF47A7102E0A1
:10B56000B9B2B14218D00489E40701F1FF37F7D529
:10B570008489A4B20AB1147001320CF1010CE0E725
:10B5800090F904E0BEF1FF3F02D0BEF1030F0FDDE2
:10B59000002002B0BDE8F081FDF7C0FBAB68002BD6
:10B5A0005CD01A689B881383012002B0BDE8F0814B
:10B5B0004FEACE08DFF8ACC008EB0E070CEB8707AC
:10B5C00078680028E5D06C793A6264000025E4B21E
:10B5D000BC75F9757D76BE763B767E753D75838844
:10B5E000FA61990514D40388DA050CD44FF4805419
:10B5F00001E0013C28D003889B05FAD403889BB264
:10B6000043F48073038083889BB243F44073838048
:10B61000F0440CEB88024FF4805401E0013C13D05D
:10B62000537D002BFAD10CEB880898F8144084F075
:10B63000010002B0BDE8F0818DE80C00FDF76EFB63
:10B6400068689DE80C0073E7054A1388013370466B
:10B650009BB21380FFF7B8FD20469AE7012098E7D8
:10B66000BC350020A034002037B506236A460446C6
:10B670000D460C300321FFF72FFF024690B1B4F9BD
:10B680001A106846FCF7C2FE2880B4F91E100DF1AE
:10B690000200FCF7BBFEA880B4F91C1001A8FCF75F
:10B6A000B5FE6880104603B030BD07B5032301AA7C
:10B6B0000021FFF711FF9DF805309DF804001B02E3
:10B6C00043EA00439DF80600184303B05DF804FB0D
:10B6D00008B5FFF7EAFF014B586008BD381F00208E
:10B6E00008B5FFF7E2FF014B186008BD381F0020C6
:10B6F0002DE9F04F87B090F855300190002B77D1AD
:10B7000004AB0393374B1B7D002B00F0CC80019BD7
:10B71000354A10330293019B5B69934200F0EE813E
:10B7200032498B420CBF302138211A88019C029883
:10B7300022F040021204120C1A801A8892B222F0EF
:10B740003802114319801A8892B242F040021A80DE
:10B7500094F84E201A21FDF71BFB012002F04AFB52
:10B760006369214A934200F0908220498B4214BFC2
:10B77000082100211A88029822F040021204120CBB
:10B780001A801A8892B222F038021143198019885F
:10B79000039A89B241F04001198006234321FFF743
:10B7A0009BFE002800F0F3819DF810409DF8125098
:10B7B0009DF813309DF811109DF814009DF8152088
:10B7C00041EA042143EA0523019C1BB242EA00221C
:10B7D00063872187A2875BB2013300F0AD8107B098
:10B7E000BDE8F08F381F002000380040003C0040CA
:10B7F0001D09013D032D03F00F0300F23E82C04AF4
:10B8000032F8150040FA03F2D40740F136820124E1
:10B8100004FA03F3013B184032F05CFFB94BBA4A1B
:10B820005B5D184412EBC00500F027820023202145
:10B83000EB71A97152F83000B44A00F13F4303F5AF
:10B840007E039B0AD25C02F01F035209032A04FA0A
:10B8500003F300F02682042A00F01E82022A00F080
:10B860001682AB88049304A90023039105932BF05F
:10B870002BFB0199A64B41F80C3F284625F0F0F927
:10B88000AB88B3FA83F3C3F11F03012212FA03F367
:10B890003FF438AF9F490A6813430B609E4B1B7DF2
:10B8A000002B7FF434AF019B9C4A5B69934200F00C
:10B8B000FF819B498B420CBF302138211A88994C5B
:10B8C000994EDFF86C9222F040021204120C1A809A
:10B8D0001A8892B222F03802114319801A8801990D
:10B8E00092B2103142F0400202911A800846802242
:10B8F0006B21FDF74DFA8D48DFF838E24FF0960BDB
:10B900004FF0100C4FF47A75D9F80430C3F30803E4
:10B91000002B40F09681EFF31183002B40F09181D2
:10B920002168826800BF23689942F9D1376805FB16
:10B9300007F39B1AB3FBF7F305FB013101270091D5
:10B94000D9F80430C3F30803002B40F04181EFF332
:10B950001183002B40F03C812368816800BF22687E
:10B960009342F9D1D6F800A005FB0AF2521AB2FBB5
:10B97000FAF205FB0323009A9B1AB3F57A7FDFD313
:10B98000BBF1010BC0D1032268210298DFF8A0A10E
:10B99000FDF7FEF996236548DFF898C14FF01008CF
:10B9A0004FF47A759E46DAF80430C3F30803002B8F
:10B9B00040F02B81EFF31183002B40F026812168AA
:10B9C000826800BF23689942F9D1376805FB07F305
:10B9D0009B1AB3FBF7F305FB013101270091DAF85D
:10B9E0000430C3F30803002B40F0D580EFF311833C
:10B9F000002B40F0D0802368816800BF226893420A
:10BA0000F9D1D6F800B005FB0BF2521AB2FBFBF2EB
:10BA100005FB0323009A9B1AB3F57A7FDFD3BEF1AF
:10BA2000010EC0D1029D03226B2128467446764642
:10BA3000FDF7AEF90F2002F0DDF910226A21284649
:10BA4000FDF7A6F90F2002F0D5F922466C21284611
:10BA5000FDF79EF90F2002F0CDF9019C192194F811
:10BA600050202846FDF794F90F2002F0C3F9182260
:10BA70001B212846FDF78CF90F2002F0BBF910229C
:10BA80001C212846FDF784F90F2002F0B3F910229B
:10BA900037212846FDF77CF90F2002F0ABF901228F
:10BAA00038212846FDF774F90F2002F0A3F96369E5
:10BAB0001A4A934200F0FA80194FBB4214BF08277C
:10BAC00000271A8822F040021204120C1A801A88E9
:10BAD00092B222F0380217431F801A8892B242F0C5
:10BAE00040021A80012002F085F90B4A01231375E8
:10BAF000019B0A4A5B6993427FF412AE302114E63F
:10BB0000B4340408B034040860A70020A834040842
:10BB1000D9850008003C0140381F00200038004053
:10BB2000003C004098A900209CA9002010E000E003
:10BB300000ED00E094A90020019B93F93830013317
:10BB40007FF44DAE0A26322031F0F8F84FF4FA7542
:10BB500002F004F9044602F001F9001BB0F57A7F07
:10BB6000F9D3013DF4D1072030F04AFF4FF47A7544
:10BB700002F0F4F8044602F0F1F8001BB0F57A7F09
:10BB8000F9D3013DF4D1013EDDD1FEF7B3FE019BB7
:10BB9000B3F93A301FE6EFF3118988F31288816810
:10BBA0000368DB0344BFCCF8007081682368DCF8CD
:10BBB00000205FFA89F989F31188D6F800901A44B9
:10BBC00005FB09F35B1AB3FBF9F305FB023321E72D
:10BBD000EFF311888CF3128881680368DB0344BF9C
:10BBE000CEF8007081682368DEF800205FFA88F8DC
:10BBF00088F31188D6F800801A4405FB08F35B1A15
:10BC0000B3FBF8F305FB0233B5E6EFF3118288F3DB
:10BC1000128887680368D90303D50123CCF8003064
:10BC200087682368DCF80010D2B282F3118832688A
:10BC3000194405FB02F3DB1BB3FBF2F305FB0131F7
:10BC4000CBE6EFF311828CF3128887680368D9037F
:10BC500003D50123CEF8003087682368DEF8001092
:10BC6000D2B282F311883268194405FB02F3DB1B60
:10BC7000B3FBF2F305FB013160E601990D4B41F88E
:10BC80000C3F002024F0ECFF3AE5002172E50A4A5F
:10BC9000516C0B435364E4E5074A116B0B43136388
:10BCA000DFE5054A116C0B431364DAE5374608E714
:10BCB000302103E6D985000800380240F0B5C600FF
:10BCC00033189B00254DEA585468A28A83B092B27B
:10BCD0000192019A2B4412F4706F1CBF01221A7555
:10BCE000019B13F4E06F07460CD1A38A3E4423F472
:10BCF000706305EB86051B041B0C0022A3826A758A
:10BD000003B0F0BD238BA38823F480631B041B0CBA
:10BD1000A380019B9B05E8D423889805E5D423885C
:10BD2000D9050ED52388DA05FCD423889BB243F4C9
:10BD30000073238023889B05FCD43846FFF744FA20
:10BD4000D3E723889BB243F400732380A38823F4B2
:10BD500040731B041B0CA380C7E700BFA034002066
:10BD6000F0B5037A012B83B0014664D0022B68D171
:10BD7000036913B11A689B885383C86840F2E9339A
:10BD800002E0002B00F0AA800289013B12F0020FB2
:10BD90009BB2F6D0BB23838140F2E93302E0002B53
:10BDA00000F09C800289013B12F0010F9BB2F6D09B
:10BDB000838983894FF0060E4FF47A736E464FF6EF
:10BDC000FF74FF2703E0013B9BB2A3423CD00289F2
:10BDD0009507F8D587814FF47A7302E0ABB2A3429E
:10BDE00032D00289D20703F1FF35F7D5828992B2AA
:10BDF0000EB132700136BEF1010EE8D10B6913B1FC
:10BE00001A689B8813839DF800609DF801009DF8D7
:10BE100002509DF803209DF804409DF8053040EA4B
:10BE2000062042EA052243EA0423C88201200A834D
:10BE30004B8303B0F0BD90F90C00451C01D00328E2
:10BE400005DD002003B0F0BDFCF768FFD6E7C700B2
:10BE5000294E3A1806EB82025568002DF1D04C7B32
:10BE60006400E4B294754FF0000E06244FF03B0CD2
:10BE700082F817C082F819E093761476537582F829
:10BE800014E0AB88C2F820D09C05C2F81CD014D4B2
:10BE90002B88DA050CD44FF4805401E0013C21D00A
:10BEA0002B889B05FAD42B889BB243F480732B809C
:10BEB000AB889BB243F44073AB80074406EB870228
:10BEC0004FF4805401E0013C0CD0537D002BFAD19B
:10BED00006EB87073B7D002B95D0B2E7FCF71EFFF2
:10BEE000C86866E7054A138801339BB21380FFF7E1
:10BEF0006BF92046A6E700BFA0340020BC35002027
:10BF0000F0B583B0441C8DF8073001D0032802DD62
:10BF1000002003B0F0BDC700244E3B1806EB83039E
:10BF20005D68002DF4D04900C9B299750124002143
:10BF3000DA755C7699761C765C751975A9880DF1B1
:10BF400007028905DA611A6214D42B88DA050CD449
:10BF50004FF4805401E0013C1ED02B889B05FAD49D
:10BF60002B889BB243F480732B80AB889BB243F445
:10BF70004073AB80074406EB87024FF4805401E026
:10BF8000013C09D0537D002BFAD106EB87073C7D9D
:10BF900084F0010003B0F0BD054A138801339BB261
:10BFA0001380FFF711F92046B3E700BFA03400204B
:10BFB000BC35002030B40578012D09D0022D04D104
:10BFC00001F07F0130BCFCF7E3BE002030BC7047BD
:10BFD000134630BC0A46417990F9040090E72DE9F8
:10BFE000F04F4FF4807385B043838383C38300F1A4
:10BFF0000C050446322001F057FF1122002128468B
:10C00000FFF7D8FF602201212846FFF7D3FF642005
:10C0100001F04AFF02A920460027FFF725FB012374
:10C02000B946B8463E460193012E14BF1122122292
:10C0300000212846FFF7BEFF002E0CBF4FF0010B7A
:10C040004FF0FF3B4FF00A0A012202212846FFF77A
:10C05000B1FF142001F028FF02A92046FFF704FBDE
:10C06000BDF90A20BDF90C00BDF90810354B82421C
:10C070000BFB0299A8BF02468A42A8BF0A469A4211
:10C0800001FB0B880BFB007758DB012002F03CF929
:10C09000BAF1010AD8D10136022EC5D12A4B93FB41
:10C0A000F8F893FBF9F97022A3F58423002193FBA0
:10C0B000F7F7A4F81A80A4F81C90E7832846FFF746
:10C0C00079FF202201212846FFF774FF0022314624
:10C0D0002846FFF76FFF642001F0E6FE019B23B9BD
:10C0E0004FF480736383A383E383607E10B301F016
:10C0F00051FA054602F07EFBE0B135B12223002162
:10C10000AB71E971284602F00FF921460F4B41F857
:10C11000083F284624F0A4FD65B1AB88B3FA83F349
:10C12000C3F11F03012212FA03F303D008490A687E
:10C1300013430B60012005B0BDE8F08F002301938D
:10C14000A9E700BF01F0FFFF00D03B000B8400080F
:10C15000003C0140012248212CE70122582129E717
:10C160000220FCF71BBB00BF0220A7E50120FCF763
:10C1700015BB00BF0120A1E50020FCF70FBB00BFED
:10C1800000209BE51549164B16480A6810B48C68C8
:10C190001549B2FBF4F203FB02F30360D1F88820E7
:10C1A000124B134C42F47002C1F888201A68002028
:10C1B00042F001021A6098601A6822F0847222F438
:10C1C00080321A605C601A684FF0006422F48022AA
:10C1D0001A60D8608C605DF8044B70470000002046
:10C1E00040420F007482002000ED00E00038024061
:10C1F00010300024044B4FF4F0700A21022283E82F
:10C200000700FFF7BFBF00BF000000200B4B00225C
:10C2100010B4027203F5C074032102E0072A09DC9E
:10C220009979890702D51979815401329C4203F129
:10C230001803F3D15DF8044B704700BF6424040871
:10C240001A230370704700BF2C2202230270437030
:10C25000704700BF436A8269D154436A0169826BA7
:10C2600001338B4228BF00234362002A2FD0EFF313
:10C270001182502383F31288836B1968C9072CD469
:10C2800070B45E686EB9456A816A8D4217D0846960
:10C290000C44DC600ED9691A59608562002180F86F
:10C2A0005C10196841F00101D2B2196082F3118863
:10C2B00070BC70470469611A59608662EEE7012319
:10C2C00080F85C30D2B282F3118870BC7047826D06
:10C2D000D36843F08003D3607047D2B282F31188F1
:10C2E000704700BF426B10B462B1C36CC26844694E
:10C2F000D11A013B615C5DF8044B08BF1346C3646F
:10C30000C8B27047016A4369C4685B5C0131A142ED
:10C3100028BF114601625DF8044BD8B2704700BFD8
:10C32000836B13B190F85C007047836A406A181AF7
:10C33000B0FA80F040097047416A836A99420AD393
:10C34000CB1A816B026961B14968501E0B4483426C
:10C350000AD2C01A704702691144CB1A816B0029B6
:10C36000F2D1501EC01A704700207047436B43B192
:10C37000C26C5B6893422FBF981AC0689B1AC018A2
:10C380007047C269036A9A422FBFD01AC0688018EA
:10C39000C01A70470A4B30B503F1140493F900201A
:10C3A0005D78072AC8BF143A811804330D7313F857
:10C3B000025C855413F8012C0A76A342EED130BDFD
:10C3C000C4FE030803682DE9F041DF691FB13B4655
:10C3D000BDE8F0411847002A164611DD04460D4617
:10C3E0000E4400E023689B68204698470028F9D057
:10C3F000236815F8011B1B6820469847AE42F1D10F
:10C40000BDE8F08100233E213D220170427083701F
:10C41000C3707047152303701623C37017238371ED
:10C420002D234370322303713323C371704700BF40
:10C43000038A2DE9F0478589ADB21D4029D00F460A
:10C4400006464FF000484FF00009B5FA85F328FA88
:10C4500003F2D24391B21B3B15403182042B16D814
:10C46000DFE803F03129211903007B6A002B32D069
:10C4700003F1FF3A1FFA8AFAC7F824903C6A34B1F4
:10C4800023682046514698476468002CF8D1002D57
:10C49000DBD1BDE8F0873868716B036889B29847D3
:10C4A000002DD2D1F5E77868B16B036889B298475F
:10C4B000002DCAD1EDE7B868F16B036889B29847DF
:10C4C000002DC2D1E5E7F868316C036889B298475E
:10C4D000002DBAD1DDE7F36A1FFA83FACEE700BF79
:10C4E00030B50446806D61718389A26823F40053DE
:10C4F0001B041B0C838185B0A379009213F0040206
:10C5000030D04FF4805213F00203ADF8042056D11E
:10C51000ADF806304FF480630022ADF8083011F01A
:10C520000103ADF80C2028D1ADF80A3008238D079F
:10C53000694648BFADF80A302AF0DEFAA279A36D49
:10C54000D10724D412F0080F9A8A1BD122F00802D6
:10C550001204120C9A829A8992B242F400529A8181
:10C5600005B030BD13F00203ADF8042024D04FF421
:10C5700000551346ADF80650CEE70423ADF80A3057
:10C580000C23D4E792B242F008029A82E3E70D4905
:10C590008B420FD0A1F54C418B4209D00A498B4206
:10C5A000D0D102200121FEF76CFCA279A36DC9E76E
:10C5B0000120F7E70020F5E7ADF80630ACE74FF4CF
:10C5C0000053A5E7001001400048004010B50446A4
:10C5D000806DA160838923F400531B041B0C8381AD
:10C5E000A37984B013F00402009135D04FF4805247
:10C5F00013F00203ADF8042056D1ADF806304FF425
:10C6000080636279ADF80830D1074FF00003ADF8D0
:10C610000A30ADF80C3045BF0423ADF80A300823CA
:10C620000C236946920748BFADF80A302AF064FA35
:10C63000A279A36DD1071FD412F0080F9A8A16D1E0
:10C6400022F008021204120C9A829A8992B242F4E1
:10C6500000529A8104B010BD13F00203ADF804201B
:10C660001FD04FF400511346ADF80610C9E792B23F
:10C6700042F008029A82E8E70D498B420FD0A1F5FB
:10C680004C418B4209D00B498B42D5D1022001216C
:10C69000FEF7F7FBA279A36DCEE70120F7E70020B4
:10C6A000F5E7ADF80630ACE74FF40053A5E700BF5F
:10C6B00000100140004800402DE98048013085B05D
:10C6C000C3B203938B4D8C4F8C4C8D4E0A23029337
:10C6D0003220DFF8309230F031FB4FF4FA7A4FF02D
:10C6E000100C4FF47A70D9F80430C3F30803002B10
:10C6F00040F0C180EFF31183002B40F0BC8029682B
:10C70000A26800BF2B689942F9D1D7F800E000FB7E
:10C710000EF39B1AB3FBFEF300FB01314FF0010E49
:10C720000191D9F80430C3F30803002B40F087804F
:10C73000EFF31183002B40F082802B68A16800BFCB
:10C740002A689342F9D1D7F800B000FB0BF2521AD5
:10C75000B2FBFBF200FB0323019A9B1AB3F57A7F2D
:10C76000DFD3BAF1010ABED1039B002B40F0BD809C
:10C770004FF47A7ADFF88C9150464FF0100CD9F8CC
:10C780000430C3F30803002B40F09280EFF31183D1
:10C79000002B40F08D802968A26800BF2B68994269
:10C7A000F9D1D7F800E000FB0EF39B1AB3FBFEF3C0
:10C7B00000FB01314FF0010E0191D9F80430C3F3B1
:10C7C000080303BBEFF31183EBB92B68A16800BF2B
:10C7D0002A689342F9D1D7F800B000FB0BF2521A45
:10C7E000B2FBFBF200FB0323019A9B1AB3F57A7F9D
:10C7F000E3D3BAF1010AC2D1029B013B02937FF459
:10C8000067AFFEF777F8EFF311888CF31288A16811
:10C810002368DB0344BFC6F800E0A1682B683268D8
:10C820005FFA88F888F31188D7F800801A4400FB73
:10C8300008F35B1AB3FBF8F300FB0233D4E7EFF322
:10C8400011888CF31288A1682368DB0344BFC6F803
:10C8500000E0A1682B6832685FFA88F888F31188D5
:10C86000D7F800801A4400FB08F35B1AB3FBF8F317
:10C8700000FB023370E7EFF311828CF31288D4F8D7
:10C8800008E02368D90303D501233360D4F808E016
:10C890002B683168D2B282F311883A68194400FBE0
:10C8A00002F3A3EB0E03B3FBF2F300FB013135E718
:10C8B000EFF311828CF31288D4F808E02368D903CF
:10C8C00003D501233360D4F808E02B683168D2B275
:10C8D00082F311883A68194400FB02F3A3EB0E03BC
:10C8E000B3FBF2F300FB013164E7184630F088F83F
:10C8F0003EE700BF98A900209CA9002010E000E0BE
:10C9000094A9002000ED00E038B5484B5A89998978
:10C91000914224BF00225A81198ADA89914224BFA8
:10C920000022DA81DA78CAB1072A41496AD091F83F
:10C930005300404D012400210A282C709C70D971AD
:10C940005DD00C2807D0002A6CD0DFED3B7A072A97
:10C950000ED00A2862D0DFED397A09E0344A92F825
:10C9600053000A2856D00C285BD1D979DFED347AF0
:10C97000344C9FED350AA278002918BFF0EE407ABA
:10C98000062A04D8314901EB820191ED050A21798B
:10C9900079B1013A032A0BD8F7EE007A87EE800AC4
:10C9A00032F01CFA2388984228BF1846208038BDF0
:10C9B00038BD9B781F4A07EE103A1178B8EEC77A57
:10C9C00067EE277A07EE101AB8EEC77A27EE277AB5
:10C9D000B4EEC70AF1EE10FAEADD80EE277AFDEE3A
:10C9E000C77A17EE903A102BA8BF1023012BB8BFBF
:10C9F0000123DBB28B4238BF0B46137038BDDFED2D
:10CA0000147AA4E791F853000A2803D00C28ACD07C
:10CA1000D9799AE7D979DFED0E7AA9E7DFED0D7ABA
:10CA2000A6E7D979DFED047AA2E700BF28750020D8
:10CA30003C750020D45200206F1203396F12833AE4
:10CA40000AD7A339287F00206F120338C4FE0308D9
:10CA50005304E9380F506E3A2DE9F047AC4FAD4E14
:10CA600016F0A8FABE421ED2DFF82C83DFF82C9312
:10CA70004446258862197DB14A450DD2052D0BD952
:10CA800033886188C3F30B03994200F0E4801446B5
:10CA900025886219002DEFD1716830461436FCF7F5
:10CAA0006EFABE42E4D39C4A1378A3F1170102291F
:10CAB0000FD99A4911F83300002840F0FB80D800C4
:10CAC0000144497829B1964911F833300BB918233C
:10CAD0001370944B5A78022A00F2DD8092499348F1
:10CAE00002EB420201EB82011A780160022A00F295
:10CAF000DB8002EB82018E4BC2EBC10203EB4203EF
:10CB0000998C5A8C8B4C9142236001D300225A8419
:10CB1000894B9A78042A00F0EE8032B91A88B2F56F
:10CB2000F07F84BF4FF4F0721A80844DFFF7ECFE63
:10CB30002B68834A1A40002A00F0E680D80700F1EB
:10CB4000D580590400F1CD801A0700F1BC809B0408
:10CB500000F1C08025F0D8F910B97A4825F0E8FD39
:10CB60004FF40070FCF742FA4FF48020FCF73EFAD5
:10CB70004FF40010FCF73AFA4FF00070FCF736FA69
:10CB80004FF08060FCF732FA1AF076FB0021302279
:10CB90006D4833F0DEF820682CF02EFF6B4B2568D3
:10CBA00003F1500103E00433994200F081801A78C8
:10CBB000002AF8D19C78D8788442F4D26449654B35
:10CBC0000A7028461D6028F0D3FC634A6349107937
:10CBD000634A644B1160C822642111FB00210022CA
:10CBE00059609A60DA601A615A619A61DA6183F871
:10CBF000202083F821201DF04DFB5B4B9FED5B5AFD
:10CC00001B885B4A9FED5B6A55795B4C5B495C48CE
:10CC1000086006EE903AF8EEE66A1388C5EE265AEA
:10CC200007EE103A53881279C4ED005A07EE903A95
:10CC3000B8EEC77A534BF8EEE77A1D725A7227EEB8
:10CC4000067A67EE867ABDE8F04783ED017AC3ED98
:10CC5000007A16F097B963799B077FF418AF716873
:10CC600094F804A03046FCF78AF93388BAEB133FF6
:10CC700004D01436BE42FFF4FBAE14E7738870682C
:10CC8000AA1FC3F30B039A4204F10601A8BF1A4678
:10CC900031F064FFEDE700225A701A7823482249E8
:10CCA0000160022A7FF625AF00221A70204B27E789
:10CCB000012283E7D8000C186468002C7FF400AFD1
:10CCC00017241470FCE63048FCF790F92B689B049D
:10CCD0007FF540AF2D48FCF789F94020FCF786F935
:10CCE00038E72B48FCF782F92B682DE72948FCF739
:10CCF0007DF92B6825E79A8AB2F57A7FBFF415AFE4
:10CD00004FF47A729A8210E743F008032B6015E71C
:10CD1000180600089001000810530020842E040813
:10CD2000A42C0408B8430020C4430020446300201E
:10CD3000C03E002040630020287F0020F43F0020F8
:10CD400009600002905B0020F41F0020283D0020B5
:10CD5000A00F00202820002054430020E65200208D
:10CD6000302000209049002078250020C0C9FB48D1
:10CD70007C23002017B7D1387C2500209442002066
:10CD80003661023D7042002001600002094000024D
:10CD9000092000020860000202400008008000082C
:10CDA00038B50D4C0D4DAC4206D2616820461434A6
:10CDB000FCF7E5F8AC42F8D3FDF762F9084A094BF5
:10CDC000094C1460002209491A705A70084808601A
:10CDD000BDE838401EF0F8B99001000818060008B8
:10CDE00040630020B8430020C03E00204463002080
:10CDF000C4430020F0B50C2934D8DFE801F08933B2
:10CE000033335E333333343333330700048C968942
:10CE1000B2F802E01788734D24F480542404240CE3
:10CE20000484038C8488818B23F4005321F4E6412D
:10CE30001B0409041B0C46EA0E06090C43EA0633E0
:10CE400041EA0721A8429BB2A4B289B200F09E80B9
:10CE500005F58065A84200F09980926884808183FE
:10CE600002640384F0BD048C9589B2F802C0B2F864
:10CE700000E05C4F24F480742404240C0484038CAC
:10CE80008688818B23F400731B0421F073011B0C33
:10CE900045EA0C04090443EA0423090CB8429BB296
:10CEA000B6B241EA0E015CD04F4CA04259D0926814
:10CEB00086808183C2630384F0BD048C9589B2F8B7
:10CEC00002C0B2F800E0474E24F010042404240C01
:10CED0000484038C8788018B23F0200321F4E6412E
:10CEE0001B0409041B0C45EA0C04090C43EA041357
:10CEF00041EA0E21B0429BB2BFB289B25DD03A4C3A
:10CF0000A0425AD092688780018382630384F0BD77
:10CF1000048C9789B2F802E01688324D24F001049F
:10CF20002404240C0484038C8488018B23F00203E2
:10CF30001B0421F073011B0C47EA0E0709043B4355
:10CF4000090CA8429BB2A4B241EA060125D005F51E
:10CF50008065A84221D09268848001834263038463
:10CF6000F0BDD589148A578A23F4006343EA052566
:10CF70004FF6FF332B40958826F440563C4343EA56
:10CF8000052346EA04169BB2B6B290E7158A24F44C
:10CF9000804444EA8514A4B25FE7D689158A578A8B
:10CFA00023F00803334324F4407496883D4323F070
:10CFB00004032C433343A4B2CDE7D489158A568A9F
:10CFC00023F0800343EA04134FF6BF741C40938898
:10CFD00027F44067354344EA031347EA85079BB2C9
:10CFE000BFB28FE700000140000401402DE9F84F77
:10CFF0004FF4B47200218B488B4C8C4D8C4E8D4F6E
:10D00000DFF84C82DFF84C9232F0A3FE8A488B495D
:10D01000DFF844E2DFF844C2002213588B4200F0EC
:10D02000C280B3F1804F00F0D180AB4200F0D580D8
:10D03000B34200F0D580BB4200F0D580734500F0CC
:10D04000D580634500F0D580434500F0D5804B4541
:10D0500000F0D580DFF808A2534500F0D3800AF530
:10D06000806A534500F0D180AAF5983A534500F004
:10D07000CF800AF5806A534500F0CD800AF5806ABA
:10D08000534500F0CB801832B2F5CC7FC5D16A4E43
:10D090006B4F06F5CC784FF0030A4FF0020902E01F
:10D0A000183646457DD0B379002BF9D033791C0969
:10D0B000013C032C03F00F03F2D8624A32F814004B
:10D0C00040FA03F2D207EBD5012505FA03F3013B41
:10D0D000184031F0FFFA5C4B1B5D184417EBC0029F
:10D0E000DED057F83030594C317A03F13F4000F52B
:10D0F0007E00800A205C00F01F044009032805FA26
:10D1000004F55DD0042855D0022804D14648406C6F
:10D11000054345484564B2F804E0BEFA8EF2C2F118
:10D120001F0292B2D00803EB800002F00702046AEB
:10D1300092000F25954024EA05040462046A01FA6E
:10D1400002F22243002502624FF0010C2A4603E05E
:10D15000102A05F10205A3D00CFA02F030EA0E0104
:10D1600002F10102F4D11C680AFA05F1C9430C402E
:10D170001C60D3F800B009FA05F444EA0B041C6003
:10D180009C680C409C609C689C605C6824EA000081
:10D19000586058685860D8680140D960D968D9602B
:10D1A000D6E7BDE8F88F4FF0010A636C43EA0A0343
:10D1B000636468E71C48006B05431B480563AAE7E6
:10D1C0001948006C054318480564A4E74FF0010AAC
:10D1D000236C43EA0A03236455E74FF0020AF7E79A
:10D1E0004FF0040AF4E74FF0080AF1E74FF0100A95
:10D1F000EEE74FF0200AEBE74FF0020AD5E74FF4D5
:10D20000803AD2E74FF4003ACFE74FF4802ACCE7D8
:10D210004FF0400ADCE74FF0800AD9E74FF4807AFC
:10D22000D6E700BF08540020003802400004004048
:10D2300000080040000C0040642404080000014085
:10D2400060A70020B4340408B0340408A8340408EB
:10D250000004014000400140001000400014004064
:10D260000044014000286AD003682DE9F04F03F123
:10D270003F4404F57E045F4EA40A0125345D04F0AA
:10D280001F066409032C05FA06F559D0042C00F09A
:10D29000AC80022C59D08588B5FA85F0C0F11F000A
:10D2A00080B2C40803EB840400F00700266A800003
:10D2B0000F27874026EA07062662276A01F0030641
:10D2C0008240701E3A430128C1F3810CC1F300185B
:10D2D0002262C1F341113DD90024224601274FF0BB
:10D2E000030E03E0102A04F1020426D007FA02F02C
:10D2F000A84302F10102F5D1D3F800C00EFA04F000
:10D30000C04300EA0C0CC3F800C0D3F8008006FA52
:10D3100004FC4CEA080CC3F800C0D3F80CC000EAC7
:10D320000C00D860D3F80CC001FA04F040EA0C00FD
:10D33000102AD86004F10204D8D1BDE8F08F7047FC
:10D340002D4C266C35432564A5E72B4C666C354384
:10D350006564A0E7002002464FF0010E4FF003097C
:10D3600004E00132102A00F102003CD00EFA02F76C
:10D3700037EA0504F5D1D3F800A009FA00F4E44334
:10D380000AEA040AC3F800A0D3F800B006FA00FACB
:10D390004AEA0B0AC3F800A0D3F808A004EA0A0A74
:10D3A000C3F808A0D3F808B00CFA00FA4AEA0B0A4E
:10D3B000C3F808A0D3F804A02AEA07075F60D3F8EF
:10D3C00004A008FA02F747EA0A075F60DF683C40FA
:10D3D000DC60DF6801FA00F401323C43102ADC60B3
:10D3E00000F10200C2D1BDE8F08F034C266B35433B
:10D3F000256350E7A83404080038024003682DE98B
:10D40000F04F03F13F4404F57E04604EA40A012569
:10D41000345D04F01F066409032C05FA06F500F0DC
:10D42000AF80042C00F0A780022C54D08588B5FA78
:10D4300085F0C0F11F0080B2C40803EB840400F043
:10D440000700266A80000F27874026EA0706266223
:10D45000276A01F0030602FA00F0721E3843012A1F
:10D46000C1F3810CC1F300182062C1F3411137D917
:10D470000024224601274FF0030E03E0102A04F196
:10D48000020426D007FA02F0A84302F10102F5D106
:10D49000D3F800C00EFA04F0C04300EA0C0CC3F845
:10D4A00000C0D3F8008006FA04FC4CEA080CC3F86C
:10D4B00000C0D3F80CC000EA0C00D860D3F80CC050
:10D4C00001FA04F040EA0C00102AD86004F10204CA
:10D4D000D8D1BDE8F08F2E4C666C35436564A5E766
:10D4E000002002464FF0010E4FF0030904E0013224
:10D4F000102A00F102003CD00EFA02F737EA0504C8
:10D50000F5D1D3F800A009FA00F4E4430AEA040ACA
:10D51000C3F800A0D3F800B006FA00FA4AEA0B0AF2
:10D52000C3F800A0D3F808A004EA0A0AC3F808A0C8
:10D53000D3F808B00CFA00FA4AEA0B0AC3F808A0BC
:10D54000D3F804A02AEA07075F60D3F804A008FA1A
:10D5500002F747EA0A075F60DF683C40DC60DF688B
:10D5600001FA00F401323C43102ADC6000F10200B1
:10D57000C2D1BDE8F08F064C266B3543256355E7D5
:10D58000034C266C3543256450E700BFA8340408DB
:10D590000038024010B50409013C032C17D80D4B8C
:10D5A00033F8142000F00F0042FA00F313F00103E7
:10D5B0000DD0012303FA00F00138104031F08AF851
:10D5C000054A064B125D104403EBC00010BD00205D
:10D5D00010BD00BFB4340408B034040860A70020B4
:10D5E00001490248FEF724BF4855002000180040BA
:10D5F00001490248FEF71CBF2055002000480140A9
:10D6000001490248FEF714BFD05400200004014035
:10D6100001490248FEF70CBFD0540020000401402D
:10D6200001490248FEF704BFA8540020000C004046
:10D6300001490248FEF7FCBE80540020000800406B
:10D6400001490248FEF7F4BE58540020000400408F
:10D6500002494FF08040FEF7EBBE00BF305400207F
:10D6600010B5064C06482146FEF7E2FE04F1F00133
:10D670000448BDE81040FEF7DBBE00BF08540020A0
:10D68000000001400044014001490248FEF7D0BEBD
:10D690000854002000000140F0B50468A30AA3F577
:10D6A0008013522B2BD8DFE803F02B7B978F2A2A8D
:10D6B000932A2A2A2A2A2A2A2A2A2A2A2A2A2A2A61
:10D6C0002A2A2A2A2A2A2A2A2A2A2A2A2A2A2A2ABA
:10D6D0002A2A2A2A2A2A2A2A2A2A2A2A2A2A2A2AAA
:10D6E0002A2A2A2A2A2A2A2A2A2A7F832A2A2A2AEC
:10D6F0002A2A2A2A2A2A2A2A2A2A2A878B00F0BD9D
:10D700004FF0480E01264779B0004FEA970C0029E8
:10D710006FD063460227A5899F4083190CEB430312
:10D720002F4303F1040C3D4DBFB245F8231045F8DB
:10D730002C20A781EFF31181502282F312888219E5
:10D7400005EBC2021369002B4AD01362043382191D
:10D7500005EBC202576917B11F6053690433821980
:10D7600005EBC202976917B11F60936904338219F0
:10D7700005EBC202D76917B11F60D36904330027D4
:10D78000CAB21F6082F31188304405EBC000036AFF
:10D790004BBBA38923F001031B041B0CA381F0BD29
:10D7A0004FF0700E0226AEE74FF0200E0026AAE7DB
:10D7B0004FF0E80E0526A6E74FF4887E0626A2E77E
:10D7C0004FF49C7E07269EE74FF0C00E04269AE792
:10D7D0004FF4B07E082696E74FF0980E032692E7A6
:10D7E00005EB0E03B3E7A3899BB243F00103A381CA
:10D7F000F0BD0223BF0803FA07F7A389074D9BB2C8
:10D8000023EA070387190CEB470CA3810CF10403EF
:10D8100045F82C1045F823208CE700BF0854002061
:10D8200010B5036882480139834282B089B200F0A2
:10D83000CA80A0F58060834200F0C58000F580407A
:10D84000834200F0B78000F58060834200F0B28030
:10D8500000F58060834200F0AD80764C1888246823
:10D860006408B4FBF2F4013CA4B282B2B3F1804F7D
:10D870000AD07148834207D000F58060834203D00C
:10D8800000F58060834202D122F0700292B26B48B0
:10D89000834200F0A18000F58060834200F0A68002
:10D8A00022F4407200F56C4092B283421A80D96231
:10D8B0001C854FD05E4A93424CD001229A821A882E
:10D8C00092B242F001021A80B3F1804F00F09880CA
:10D8D000594A934200F0968002F58062934200F02C
:10D8E000938002F58062934200F0908002F580629E
:10D8F000934200F08D8002F58062934200F08A80AE
:10D9000002F57042934200F0878002F57052934214
:10D9100000F0848002F58062934200F0818002F57D
:10D92000806293427ED0A2F5983293427CD002F579
:10D93000806293427AD002F58062934208BF0D2242
:10D9400015D002A84FF0012340F8043D29F04CF80F
:10D9500002B010BD0122002119869A821A88384827
:10D9600092B242F0010283421A80ADD10A46354B91
:10D9700003EBC20301A85C798DF804400123002267
:10D980008DF805308DF807308DF8062029F02CF839
:10D990001B2C08D02E2CDBD12B4B019301A829F096
:10D9A00023F802B010BD294B019301A829F01CF8FF
:10D9B00002B010BD1F4C18882468B4FBF2F4013C7F
:10D9C000A4B282B252E71B4C18882468B4FBF2F46C
:10D9D000013CA4B282B257E701201A80D9621C85AB
:10D9E00098821A8892B202431A8071E701201A8045
:10D9F000D9621C8598821A8892B202431A8063E722
:10DA00000122B4E70222B2E70322B0E70422AEE724
:10DA10000522ACE70622AAE70722A8E70822A6E724
:10DA20000922A4E70A22A2E70B22A0E70C229EE724
:10DA300000040140748200200004004000100040F7
:10DA400000000140202C04082C01000119010001F4
:10DA50002B4B98423CD0B0F1804F3BD0A3F57C4398
:10DA6000984239D003F58063984237D003F580633C
:10DA7000984235D003F58063984233D003F5806334
:10DA8000984231D003F5704398422FD003F570537C
:10DA900098422DD003F5806398422BD003F5806324
:10DAA000984229D0A3F59833984227D003F5806394
:10DAB000984207D003F58063984208BF0D2202D038
:10DAC000002070470C220F4B03EBC20318797047FC
:10DAD0000022F8E70122F6E70222F4E70322F2E748
:10DAE0000422F0E70522EEE70622ECE70722EAE748
:10DAF0000822E8E70922E6E70A22E4E70B22E2E748
:10DB000000000140202C04082DE9F04F013085B0C1
:10DB1000C3B203930B4602918B4C8C4E002B00F04A
:10DB20009A8032208A4D8B4FDFF82C922FF006F925
:10DB30004FF4FA7A4FF0100C4FF47A70D9F80430A1
:10DB4000C3F30803002B40F0DE80EFF31183002BBA
:10DB500040F0D9802968A26800BF2B689942F9D1AA
:10DB6000D7F800E000FB0EF39B1AB3FBFEF300FBBB
:10DB700001314FF0010E0191D9F80430C3F30803CD
:10DB8000002B40F08780EFF31183002B40F0828060
:10DB90002B68A16800BF2A689342F9D1D7F800B07A
:10DBA00000FB0BF2521AB2FBFBF200FB0323019ABB
:10DBB0009B1AB3F57A7FDFD3BAF1010ABED1039B7A
:10DBC000002B40F0BD804FF47A7ADFF88C915046FC
:10DBD0004FF0100CD9F80430C3F30803002B75D1B3
:10DBE000EFF31183002B71D12968A26800BF2B6865
:10DBF0009942F9D1D7F800E000FB0EF39B1AB3FB72
:10DC0000FEF300FB01314FF0010E0191D9F8043011
:10DC1000C3F3080313BBEFF31183FBB92B68A168AF
:10DC200000BF2A689342F9D1D7F800B000FB0BF28D
:10DC3000521AB2FBFBF200FB0323019A9B1AB3F5C5
:10DC40007A7FE3D3BAF1010AC4D1029B013B02936C
:10DC5000002B7FF466AF05B0BDE8F08FEFF31188BD
:10DC60008CF31288A1682368DB0344BFC6F800E088
:10DC7000A1682B6832685FFA88F888F31188D7F8B2
:10DC800000801A4400FB08F35B1AB3FBF8F300FBB7
:10DC90000233D2E7EFF311888CF31288A16823686E
:10DCA000DB0344BFC6F800E0A1682B6832685FFA66
:10DCB00088F888F31188D7F800801A4400FB08F32D
:10DCC0005B1AB3FBF8F300FB023370E7EFF311824A
:10DCD0008CF31288D4F808E02368D90303D5012314
:10DCE0003360D4F808E02B683168D2B282F311882F
:10DCF0003A68194400FB02F3A3EB0E03B3FBF2F303
:10DD000000FB01317FE7EFF311828CF31288D4F826
:10DD100008E02368D90303D501233360D4F808E071
:10DD20002B683168D2B282F311883A68194400FB3B
:10DD300002F3A3EB0E03B3FBF2F300FB013118E790
:10DD400018462EF05DFE3EE710E000E094A90020AA
:10DD500098A900209CA9002000ED00E0204B5B6802
:10DD6000C3F3080330B4BBB9EFF31183A3B91D4B60
:10DD70001D4C1868A16800BF1A689042F9D11B4B6E
:10DD80001C684FF47A7202FB04F3591AB1FBF4F1E8
:10DD900030BC02FB00107047EFF31182102383F3B5
:10DDA000128811498C680B6813F4803F104B02D025
:10DDB000012018608C680B49D2B20D68186882F394
:10DDC00011880A4B19684FF47A72284402FB01F358
:10DDD0001B1B30BCB3FBF1F302FB0030704700BFEC
:10DDE00000ED00E098A9002010E000E09CA90020D0
:10DDF00094A900202DE9F84F8046FFF7AFFF254E8C
:10DE00002549DFF8A0E0254A254D844610274FF428
:10DE10007A740120DEF80430C3F30803D3B9EFF3BA
:10DE20001183BBB90B68D2F808A000BFD1F80090ED
:10DE30004B45F7D1D6F800B004FB0BF9A9EB0A0962
:10DE4000B9FBFBF904FB0393A3EB0C034345E1D3BC
:10DE5000BDE8F88FEFF3118A87F31288D2F808B083
:10DE60001368DB0344BF2860D2F808B00B68D5F80C
:10DE700000905FFA8AFA8AF31188D6F800A09944D4
:10DE800004FB0AF3A3EB0B03B3FBFAF304FB093324
:10DE9000DAE700BF9CA9002098A9002010E000E06C
:10DEA00094A9002000ED00E02DE9F04FDFF830C12B
:10DEB000474A4849484E494D8046102718F1FF38D7
:10DEC000C0F08480DCF80430C3F30803002B5CD17D
:10DED000EFF31183002B58D10B68946800BF0868DA
:10DEE0008342F9D1D6F800904FF47A7000FB09FE16
:10DEF000AEEB040EBEFBF9FE00FB03EEDCF80430D3
:10DF0000C3F308034FF47A740120FBB9EFF31183D4
:10DF1000E3B90B68D2F808A000BFD1F800904B45D8
:10DF2000F7D1D6F800B004FB0BF9A9EB0A09B9FB4D
:10DF3000FBF904FB0393A3EB0E03B3F57A7FBDD289
:10DF4000DCF80430C3F30803002BDFD0EFF3118AB1
:10DF500087F31288D2F808B01368DB0344BF286047
:10DF6000D2F808B00B68D5F800905FFA8AFA8AF305
:10DF70001188D6F800A0994404FB0AF3A3EB0B0325
:10DF8000B3FBFAF304FB0933D5E7EFF3118487F30E
:10DF90001288D2F808901368D80303D501232B60A8
:10DFA000D2F808900B682868E4B284F31188D6F898
:10DFB00000A04FF47A7400EB030E04FB0AF3A3EB0A
:10DFC0000903B3FBFAF304FB0E3E97E7BDE8F08FBD
:10DFD00010E000E098A900209CA9002094A900204E
:10DFE00000ED00E030B4EFF31183102282F31288C9
:10DFF0000649074C0A680748013200250A60256077
:10E00000DBB2026883F3118830BC704798A9002006
:10E0100094A9002010E000E038B5264B9C68636BA3
:10E0200073B1A36DA26BD2B1998A1A88C90592B255
:10E0300001D5D20700D438BD4FF6F7721A8038BD2B
:10E04000A36D99891A88890692B2EBD59206E9D513
:10E05000E26AD2B19888216B80B29047E1E7998952
:10E060001A880D0692B2DFD51006DDD5A26A616A64
:10E070008A4219D0A1692569885C98800132B2FB77
:10E08000F5F105FB1122A262CEE79B88E269616986
:10E09000DBB28B54E269E068A36D0132B2FBF0F1B0
:10E0A00000FB1122E261BDE7DA6822F08002DA604B
:10E0B000BAE700BF7034002038B5264B5C68636B4C
:10E0C00073B1A36DA26BD2B1998A1A88C90592B2B5
:10E0D00001D5D20700D438BD4FF6F7721A8038BD8B
:10E0E000A36D99891A88890692B2EBD59206E9D573
:10E0F000E26AD2B19888216B80B29047E1E79989B2
:10E100001A880D0692B2DFD51006DDD5A26A616AC3
:10E110008A4219D0A1692569885C98800132B2FBD6
:10E12000F5F105FB1122A262CEE79B88E2696169E5
:10E13000DBB28B54E269E068A36D0132B2FBF0F10F
:10E1400000FB1122E261BDE7DA6822F08002DA60AA
:10E15000BAE700BF7034002038B5264B1C68636BEB
:10E1600073B1A36DA26BD2B1998A1A88C90592B214
:10E1700001D5D20700D438BD4FF6F7721A8038BDEA
:10E18000A36D99891A88890692B2EBD59206E9D5D2
:10E19000E26AD2B19888216B80B29047E1E7998911
:10E1A0001A880D0692B2DFD51006DDD5A26A616A23
:10E1B0008A4219D0A1692569885C98800132B2FB36
:10E1C000F5F105FB1122A262CEE79B88E269616945
:10E1D000DBB28B54E269E068A36D0132B2FBF0F16F
:10E1E00000FB1122E261BDE7DA6822F08002DA600A
:10E1F000BAE700BF7034002070B4EFF311865023EB
:10E2000083F31288836B1A68D20720D45D686DB9D6
:10E21000446A826A944217D081691144D9600ED948
:10E22000A21A5A608462002280F85C201A6842F0C8
:10E230000102F1B21A6081F3118870BC7047016964
:10E240008A1A5A608562EEE7012380F85C30F3B2E7
:10E2500083F3118870BC704703685B6A03B1184789
:10E26000704700BF03681B6A03B11847704700BFBF
:10E2700003682DE9F041DF691FB13B46BDE8F0417D
:10E280001847002A164611DD04460D460E4400E0EC
:10E2900023689B68204698470028F9D0236815F822
:10E2A000011B1B6820469847AE42F1D1BDE8F081C2
:10E2B00003689B69184700BF03685B69184700BF84
:10E2C00003681B69184700BF0368DB68184700BF75
:10E2D00003689B68184700BF03685B68184700BF66
:10E2E00003681B68184700BF38B50C46097849B168
:10E2F000054601342B6828461B68984714F8011B13
:10E300000029F7D138BD00BF064B53F820302BB1A0
:10E310001A689B8851690B4201D11383704753835C
:10E32000704700BF64A90020026802F13F4303F573
:10E330007E032DE9F04F9B0A544DEB5C03F01F0563
:10E340005B090124032B04FA05F400F09980042BE7
:10E3500000F09180022B3ED001F00306731E012BCA
:10E36000C1F3810CC1F300188588C1F3411137D97D
:10E370000024234601274FF0030E03E0102B04F185
:10E38000020426D007FA03F0A84303F10103F5D1F4
:10E39000D2F800C00EFA04F0C04300EA0C0CC2F838
:10E3A00000C0D2F8008006FA04FC4CEA080CC2F85F
:10E3B00000C0D2F80CC000EA0C00D060D2F80CC04B
:10E3C00001FA04F040EA0C00102BD06004F10204C2
:10E3D000D8D1BDE8F08F2E4B5D6C2C435C64BBE75D
:10E3E000002003464FF0010E4FF0030904E0013313
:10E3F000102B00F102003CD00EFA03F737EA0504B7
:10E40000F5D1D2F800A009FA00F4E4430AEA040ABC
:10E41000C2F800A0D2F800B006FA00FA4AEA0B0AE5
:10E42000C2F800A0D2F808A004EA0A0AC2F808A0BC
:10E43000D2F808B00CFA00FA4AEA0B0AC2F808A0AF
:10E44000D2F804A02AEA07075760D2F804A008FA15
:10E4500003F747EA0A075760D7683C40D460D7689B
:10E4600001FA00F401333C43102BD46000F10200A8
:10E47000C2D1BDE8F08F064B1D6B2C431C636BE7CC
:10E48000034B1D6C2C431C6466E700BFA8340408D2
:10E49000003802402DE9F04F4A484B494B4B4C4C59
:10E4A0004FF0010A4FF002094FF004084FF0080C3A
:10E4B0004FF0100E20274026802530F8022B12F056
:10E4C000010F03D01960A3F804A0083312F0020F63
:10E4D00003D01960A3F80490083312F0040F03D09E
:10E4E0001960A3F80480083312F0080F03D01960F4
:10E4F000A3F804C0083312F0100F03D01960A3F87A
:10E5000004E0083312F0200F02D019609F80083316
:10E5100012F0400F02D019609E80083312F0800F75
:10E5200002D019609D80083312F4807F05D04FF42B
:10E53000807B1960A3F804B0083312F4007F05D083
:10E540004FF4007B1960A3F804B0083312F4806F15
:10E5500005D04FF4806B1960A3F804B0083312F4AF
:10E56000006F05D04FF4006B1960A3F804B00833B6
:10E5700012F4805F05D04FF4805B1960A3F804B0FB
:10E58000083312F4005F05D04FF4005B1960A3F864
:10E5900004B0083312F4804F05D04FF4804B19605B
:10E5A000A3F804B00833D20B04D04FF40042196032
:10E5B0009A80083301F58061A1427FF47EAFBDE807
:10E5C000F08F00BFB43404080000024060A70020B0
:10E5D00000100240002855D0026802F13F4303F5C5
:10E5E0007E032DE9F04F9B0A544DEB5C03F01F05B1
:10E5F0005B090124032B04FA05F444D0042B00F03A
:10E600009780022B44D001F00306731E012BC1F347
:10E61000810CC1F300188588C1F341113DD9002454
:10E62000234601274FF0030E03E0102B04F10204F0
:10E6300026D007FA03F0A84303F10103F5D1D2F87D
:10E6400000C00EFA04F0C04300EA0C0CC2F800C08F
:10E65000D2F8008006FA04FC4CEA080CC2F800C0AC
:10E66000D2F80CC000EA0C00D060D2F80CC001FA5D
:10E6700004F040EA0C00102BD06004F10204D8D161
:10E68000BDE8F08F70472E4B1D6C2C431C64BAE71D
:10E690002B4B5D6C2C435C64B5E7002003464FF0C8
:10E6A000010E4FF0030904E00133102B00F10200CA
:10E6B0003CD00EFA03F737EA0504F5D1D2F800A0F2
:10E6C00009FA00F4E4430AEA040AC2F800A0D2F806
:10E6D00000B006FA00FA4AEA0B0AC2F800A0D2F823
:10E6E00008A004EA0A0AC2F808A0D2F808B00CFA96
:10E6F00000FA4AEA0B0AC2F808A0D2F804A02AEAF3
:10E7000007075760D2F804A008FA03F747EA0A0798
:10E710005760D7683C40D460D76801FA00F40133F1
:10E720003C43102BD46000F10200C2D1BDE8F08F51
:10E73000034B1D6B2C431C6365E700BFA834040822
:10E740000038024010B1036882885A83704700BFC6
:10E7500010B1036882881A83704700BF18B103683C
:10E76000828809B95A8370471A8370470E4B1B88F9
:10E7700001463BB90D4B0E4A1B7810680BB981F06E
:10E780000101EBE70B4B5A691AB118B91A6810600E
:10E7900058747047084A18681188084A92FBF1F2C9
:10E7A000012102605974704770A9002072A90020ED
:10E7B00074A9002078A9002090A9002020A10700BA
:10E7C00010B40A4B0A4A1C7801238340234052F8B4
:10E7D000200029B9B3FA83F149095DF8044BBDE77C
:10E7E000191C18BF01215DF8044BB7E760A9002090
:10E7F00064A9002030B1036882881B691A4214BFE3
:10E8000001200020704700BF2DE9F0410B4E346815
:10E8100073691C400FD0DFF828800127B4FA84F315
:10E82000C3F11F0307FA03F558F82300036898475C
:10E83000AC437561F2D1BDE8F08100BF003C0140FE
:10E84000785300202DE9F0410B4E346873691C4069
:10E850000FD0DFF828800127B4FA84F3C3F11F0337
:10E8600007FA03F558F8230003689847AC4375612D
:10E87000F2D1BDE8F08100BF003C01407853002098
:10E880002DE9F0410B4E346873691C400FD0DFF85E
:10E8900028800127B4FA84F3C3F11F0307FA03F5B4
:10E8A00058F8230003689847AC437561F2D1BDE87E
:10E8B000F08100BF003C0140785300202DE9F04179
:10E8C0000B4E346873691C400FD0DFF82880012795
:10E8D000B4FA84F3C3F11F0307FA03F558F82300D1
:10E8E00003689847AC437561F2D1BDE8F08100BF81
:10E8F000003C0140785300202DE9F0410B4E346874
:10E9000073691C400FD0DFF828800127B4FA84F324
:10E91000C3F11F0307FA03F558F82300036898476B
:10E92000AC437561F2D1BDE8F08100BF003C01400D
:10E93000785300202DE9F0410B4E346873691C4078
:10E940000FD0DFF828800127B4FA84F3C3F11F0346
:10E9500007FA03F558F8230003689847AC4375613C
:10E96000F2D1BDE8F08100BF003C014078530020A7
:10E970002DE9F0410B4E346873691C400FD0DFF86D
:10E9800028800127B4FA84F3C3F11F0307FA03F5C3
:10E9900058F8230003689847AC437561F2D1BDE88D
:10E9A000F08100BF003C014078530020084A09482C
:10E9B00008B5536C43F4804353640021402231F086
:10E9C000C8F9054B4FF0FF321A60C3F8032008BDA9
:10E9D0000038024078530020B853002003685B6A77
:10E9E000184700BF2DE9F041044618460D4616466B
:10E9F00098462FF075F92768E6722844A0722946D8
:10EA00007D69434632462046AC46BDE8F04160474A
:10EA1000036810B504461B689847236820469B6826
:10EA20009847A37B0133A37310BD00BF10B50368E3
:10EA300004469B689847FF2301226373227310BD2D
:10EA400038B50B4C23688BB15A68821A002A0546E8
:10EA500004DA0CE05A68AA1A002A07DB9A682260D6
:10EA600018461A6890472368002BF3D138BD38BD8B
:10EA7000C43C00202DE9F04FA24AA349147895B078
:10EA800000F59C43203307900B60002C00F0488574
:10EA90009E4B07991B6899429D4B089340F28980D1
:10EAA0001E689C499C4BDFF8B8A20491013C059379
:10EAB000147006F48056002E40F08780974B1B7828
:10EAC000022B00F0FD84042B0AD1FFF747F9944B89
:10EAD000944A1B68C31A9342C2BF934B00221A8008
:10EAE000924B079A9A429AF8023000F2C783002BA1
:10EAF00040F0C8838E4B0993089B1E6816F480571C
:10EB000040F0B784DFF85C92059BB3F90610049BD4
:10EB10005C8BA142B4BF00240124864B1B6813F018
:10EB200080535CD0099A127812F001025DD00498EB
:10EB3000408C884241F37880002C5CD17E4D95F862
:10EB40008810002957D17D487D49006890F82D0034
:10EB500000250D604D608D607A4900284CD1087009
:10EB6000002A4DD0F1064BD5774A1278D20647D409
:10EB7000002F45D1002B43D1750241D4734B1B7834
:10EB8000002B02F04180724B9B78002C42F09E805B
:10EB90003BB1704A704B12681B689B1A002BC2F283
:10EBA000A5801020644D24F04DFB012385F88930A9
:10EBB00026E01E68574A584B049206F48056059387
:10EBC000DFF89CA1002E3FF479AF00215948FBF7F4
:10EBD00049FA00287FF472AF20F0ACFE6EE77002B5
:10EBE000A0D4099A127802F00102534D002185F851
:10EBF0008810002CA7D0534901200870002AB1D1F9
:10EC0000564B1A78002A40F0C9800499059D488B1C
:10EC1000B5F90070898BB5F90250B842B4BF8026AF
:10EC2000002646F04003B942D8BF33469B0843F064
:10EC30008006A842B8BF3346059F43F04006A9426C
:10EC4000C8BF33469B08B7F90450B7F9066043F0D4
:10EC500080078542C8BF3B4643F040078D42B8BF9E
:10EC60003B469B0843F08007334D8642C8BF3B4676
:10EC700043F0400795F88AE08E42B8BF3B469E4578
:10EC800001F00382A5F88C2085F88E202F4985F8A5
:10EC90008A300E78002E01F0ED805F2B01F09F810D
:10ECA0006F2B01F0BA81099B1B78DB0776D495F8AE
:10ECB0008E10002972D1B5F98C30322B6EDD95F8AB
:10ECC0008A200120572A85F88E0001F03E85089B96
:10ECD0001B685C0741F13B805A2A41F0388095F867
:10ECE0009030002B41F0A08795F8923083F001031B
:10ECF00085F89230002B41F0E3870C2024F0A2FA33
:10ED000001F080B9C03C0020843B0020BC3C0020C6
:10ED1000287D0020645B0020FC9D0020AC48002082
:10ED20009023002060E316008A490020404B4C00ED
:10ED300008750020285100205C1F0020406300203F
:10ED40008C500020142500203E630020A00F0020DE
:10ED50000053002098A90020705300204B4400204D
:10ED600090490020783D0020B6490F68440037B133
:10ED7000261803EB86067F787678BE4208D20444D4
:10ED8000B14EB24803EB840300240B60348004606E
:10ED9000FA3A0023A5F88C2085F88E30089BAC4AFF
:10EDA0001B680792AB4C5F0700F1A2850DF1480B81
:10EDB000DFF8C8820A940023CBF80430454612934A
:10EDC000192740F6330340F28336059C02E00435F0
:10EDD000A94522D0A878E978884217FB006EF6D2C0
:10EDE0006878043017FB016134F910009842A8BF1D
:10EDF0001846B0F5617FB8BF4FF461707045E6DD2D
:10EE00008842E4DC29782729E1D85846043506935E
:10EE1000FBF718F9A945069BDCD18F4B8F4A1B786D
:10EE20000A9C9BE8030082E80300002B40F03A8133
:10EE30008B4B1F78002F00F0E58401218748FBF7FA
:10EE400011F9002840F04F819AF80330002B40F070
:10EE50004A8123881DB225F00105AEB2B342268057
:10EE600000F06B857F4D02270E204FF014094FF004
:10EE7000FF082F7085F8019085F8028024F0E2F9F0
:10EE8000394676482688FBF7EDF8002841F078806F
:10EE900026F002039BB2B34223800AD0714B1421A7
:10EEA000FF2202250E201D7059709A7024F0CAF9B5
:10EEB0002688DFF8CCB1DFF8CCA19BF80010DAF897
:10EEC0000400B50708BF81F00201C1F34001FFF75C
:10EED00045FC24216148FBF7C5F830B9099A13783D
:10EEE000590744BF23F004031370079B1B6813F0FA
:10EEF0000A0F1DD005215948FBF7B4F8002800F08F
:10EF00006A8625886F0740F1F18754480621FBF790
:10EF1000A9F8002800F04C866E0640F1B88707215A
:10EF20004E48FBF79FF8002840F02885079B1B6898
:10EF30009D0600F13784268848480C21FBF792F89B
:10EF4000002800F07C8146F48073B342238009D00E
:10EF5000444B02251421FF220E201D7059709A7017
:10EF600024F070F9404B1B78082B00F074810E2BB5
:10EF700000F07181089B1B685D0548D53B4B1B79F0
:10EF8000002B00F0948014213448FBF76BF8002824
:10EF900040F0928025F0DAF9012024F095F800285D
:10EFA00035D0DFF8E48000254FF0CC0902E0DDB277
:10EFB000022D2CD809FB05F76B1C58F80760002EB2
:10EFC000F5D1032290F9023002960192C2782849C5
:10EFD00051F822200092184632463346012123F090
:10EFE000AFFC034605EB450000EB0010049353B162
:10EFF000314608EB8000CC2230F0ABFE049B48F891
:10F0000007300135EDB223F00DFA0028D0D1099B6D
:10F010001B78D80740F182809BF80010154A164DE6
:10F02000DAF80000012301F0010113702B70FFF7E3
:10F0300095FB079B1B685A0700F1E48015B0BDE8FB
:10F04000F08F00BF64530020685300206C530020F1
:10F05000E06200203C6300204C7F0020285100200B
:10F060009C430020C4390020105300208C4E002007
:10F07000542804088025002009750020283D002020
:10F0800060A9002064A90020F49A002098F80220CA
:10F0900098F803309A42C0F0408608F10408A84569
:10F0A0003FF4C6AE98F800102329F6D1EEE7099B8D
:10F0B0001B78D9077FF56EAF4FF40F702CF002FA72
:10F0C0000028A4D00DF00CFB4FF40F702CF09CF92D
:10F0D00000289CD00DF004FB4FF40F702CF094F935
:10F0E0000028EFD193E7079B1B689A077FF5B1AE25
:10F0F0002688F3073FF5CCAE46F001039E422380FD
:10F100003FF4C6AEB44B1421FF2202250E201D7021
:10F1100059709A7024F096F82688B9E6AF4B1E789D
:10F12000002E65D1AE4B1B68002B61D0DFF8008349
:10F13000DFF8009318F8030C99F800704146A8F125
:10F14000030517F0FDFF002800F08685002F40F032
:10F15000D78505F10801687917F0F2FF002841F022
:10F160000585A049A87A17F0EBFF002800F08785F5
:10F17000022F41F012859C49E87B17F0E1FF00283F
:10F1800041F007859949287D17F0DAFF002800F043
:10F190008785042F41F0E6849549687E17F0D0FFFB
:10F1A000002841F0DB849349A87F17F0C9FF0028AD
:10F1B00000F08785062F41F0CD848F4995F8230014
:10F1C00017F0BEFF002841F0C1848C4995F8280053
:10F1D00017F0B6FF002800F08785082F41F0E18482
:10F1E000874995F82D0017F0ABFF002840F0878580
:10F1F000844B01221A7018F02FFA079B1B685A07DC
:10F200007FF51CAF032017F0D3FF002800F05587CF
:10F21000238813F008047FF411AF08200FF0B8F82A
:10F22000059E7948794D7A497A4A7B4BF688006881
:10F230002E80086014601C6015B0BDE8F08F26F4C5
:10F2400080739BB2B34223807FF482AE734B1B78F2
:10F25000082B7FF48CAE228822F040039BB29A42A6
:10F2600023803FF487AE5C4B02251421FF220E2041
:10F270001D7059709A7023F0E5FF7BE613B90123E6
:10F280008AF80230664B09931B201D789AF82140BA
:10F2900017F08EFF012C05F00108814600F0B986B9
:10F2A00005F0020306939AF820305E4EDFF888B12D
:10F2B0005D4F052B00F2D080DFE813F0C000830023
:10F2C0000600FE000001F300012C04BF05238AF8AC
:10F2D0002030B8F1000F12D0049B3088B3F9181019
:10F2E0000022134661F30F0260F31F4261F30F0324
:10F2F000059861F31F4303600323426006934B4D5F
:10F30000DAF814202B689A4280F0A48547F2305234
:10F310000323CAF81C208AF8203002200FF050F88E
:10F3200020F008FB2A68DAF81C3013440422CAF8DB
:10F3300018308AF82020012C40F00F872B68DAF86B
:10F3400018209A4280F088809BF8000020B917F0BE
:10F350002FFF002840F080803B6823F002033B60D1
:10F360002A687388642101FB03234FF48060002224
:10F37000CAF810308AF820208AF803200EF0F0FF37
:10F380009AF8203095E717F019FF012807D1274D8B
:10F3900073882A68642101FB0323CAF81030B9F18D
:10F3A000000F02D0B379002B7DD1012C54D01F4D1A
:10F3B000DAF810202B689A42C0F0C48601238AF83C
:10F3C0002030012C6DD0F379012B00F09E8017F0D6
:10F3D00075FE9AF820306CE7C439002009750020CA
:10F3E0000C75002070380020753800207A38002015
:10F3F0007F38002084380020893800208E38002093
:10F400009338002080250020E46200206025002041
:10F410006C250020642500205C250020105300206E
:10F4200008750020544300203863002098A900206C
:10F43000663800201C000020A00F0020B8F1000F4B
:10F44000A1D14FF48060B9F1000F00F094820EF06A
:10F450009FFF0023CAF81030069B002B3FF44CABF3
:10F46000184623F0EFFE089B1E6816F480573FF401
:10F4700049AB1D21B348FAF7F5FD00287FF442ABF4
:10F48000B14B03F1500903E00433994500F01A86AB
:10F490001A78262AF8D19978DA789142F4D2FFF7CF
:10F4A00033BBAA4D5CE717F009FE03224FF47A73D1
:10F4B0008AF82020CAF81C30A44D2EE7A34D3AE765
:10F4C000049A0599537DD27D013B31F913301AB16D
:10F4D000C3F53B6308331BB2A3F57A7307EE903A8A
:10F4E0009FED9B7A9B4AF8EEE77A40F2FF3167EE98
:10F4F000877AFCEEE77ACDED067ABDF818308B42BC
:10F5000028BF0B461380FFF7EBBA17F0D7FD032295
:10F5100040F6B8338AF82020CAF81C308B4DFCE640
:10F520008D4F3B78002B3AD0DFF86482DFF864B26D
:10F530008A4BDFF864A2049345465E464FF47A791D
:10F540000DE0049A115D9847032C26DC80B93B78C6
:10F550002AF8020F01349C4205F1040521DA072C38
:10F56000E1B23046DBF80430EBDD984700B2EEE75D
:10F5700038F824206B88801A9B1A09FB00F040F6AB
:10F58000CA0290FBF3F000F57A70904240F2EE234D
:10F59000A8BF10469842B8BF184600B2D7E76F4AD6
:10F5A00004926F4A08926F491268079842F2010A62
:10F5B000A1FB001B12EA0A0A4FEA9B1B00F03183F1
:10F5C000694D6A486A4C6B492E780078267008703D
:10F5D0001EB168490E7886F00106674D0F2185F847
:10F5E0002410002B00F09F84644B049C0F93B4F80C
:10F5F00026C0B4F824E0049CCDF830C01846248B13
:10F6000000785F4B10945F4C0E9005940446A3FB6A
:10F6100000035B0803EB4303E31ADBB202F48052FE
:10F620000B9397F80080DFF874C1564C95F825903D
:10F630000D910BF5967305F12800099511920021A3
:10F640000A9306967546069B002B00F0A683099B3D
:10F6500033F911301FFA83FEAE454FEA410203D35E
:10F660000C9EB64540F2E6835CF821309B4580F065
:10F670009D83A35EBAF1000F40F0BB830131414589
:10F68000A35200F10600DEDB0D9A099D3E4B85F882
:10F6900024200F2A0CBF0122002285F825901A7021
:10F6A00000F048843148DFF8F8A03249274D0122A4
:10F6B000027004200A700EF083FE2B68DAF808103E
:10F6C000DAF80420CAF80C305B1A934284BF002396
:10F6D0008AF821303C78089B1E68002C01F01681C6
:10F6E000049A2A4DB2F824E0178B264916F4805666
:10F6F000284640F0568432460EE0437803EB8303FD
:10F7000003EB830303F2EE239BB20132A24221F802
:10F71000023B00F102000ED015F81230002B00F071
:10F720008D83022BE9D001320B8821F8023BA242E3
:10F7300000F10200F0D10F9A137801331370FFF734
:10F74000BAB900BF28510020283D002098A9002008
:10F750006F12833F8A490020EC3D0020645B00204B
:10F76000287D0020D34D6210603B0020EC0000207B
:10F7700081490020ED0000205C1F0020DD3C0020BE
:10F78000ABAAAAAAFC9D00205A440020343E0020C7
:10F79000003E0020C87400205A1F0020E03C0020DA
:10F7A00090490020C54B1B78980704D5C44D2B7D8C
:10F7B000042B00F2DA84268816F0300F3FF4BCAB3D
:10F7C00010200EF0CDFD20200EF0CAFDBD4B268886
:10F7D00000221A70BC49BD48BD4FBE4D00220A60D0
:10F7E000BD493A6000232A60426082610360836001
:10F7F0004361C3610B604A608B604B618A61CB617E
:10F80000FFF79ABBDFF814B3DFF81483B34D0BF1A5
:10F810005A064FF0010959461BF8010C17F090FCED
:10F82000F8B19BF804009BF802309BF803E000EB72
:10F83000400105EB8101013BD1F89C2003EB430320
:10F84000434493420DD095F8C82081F898E009FA16
:10F8500000F022EA0000C1F89C30C1F8A07085F8E1
:10F86000C8000BF1060B5E45D5D19D499D4A9E4BC4
:10F870009E4D09681B78D2F800900A910693A5F175
:10F88000980B00266B6863B31F7857B3AA68A9EB7F
:10F890000202002A0ADB9BF8C8200121B14022EABB
:10F8A000010209F5FA718BF8C820A960069AC2B165
:10F8B0002A7859780432D2B2002940F0BB810499E9
:10F8C0000598098B30F9122001F1C800824240F3FB
:10F8D0000B849BF8C8109A7841FA06F3D80740F1D8
:10F8E000E1840136042E05F10C05CBD1FFF7A5BA52
:10F8F0007A4D95F892305BB1099B1B78DE0707D5EE
:10F90000059BB3F90620049B5B8B9A4200F3BC84F1
:10F9100011217748FAF7A6FB002800F0718195F8CD
:10F9200096302BB995F8903013B93223A5F894305E
:10F93000012385F89630FFF739BA02216C48FAF7AF
:10F9400091FB00283FF4A4AA2580B7073FF5B1AA90
:10F9500046F00203B34223803FF4ABAA654B02207A
:10F960001421FF2218700E2059709A7023F06AFC3F
:10F970002688FFF79EBA0EF0F3FC6AE55E4AB2F9FC
:10F980000030002BB8BF5B42B3F5E17FBFF6CEAAD3
:10F99000B2F90230002BB8BF5B42B3F5E17FBFF68E
:10F9A000C5AA564B93ED096AD3ED076A93ED057A24
:10F9B000D3ED037A76EE866A77EE877A76EEA66ADC
:10F9C000B7EE007A37EE666A77EEA77AB0EEC66ACF
:10F9D000F0EEE75AB4EEE56AF1EE10FAB4BFB0EE1D
:10F9E000655AB0EE465AB5EE405AF1EE10FA40F0C4
:10F9F0001B849FED437AB4EEE56AF1EE10FA44BF42
:10FA00009FED486A36EE477AB7EE006AF4EEC66AB2
:10FA1000F1EE10FAC8BFDFED446AF5EEC07AC8BF58
:10FA200036EEC77AF1EE10FA48BFB1EE477AF6EE3D
:10FA3000007A27EE677ADFED3B7A77EE276ABDEE34
:10FA4000E66A16EE103A2033402B40F2B086DFED26
:10FA50002D6A2D4ADFED2B7AC2ED006AFDEEC76AF2
:10FA6000C2ED017A16EE903A2033402BC2ED027AB5
:10FA700000F28980DFED2C7AB4EEE77AF1EE10FA2D
:10FA800041F3BE809FED216ADFED216A01E0B0EE17
:10FA9000677AB4EEE67AF1EE10FA77EE467AF6DCA3
:10FAA0009FED1C7AF4EEC77AF1EE10FA41F1A480D2
:10FAB0009FED166ADFED186A40E000BF3E6300204C
:10FAC00050920020124A0020FC4A0020AC4A00203C
:10FAD000E8240020DC250020D44A00205C1F002000
:10FAE0004463002098A9002081490020F41F0020D1
:10FAF00028510020C4390020EC620020680F00204B
:10FB0000A7DFA834000000009C000020DB0FC940E4
:10FB1000E4CB1641DB0F49C0E4CB16C17D37002092
:10FB2000F4FE0308DB0FC93FDB0F494092E741B900
:10FB30009730083C15A82ABEF0EE477AF4EEE67A34
:10FB4000F1EE10FA37EE867AF6D45FED0A7AB4EE6B
:10FB5000E77AF1EE10FA40F3A8865FED0D7A37EE02
:10FB6000C77A27EE076A5FED0F5A5FED0F6A5FED08
:10FB70000F7AE6EE256A67EE065AE6EE267AA5EEDD
:10FB8000A77AF0EE477AC64BC2ED037A1A6812F4F0
:10FB9000003240F08286C34B1046995C0A2902F17C
:10FBA0000C0200F0798501301828F6D1FFF7BEB9B4
:10FBB00025F040039BB2AB4223803FF4B0A9BA4B7F
:10FBC00002251421FF220E201D7059709A7023F017
:10FBD00039FBFFF7A4B9238823F00405ADB2AB428B
:10FBE00025803FF492A9B04B02251421FF220E205C
:10FBF0001D7059709A7023F025FB2588FFF785B991
:10FC000095F89030002B3FF4D1A8099B1B7813F096
:10FC1000010302BF012285F8903085F89120FFF79B
:10FC2000C5B8A2490E78D3E4A14D012185F888100A
:10FC3000FEF7E1BF012900F049859BF8C8200123A8
:10FC4000B34001361343042E8BF8C83005F10C0580
:10FC50007FF418AEFFF7F1B808F10501687917F0E5
:10FC60006FFA00283FF47DAA012F40F07F8705F14D
:10FC70000D01A87A17F064FA002840F08E878D49AC
:10FC8000E87B17F05DFA00283FF47CAA032F40F0D0
:10FC900080878949287D17F053FA002840F0628751
:10FCA0008649687E17F04CFA00283FF47CAA052F9D
:10FCB00040F054878249A87F17F042FA002840F0AC
:10FCC0004987804995F8230017F03AFA00283FF455
:10FCD0007CAA072F40F03A877B4995F8280017F057
:10FCE0002FFA002840F05D87784995F82D0017F02D
:10FCF00027FA00283FF47CAA092F3FF479AA0926A5
:10FD0000334603EB83031D44714B6978AA7889F865
:10FD1000006019705A70FFF76BBA6E48FAF7A2F9D3
:10FD200000283FF485A85E4B1B6813F4003340F0B5
:10FD3000898600225B4B1046995C142902F10C0263
:10FD400000F0948501301828F6D1FFF771B85D2ACC
:10FD500000F0AD825B2A00F0C7855E2A00F01686AF
:10FD6000562A00F0B686972A00F00887A72A00F0E6
:10FD70005D86594C23889B0740F0CC85A2F1B703E0
:10FD8000072B00F2BE82DFE813F0B602BC02BC0211
:10FD9000BC02B002BC02A202A202002D48D05CF854
:10FDA00021309B454FEA4102FFF463AC4B4B4B4E75
:10FDB0009B5C06EB020E002B00F0D580022B47D196
:10FDC0009EF8013003EB830303EB830303F2EE237E
:10FDD0009BB20329DFBF012606FA01FE0D9E26EA2B
:10FDE0000E06CEBF1BB21BB20D96BAF1000F3FF448
:10FDF00045AC0B9E20F81630B9F1000F03D10E9ED2
:10FE0000022E7FF63BACB0F802900388B0F804E015
:10FE10004B449E44324B0FFA8EFE83FB0E63314EF1
:10FE2000A3EBEE7326F802E01BB24FF0010925E4C4
:10FE30002B464A000A9E4CF821601BE4D3B2022BE9
:10FE400004D9032B7FF46FAC73465EE43B465CE45D
:10FE5000A35ABEE7244B1B78002B7FF457AAB8F1B6
:10FE6000000F3FF453AA012C7FF4F6AA9AF8203031
:10FE7000FFF71FBA31461748FAF7F4F8002800F0E8
:10FE8000E08085F88F6020F095F9FEF70CBF45F013
:10FE90004003AB4223807FF492AEFFF740B800BF2F
:10FEA00070370020081A0408C43900208149002056
:10FEB0005C1F0020753800207A3800207F38002031
:10FEC00084380020893800208E38002093380020A4
:10FED00010750020285100203C630020343E002093
:10FEE00056555555CC1F00200425002045F004032D
:10FEF0009D4223800AD0B24B02251421FF220E20FE
:10FF00001D7059709A7023F09DF92588AD4BAE4A4B
:10FF1000B3F90430AD4982FB0302DB17C3EBA20344
:10FF20000B80FEF7F2BFAA4AAA4B0F92AA4A05928B
:10FF300001221A701B21A948FAF794F800287FF4CF
:10FF4000B1ABDFF8C4A2A64DDAF80C202B68CAF8D2
:10FF500008309B1AC82B00F2CB84089B1E6806F45D
:10FF60008056FFF7E8BBCBB2022B40F2AC83032BE9
:10FF70007FF46EAF109B119E002E08BF2B4628E722
:10FF800026F001039BB2B34223803FF4DEAC0E2087
:10FF90002F7085F8019085F8028023F053F92688A8
:10FFA000D3E400220FE0437803EB830303EB8303E6
:10FFB00003F2EE239BB20132A24221F8023B00F190
:10FFC00002003FF4B8AB15F812301BB1022BEAD097
:10FFD0000B88F0E7D3B2032BFAD83B46EBE7B2F538
:10FFE000FA7FFEF6DBAE95F88E30002B7EF4D6AEAF
:10FFF000099B1B7801210B4085F88E1000F0C4830B
:020000040801F1
:100000001FF098FC774B0793089B774C1B68FEF713
:10001000CABE00230693FFF746B9B2F5FA7FFEF693
:10002000BDAE95F88E20002A7EF4B8AE099B1B78F1
:10003000012185F88E10D90700F1448420F0BAF828
:10004000E0E7099B694A1B781060D8077EF52FAE60
:10005000674B1B78002B3EF4A1AE9AF80330002BBF
:100060007EF49CAE95F88F300133DBB2032B85F81C
:100070008F307EF693AE5F4B5B7813B9002C7EF425
:100080008DAE1FF057FCFEF70EBE5B4A5B49106851
:10009000B5F98C20C66981FB06018911F617701A23
:1000A00000F5FF407F3082423EF7F0AD891B0A44E5
:1000B00012B2A5F88C20FEF7E9BD08200EF050F929
:1000C000FEF7BCBF4E4A049BD488059A1B8BB2F93D
:1000D00006101A1B914240F3D48023449942B4BFC6
:1000E00000240124FEF719BDC8398A425ADA9BF868
:1000F000C8109A7841FA06F3D9073FF5F2AB52429D
:1001000001200B9223F0C4F97B1E0B9A162B00F2F0
:100110006281DFE813F059026F022902980285021A
:10012000AC021402FF01E801D101BA01600198029A
:10013000A501AC021402FF018F01790163014E0198
:100140003601200116F0BAFF032240F6B8338AF8D0
:100150002020CAF81C30FFF7E0B82A68DAF81C3013
:100160001344CAF81830FFF777B90A2017F020F8BF
:1001700026880746002800F06283F10640F1BE841D
:10018000204D95F8D070002F7EF4D6AE0D2023F0D0
:1001900059F8012385F8D0302688002F7FF41AAB58
:1001A000FEF7CABE9BF8C8300122B24023EA020320
:1001B00009F5FA728BF8C830AA60FFF792BB00BF4E
:1001C000C4390020EC620020676666661C4B002084
:1001D000DD3C00205A440020FC9D002028510020D6
:1001E00098A90020E06200203C63002074530020A6
:1001F000814900200053002038740020D34D621044
:10020000384300205C1F00209049002099FB243FC8
:1002100069A2163EA7DFA83445FE7F3F88FA163E46
:10022000E3B59E3E39094E3DB4EEE56AF1EE10FAB3
:100230008CBFB0EE654AB0EE464AC4EE054A1FEDEB
:100240000D2A1FED0D5A5FED091A5FED0B2A1FED08
:100250000D3A5FED0F3A1FED114AA4EE825AE4EE1B
:10026000E12AA4EE857AA4EEA23AB0EE475AB0EEA7
:10027000637AA4EE837AA4EE874A84EE057AFFF7C8
:10028000BABB0124FEF749BC0021C448F9F7EAFED5
:1002900000287FF43DAB322385F89200A5F8943016
:1002A000FFF736BB002A0CBF0120022029E7BC4B18
:1002B00000220120BB49BC4C0B60BC4B2270079351
:1002C00023F0E6F8089BBA4C1B68FEF76CBDB94AF0
:1002D000B949B54B116002225A70B44B079316F01E
:1002E000CBFF089B1B68FEF75EBDB24AB3491160A5
:1002F000AD4B0022F0E7AF4AB1491160AA4B012291
:10030000EAE7792A00F0D5847A2A00F0CB849E2A85
:1003100000F0C0849D2A00F0B584AE2A00F0AA84C3
:10032000AD2A00F09F84EF2A00F09984FD2A00F0A6
:100330008484FB2A00F0F084FE2A00F0EA84F72A85
:1003400000F0C1847B2A00F04C84089B974A1B680C
:100350000792FEF728BDDBF8CC00DFF8688290F842
:10036000361098F8023011446429A8BF642121EAAC
:10037000E17180F83610002B40F0B38429F09CFC2A
:100380005BE4DBF8CC00DFF83C8290F8371098F89B
:1003900002301144FE29A8BFFE2121EAE17180F854
:1003A0003710002BEAD0162016F04CFFDBF8CC00FB
:1003B000E4E70A98DFF80C8241781144B1F5967FA2
:1003C000A8BF4FF4967121EAE171417098F80230AC
:1003D000002B40F0A484DBF8CC00CFE7DBF8CC00A6
:1003E000DFF8E08181781144C829A8BFC82121EA3B
:1003F000E171817098F80230002BBFD0142016F004
:1004000021FFDBF8CC00B9E7DBF8CC00DFF8B481E2
:1004100041781144C829A8BFC82121EAE17141707F
:1004200098F80230002BA9D0132016F00BFFDBF850
:10043000CC00A3E7DBF8CC00DFF888810178114419
:10044000C829A8BFC82121EAE171017098F80230DB
:10045000002B93D0122016F0F5FEDBF8CC008DE7D0
:10046000DFF860810A9898F80230417911446429D4
:10047000A8BF642121EAE1714171002BABD00E20AD
:1004800016F0E0FEDBF8CC0078E7DBF8CC00DFF814
:100490003481017A98F802301144C829A8BFC821D4
:1004A00021EAE1710172002B3FF468AF0B2016F0D6
:1004B000C9FEDBF8CC0061E7DBF8CC00DFF8048193
:1004C000C17998F802301144C829A8BFC82121EA8F
:1004D000E171C171002B3FF451AF0A2016F0B2FE5A
:1004E000DBF8CC004AE7DBF8CC00DFF8D880817974
:1004F00098F802301144C829A8BFC82121EAE17147
:100500008171002B3FF43AAF092016F09BFEDBF817
:10051000CC0033E7DBF8CC00DFF8A880417998F80D
:1005200002301144C829A8BFC82121EAE1714171F4
:10053000002B40F00384112F7FF454AF1EE7DBF84B
:10054000CC00DFF88080017998F802301144C82986
:10055000A8BFC82121EAE1710171002B40F0E683B8
:10056000102F7FF455AF09E70A99DFF858800F790B
:100570001744642FA8BF642727EAE7770F7116F0A6
:100580007BFE98F80230002B3FF425AF032039465C
:1005900016F058FEDBF8CC00F0E600BF2851002032
:1005A000C03E002040630020B8430020E0620020ED
:1005B0003C63002044630020DC430020C44300204F
:1005C000D0430020E03F00200A98DFF85C840178E7
:1005D0001144FA29A8BFFA2121EAE171017098F8C3
:1005E0000230002B3FF4F7AE012016F02BFEDBF8B3
:1005F000CC00C3E60A98DFF830848178114464297E
:10060000A8BF642121EAE171817098F80230002BC3
:100610003FF4E1AE022016F015FEDBF8CC00ADE6AB
:100620000A98DFF80484C17998F80230114481F304
:100630000801C171002B3FF4CEAE052016F002FE7A
:10064000DBF8CC009AE60A9BDFF8DC83997998F80E
:10065000020011446429A8BF642121EAE171997163
:10066000002840F074830D2F7FF4FCAEB3E6DBF876
:10067000CC00DFF8B483C17898F802301144C8295F
:10068000A8BFC82121EAE171C170002B40F0368378
:100690000F2F7FF4D3AE71E6C6490D6846003DB119
:1006A000321803EB82026D785278AA42BEF43EAC57
:1006B0003044C14DC14E002203EB80030B603280F9
:1006C0002A60FEF733BC109BFFF783BB059931F915
:1006D00012209978B2F5617F4FF4966393FBF1F3A2
:1006E000C0F2F98040F633019142A8BF11460C2FA9
:1006F000A1F5617191FBF3F100F00E82182F7FF4E8
:100700009CAAC9B2C8290B46A8BFC823DBF8CC00F5
:10071000C27DDFB297423FF490AA9A1ADFF80883AD
:10072000C77548BF0732D71098F802300137FFB2BB
:100730003BB9002F3FF481AA384622F0A9FEFFF70B
:100740007CBA182016F07EFDF3E79D4B9D491A6890
:100750004FF47A73B3FBF2F3C3EB431203EB820261
:10076000089B1B68D2001F06A1F8A82000F1128187
:10077000954A0792126855077EF514AB934A944C3C
:100780000A211180FEF70FBB9249096811F400316C
:1007900040F0AE81904B08465C5C0F2C01F10C01DF
:1007A0003EF4E2AA01301828F6D1FEF7F1BAB4EE11
:1007B000E77AF1EE10FA40F30282DFED885A9FEDFE
:1007C000886A01E0F0EE676AF4EEC66AF1EE10FAAC
:1007D00076EEE57AF6DCDFED836AF4EEE67AF1EEAA
:1007E00010FA40F1E981DFED7D5A9FED7F6A01E06B
:1007F000F0EE667AF4EEC67AF1EE10FA77EEA56ABC
:10080000F6D4DFED7A7AF4EEE76AF1EE10FA40F30F
:10081000B180DFED777A77EEE66A66EEA65A9FED55
:10082000755A9FED756ADFED757AA5EE856A26EE3D
:10083000A55AE5EE867AE5EE276AFFF70AB9F206D1
:1008400000F13F810B2016F0B3FC002840F003813B
:10085000B30600F1AA816A4D95F8D030002B3FF421
:1008600095AC002F7EF4B6AFFEF766BB51490E681B
:1008700042003EB1151803EB850576786D78B542D8
:10088000BEF4D6AA02444D4D4B4803EB820300222E
:100890000B602A800260FEF7CBBA5A4B1B78032B01
:1008A00000F068810022FFF776B9DFED577AB4EEE9
:1008B000E77AF1EE10FA44BFDFED4A7A37EEC77AF5
:1008C000FFF74FB95149089B0A603F4A1B680792DE
:1008D0003F4CFEF768BA0C2F00F03581182F7FF4DB
:1008E000ACA900210B4611E7494B01220220E1E4AB
:1008F000484A089B1E68136823F004031360012311
:1009000006F480568AF82130FEF715BF06F48056AB
:10091000FEF711BF0023BB2A129300F05781B72ABC
:1009200000F05081BE2A00F05481BD2A7FF4E9AC6A
:100930004FF6FE71384A2448D6890790908933448F
:1009400001449181D38112F035FBF8F78DFB12F051
:1009500019FBFCF781F8012022F09AFDB5F88C20F4
:10096000089BFA3A00211B68A5F88C2085F88E10A8
:10097000FEF719BADFED247AF4EEE76AF1EE10FA29
:1009800044BFDFED187A77EEE66A46E7234B022292
:1009900003208FE4224A127896077FF5E9AE214AB8
:1009A000127D042A7FF6E4AE1AF098FC089B1B68BF
:1009B000DEE600BF645300206C5300206853002023
:1009C000187D00203C750020E06200207643002066
:1009D0003C63002070370020081A0408DB0FC94070
:1009E000E4CB1641DB0F49C0E4CB16C1DB0FC93F96
:1009F000DB0F494092E741B99730083C15A82ABE61
:100A00005C1F00208D490020DB0FC9BF74530020FC
:100A10000E3F002038630020E05200205C3F0020A1
:100A20003E63002050920020E03F0020CB49089B0D
:100A30000A78CB481B68079042F004020A70C94C40
:100A4000FEF7B1B9C84B1B78032B7FF472A922F0D3
:100A5000DDFBFEF7EDB9C54AC54B528993ED007A2F
:100A600007EE902AF8EEE77AB0EEC77AB4EEE77AAE
:100A7000F1EE10FA7FF5ECAE93ED017AB0EEC77AA5
:100A8000F4EEC77AF1EE10FA7FF7E2AEB3063FF567
:100A9000E2AE20200DF07CFC95E80C00B5490A6020
:100AA000084641F8043F24F00DFDB34B01221A70B3
:100AB000B24D95F8D030002B00F028812688FEF743
:100AC00089BE10200DF04CFCAB4B26881F7001270F
:100AD000B8E612F06FFAF8F7C7FA12F053FAFBF71C
:100AE000BBFF012022F0D4FC95F88A20FFF73BB928
:100AF0009D49097803296ED019464BE610200DF068
:100B000047FC20200DF02CFC9D49081F24F0DAFC46
:100B1000994B02221A70CBE7CFB29A4B0B915B78BC
:100B2000BB423FF48AA8DFF8708238460BF044FBE2
:100B300098F802300B991BB1C9B20C2016F082FB59
:100B40000137FFB2F5E500273946E6E707263346C9
:100B5000FFF7D7B806263346FFF7D3B80526334646
:100B6000FFF7CFB804263346FFF7CBB8012633464C
:100B7000FFF7C7B822F04AFBFEF7D8B97849824A96
:100B8000089B07914FF4C8711B681180754CFEF7E4
:100B90000AB903263346FFF7B4B802263346FFF7F7
:100BA000B0B808263346FFF7ACB820200DF0D8FBCC
:100BB000714B00221A707BE7F0EE676A21E6F0EED7
:100BC000667A08E619464FF6FE73B3E61946022325
:100BD000B0E60221AEE622F019FBB5F98C20FEF753
:100BE000D7B84FF4FA6102200BF00CFA5C4B079374
:100BF000089B1B68FEF7D7B8B0EE677AFEF7A5BF73
:100C0000F0EE477AFEF74CBF002C3DF4CAAF5B4DC7
:100C100095F88930002B3DF4F3AF22F0F7FA00236A
:100C200085F88930FDF7ECBF4D4B85F8901085F8BD
:100C3000910007934B4CFEF75CBE002101200BF0A6
:100C4000E1F9B5F88C20089B45491B680791963A55
:100C5000A5F88C20002285F88E20FEF7A4B800218C
:100C60000846ECE7FF21002026F079F995F88A2064
:100C7000FFF759BB0121002026F071F995F88A2071
:100C8000FFF74EBB0021FF2026F069F995F88A2076
:100C9000FFF743BB0021012026F061F995F88A2077
:100CA000FFF738BB394A137A43F001031372FFF799
:100CB0004CBB364A137A23F001031372FFF745BB8E
:100CC0000B20FEF71BB800210420B8E7002B9ED0B4
:100CD0002F49304A09684FF47A7000FB0313136000
:100CE00095E7172016F0AEFAFFF775BB234D1EF0FF
:100CF00021FE002385F88930FDF782BF0F200B927B
:100D000016F0A0FADBF8CC000B9AC1E40127FFF73C
:100D10003DBA0021032092E7002102208FE7152031
:100D200016F090FADBF8CC00FFF728BB10200B92EE
:100D300016F088FADBF8CC000B9A11E411200B9224
:100D400016F080FADBF8CC000B9AFFF7F4BB0D200D
:100D50000B9216F077FA0B9A85E400BF3E630020F1
:100D6000E06200203C6300208D490020A04A002062
:100D70009C4E002074230020124A00205C1F00209B
:100D8000EC490020B843002078430020244B002089
:100D900098A9002070530020E03F00202DE9F04783
:100DA000C74C636820469847002800F0C380C54BB5
:100DB0001B780122042B84F83C2000F0BD80B4F99C
:100DC0001610B4F91820B4F91A3021636263A363D2
:100DD000BD4B1B88002B69D0BC4DD4ED0C7AD5EDF2
:100DE000004A95ED050A95ED015A95ED067AD5ED87
:100DF000035A95ED026AF8EEE76AD5ED047AA4EE9F
:100E0000A60AA5EE267A67EEC07AA5EEC07AE6EECF
:100E1000267A85ED057AC5ED067A2DF0DFFFD4ED53
:100E20000D6AD5ED094A95ED0E0A95ED0A5A95ED34
:100E30000F7AD5ED0D7AD5ED0C5A95ED0B6A20633E
:100E4000F8EEE66AA4EEA60AA5EE267A67EEC07A68
:100E5000A5EEC07AE6EE267A85ED0E7AC5ED0F7A1C
:100E60002DF0BCFFD4ED0E6AD5ED124A95ED170AB0
:100E700095ED135A95ED187AD5ED167AD5ED155AEC
:100E800095ED146A6063F8EEE66AA6EEA40AA6EE93
:100E9000857A67EEC07AA0EE657AE6EE867A85ED11
:100EA000177AC5ED187A2DF099FFA063884FA17FBE
:100EB000884819F071F93B88002B40F08480864EF9
:100EC000D6F8D450854B1B685B0743D4B5F9007046
:100ED000216B636BA06B824A824E92ED026AD2ED67
:100EE000006AD2ED015AC91B2163B5F90270DB1B00
:100EF0006363B5F904703568C01B07EE900AB8EE5D
:100F0000E75A07EE901AB8EEE77A07EE903AF8EE55
:100F1000E77A36EE056A36EE877A77EEA57A0135FE
:100F2000A06382ED026A82ED007AC2ED017A35603B
:100F3000BDE8F087BDE8F0876B4BB4F91600B4F953
:100F40001810B4F91A2018802063598061639A80C0
:100F5000A2633DE7B6F89420322A00F08880002A88
:100F600066D196F89130002BB0D06048D6F8F020CA
:100F70005F4980FB0273D217C2EB23122A80D6F896
:100F8000F42080FB0273D217C2EB23126A80D6F8DA
:100F9000F830A78A80FB0302DB17C3EB2213DB1BAD
:100FA000AB800023CB6086F8913012F003F8F8F79D
:100FB0005BF811F0E7FFFBF74FFD012022F068FA24
:100FC000D6F8D45082E7444E226BD6F8D450B3F50D
:100FD000C87F4FF0000323632B80398818BFD6F8F1
:100FE000D800B7F8008008BF0020B1F5C87F18BF4F
:100FF000D6F8DC30616B02440B440020B8F5C87FA2
:101000006063C6F8D820C6F8DC30688052D0D4F8C7
:1010100038E0D6F8E010A0637144B8F1010FA88061
:10102000C6F8E01068D008F1FF38A7F8008049E75B
:10103000D6F8F000236B00210344C6F8F03021639A
:101040002980D6F8F400636B61630344C6F8F4307A
:101050006980A36BD6F8F800A1630344012AC6F89F
:10106000F830A98075D0013AA6F8942079E72B884A
:1010700020491F48276BA6F8E4300023B5F802E0AA
:10108000B5F804C0C0684B608B602363C6F8F0708D
:101090002B80616BC6F8F41063636B80A16BC6F89C
:1010A000F810A363A6F8E6E0A6F8E8C0C6F8EC00DE
:1010B000AB80D8E7A36BC6F8E030A063A880B2E7A6
:1010C000F4620020804D00201E45002020450020B5
:1010D00078430020246300205C1F0020287D00202E
:1010E0006442002060420020844D00201F85EB51A7
:1010F000E05200204C200020DFF804C1DFF8F0E0CF
:10110000C8328CFB02A9C833D217C2EBE9128CFBA0
:1011100003A9DB17C3EBE913C8316B802A808CFB72
:10112000013CA28ACB17C3EBEC139B1AAB80CEF821
:101130000C0011F03FFFF7F797FF11F023FFFBF7CB
:101140008BFC404622F0A4F9B7F80080D6F8D450C2
:1011500069E7254B86F896101B6886F8902013F4F3
:10116000003334D119462148475C0B2F01F10C01A3
:1011700010D00133182BF7D1B6F8E4101C4B29809E
:10118000B6F8E670B6F8E800D6F8EC106F80A880E4
:10119000D96068E7174FD7F800C05900BCF1000FBD
:1011A00009D001EB030E00EB8E0E9CF801C09EF8F7
:1011B00001E0E645E0D20B44DFF848E00E4900EBE1
:1011C000830000233860AEF800300B60D4E70B4B8F
:1011D0001B78032B01D00B46C5E722F017F8D6F891
:1011E000D450B6F89420C7E770370020081A0408D6
:1011F000E0520020645300206C5300208D490020F1
:101200001F85EB51685300202DE9F0478C4B1B786C
:10121000DB07074644D58B4B8B4D1C788B4E012C3E
:1012200059D01CD3022C07D189498A4A09881288CF
:10123000914201D901241C70EB7AE3B12B89D3B11F
:10124000854B1B78BBB10AF0D9FF002800F09B80CA
:101250002B7B83422CBF0121002131700CE07C49A3
:101260007E4A098810886A7B801A8842E2DAEB7A23
:101270000024002BE2D131782A79632A06D8022C87
:10128000774E00F0BA803378002B5DD1754AAB7A87
:101290008C4238BF0C461470002B4CD1BDE8F0874F
:1012A0006B4B694D19885B88E878CB1A83EAE37247
:1012B0008142A2EBE3721DD32B788B421AD3614B90
:1012C0001C78E01E012861D96749097802294FD0AE
:1012D000012C5E4EA5D15F4A5D491288687B098862
:1012E000121A914239DD5D4A12888A42A4D2002442
:1012F0001C70A1E7B1EB400FE1DC524B1C78E11E02
:10130000012940F29480022ADEDC57494F4E0878CA
:10131000DFF84481DFF844C1DFF838E1002103241D
:10132000022834701C7088F80010ACF80010AEF879
:10133000001081D11FE0012C71D0022C0BD10720AD
:10134000BDE8F04721F07EBF7068381A474B9842DD
:1013500058DD72709AE7BDE8F08702241C706BE7D5
:10136000022AD2DD4049097802294FF0040464D1F1
:101370003949364E09783E48022ACCBF0022012264
:10138000C28081804BE70221317075E7022A9BDC25
:1013900095F800C091FBFCFC0CF1010CBCF1080FAE
:1013A000DFF8B4A0304EA87895F801E096F80080F8
:1013B0002A4CDFF8A090254EA8BF4FF0080C8AF801
:1013C00000C01FFA8CFA10FB0AF01EFB0AFE80B266
:1013D000DFF88CA02080A9F800E000244FF0640E14
:1013E000B8F1020F34701C70CAF804408AF801E0AA
:1013F0007FF439AF0FFA8CF1BDE73078A0B9012343
:1014000077603370C2F164021A4B00FB02F083FB79
:101410000023C017A0EBA3506430707036E708209B
:10142000BDE8F04721F00EBF7368F81A8EE7032C71
:1014300096D10D49097802299AD0044EFCE600BFE6
:101440000875002094260020D06200209A260020F3
:10145000844E0020982600209A4E002096260020D8
:10146000442500208D490020804D00207F96980063
:10147000844D00206BCA5F6B022828BF022010B485
:10148000084C094B207000EB8002C0EBC2020749F8
:101490005DF8044B013003EB4203C0B20B6021F056
:1014A000F7BF00BFB8430020C03E002040630020CB
:1014B00008B511F07FFDF7F7D7FD11F063FDFBF7DD
:1014C000CBFA0120BDE8084021F0E2BF08B50121B8
:1014D0000220FDF775F9094B1B7803F00503052B76
:1014E00008D000210120FDF76BF900210846FDF727
:1014F00067F9FEE715F0D0F9F3E700BF6C34002080
:1015000008B5FBF74DFC11F055FDF7F7ADFDBDE853
:10151000084011F037BD00BF08B511F04BFDF7F7DB
:10152000A3FDBDE8084011F02DBD00BF2DE9F04F2F
:10153000BC4B1E788BB0002E40F08180BA4BBB4C68
:101540001D78BB4FDFF80CB305F00105A4F10A09C3
:1015500054F80A0CB8B14FF0CC0808FB0698FCF719
:10156000BBFE80B154F80A0CFCF7AEFE14F8023C46
:10157000024683B924283BD075B354F80A0CFCF713
:10158000ABFE0028EED10136032E04F1CC04DFD1EE
:101590000BB0BDE8F08F012B2ED0022B33D0032BE4
:1015A00040D0042B00F06981052B00F05781062BF9
:1015B000E3D114F801ECBEF1000F00F0DC81BEF1C4
:1015C000010F00F01F8201360023032E04F8023CB5
:1015D00004F1CC04BCD1DBE7232A54F80A0C00F058
:1015E0008281944B93F832309342B8D1F9F782F963
:1015F000012304F8023CC0E74D2800F06781002376
:1016000004F8023CB9E700233C2804F8023C00F04F
:1016100057813E28B1D10122032304F8012C04F89C
:10162000023CAAE7C028EAD80021042304F8050CEC
:1016300004F8040C04F8061C04F8023C9DE77E4BF9
:1016400018680028A4D0F7F777FCDFF80CA27B4DD0
:10165000DFF8F891DAF80000FCF73EFE002897D09A
:10166000DAF80000FCF730FE09281BD03F2819D01B
:101670002B68002B67D1042800F0BE810C2800F0F5
:10168000CA807F28E6D0A0F12002D2B25E2AE1D83B
:101690000BB92028DED05A1C09F803002A6027F075
:1016A00065F9D7E72C68002C5AD1654FA34607F59A
:1016B0002078BBF1000F08BFBB4610374745F8D173
:1016C000BBF1000F00F05281103FDBF800003A68D8
:1016D000065D135D9E42204402EB040140F044810C
:1016E000661E4E4422460BB9FD2A5CD906F8013F1E
:1016F00001322A6010F8013F11F801EF9E45F2D047
:101700000AB15F4512D04F4827F038F95F4508D33A
:101710005BF8100B27F032F9092027F027F9BB45B9
:10172000F6D9494827F02AF92A680024944291D230
:10173000661E4E4416F8010F27F018F92B68013485
:101740009C42F7D386E70C2865D00A2834D00D28B0
:1017500032D07F2800F0BE80FF2B3FF67BAF92E7B0
:10176000374E002706F52078BB4602E01036464586
:101770000DD0224631684846F7F7BEFE0028F5D165
:10178000B346002FF2D1374610364645F1D13B46DD
:101790005F469B46002B98D1002F3FF45BAF294852
:1017A00027F0ECF8B4E7511C202009F8020029606A
:1017B00009F801300A46A4E727F061F923212348FC
:1017C0002EF0DEFA002800F01581A0EB0900286059
:1017D00090B1431E19F80310202940F0308109EB25
:1017E000030243B112F8011D202903F1FF304FD14C
:1017F0000346002BF6D12B604FF48072002148463F
:101800002EF0A7FA074B1B78002B3FF4C1AE0E4811
:1018100027F0B4F81EE70E4827F0B0F80A4827F082
:10182000ADF817E79C43002008750020FE9A0020C1
:101830005C1F0020905B0020BC380020C0390020D5
:10184000000A0408143504081C350408C0380020B8
:10185000243504083CFF0308B838002014F8063C7F
:1018600014F8051C994273D814F8043C83427FF4A1
:10187000C6AE062304F8023C9BE614F8043C04F8C8
:10188000030C5A40052304F8042C04F8023C74E6C7
:101890002B606C4C002204F5207809F8032002E04C
:1018A0001034444550D0216848460DF0ADFE002864
:1018B000F6D0444548D2E368984700232B609BE765
:1018C000032204F8013C04F8022C56E6022304F833
:1018D000023C52E6013B00225B482B6009F80320E2
:1018E00027F04CF8B6E6594B5949DB78594ADFF8EE
:1018F00090E11060003318BF01230B70564B574A1C
:10190000CEF80030564BC7F800214FF0400E0121B1
:1019100087F808E1C7F8FC00C7F8040187F8095107
:101920005048197027F06BF94F4827F027F84FF40B
:1019300000600CF045FD4D4B93F83230232B3FF403
:1019400055AE14F8023C32E6494827F017F8B4E7E0
:1019500014F8041C08EB03005140013304F8041C84
:1019600004F8063C827208E62246C9E64148103F68
:1019700027F004F8CCE69BE80F000DF1280C0DF1E0
:10198000080888E80F004CF824ED14F8053C14F81A
:1019900003AC0694624623444FF0010C414606A86E
:1019A000ADF822E00793ADF820A08DF824C002F036
:1019B000DDFE40B1029A304B03924146A4F10A0089
:1019C00002930AF029FEDDF80480002304F8023CAB
:1019D000B8F1000F3FF4D7AD54F80A0C20F0E6FE42
:1019E000013654F80A0CC047032E04F1CC047FF4EE
:1019F000AFADCDE52868EBE620480FF0A5FB0BB0B6
:101A0000BDE8F08F14F8053C14F8032C0694234429
:101A100007936E2A4FF0000308930993ADF8202036
:101A20007FF4D1AD06A8F7F7E9FD06A8F7F7DAFDD0
:101A300006A8F7F7D7FD06A8F7F7D4FDC3E50346D8
:101A400027E700BF000A04084C350408B84300200B
:101A500024270020B83800205C200020C5C30008DF
:101A60009C430020503504081C350408905B00207E
:101A70003035040814350408C0AA0020C0380020FE
:101A8000BC3800202DE9F04F2DED028B95B00646B5
:101A900022F05CFC9E4B1D7825B115B0BDEC028B8D
:101AA000BDE8F08F9B4B1B685805F6D5DFF8B09268
:101AB000D9F80020002A00F02781974CD4F828316B
:101AC00003F5F43348339E42C0F01E81934F94F8DF
:101AD0002C113B68C4F82861013184F82C11990756
:101AE00001F1798713F0140F41F0178713F0080FF5
:101AF00094F82C3140F0C28113F0070801F0BA8548
:101B0000282B874B029302F0B1805E209047854BD3
:101B10001B78002B6BD0804C834AD4F83431F31AF5
:101B2000934201F24384DFF83CA29AF80080B8F1B6
:101B3000000F33D1DFF80092D9F80000FCF7CCFB9E
:101B4000C0B201280ED90228784F42F04F813B786D
:101B5000002B42F02A82D4F83C31F31AB3F57A6FA5
:101B600082F0D58272480768002F40D09AF8003082
:101B7000BBB9704BD9F800001B689B781E3B012B4A
:101B80004FF0020142F26882043022F097FA0122FB
:101B900000238AF8002084F8483126E0644807686A
:101BA0002FB3D4F8443140F6B732F31A93421ED91A
:101BB00094F84031002B02F00F81013BDBB284F836
:101BC0004031002B01F0978717F8011B94F848214A
:101BD000076094F8493158480A440133006884F892
:101BE000482184F84931FCF77BFBC4F84461534A2F
:101BF000029B12781B68012A03F101030C9301F088
:101C0000FF824F4B1B787BB1DFF85C91D9F8003035
:101C100053B1414C029BD4F85C21D3F800B0ABEB3C
:101C20000202632A01F21A82DFF8408198F800A0CC
:101C3000BAF1020F01F03A873C4F97F87430032B4A
:101C400001F0DC843F4B1B7873B13F4D2B685BB1D7
:101C5000314CFCF783F8D4F86831039044F61F62E6
:101C6000C31A934200F26081384B1B78002B7FD15E
:101C7000374B1B7843B1284CD4F8B83203F50043F6
:101C8000E8339E4281F03283324B1B78002B3FF4C5
:101C900004AF214E304C314D06F2C1272068FCF7CD
:101CA0001BFB00283FF4F9AE2068FCF70DFB2B78F6
:101CB00080465A1E33B120682A70FCF70DFB0028BD
:101CC000F2D1EAE603223946781E2EF028F896F87B
:101CD000C03296F8C12286F8C38283F47F4383F032
:101CE000FF039B1A1FFA88F89BB2B8EB132FD5D1CC
:101CF00096F8C222DBB29A42D0D1781E1BF024FBA8
:101D00002B7818442870C9E7054B0293FFE600BF03
:101D10009C430020287D0020A8200020E0620020B5
:101D200098A90020F26300203F0D0300200000204E
:101D3000586300205463002050630020F3630020A8
:101D400000640020086400200C64002078640020F7
:101D50008964002012640020186400201C640020A4
:101D6000606300205C63002058500020AE3C0020DF
:101D7000604C2278002A41F03A82DFF8A49199F869
:101D80000040002C40F0AB805B4D2878002842F0EA
:101D90008C805A4C5A4DD4F8B0222978594B93FB79
:101DA000F1F313449E42FFF463AF94F8B432564A01
:101DB000C4F8B062D75CFB0702F17482B80702F185
:101DC000E981790702F12A823A074CD54F4BDFF8B7
:101DD00054810D930DF15009A3F13D0249F8202DD6
:101DE0000021A3F1400203F8401C0223112151708D
:101DF00093704846D8F80010F7F710FC4846D8F81A
:101E00000410F7F70BFCB8F80E30414903EBC3039D
:101E10009B00053381FB0321DB17C3EBA10189B2D2
:101E20004846F7F713FCB8F8103003EB830359006A
:101E300089B24846F7F70AFC364B1B789B0743BF2D
:101E4000B8F8081001F57A7189B24FF47A714846F2
:101E5000F7F7FCFB0C9B98F81420591C0C91484692
:101E60001A7022F019FA94F8B4322978013393FBEE
:101E7000F1F201FB123384F8B432F9E613F0030AED
:101E80007FF43AAE5E209047D9F80030142098478E
:101E9000214B1F4AB3F9043082FB03124FEAE37867
:101EA000C8EBA2080FFA88F85FFA88F022F05AF916
:101EB000C8F3072022F056F9D9F800305E20984781
:101EC000D9F800301C209847504622F04BF9504674
:101ED00022F048F994F82C31D9F800200CE60F4D87
:101EE0002F6E002F41F09D86044B89F80070C3F8D7
:101EF000B062BDE6E463002080640020A8200020DA
:101F000088640020A086010084640020A46300206F
:101F1000676666663E630020EC62002090640020E5
:101F2000816400205092002094F86E31002B41F023
:101F3000EA85DF4B1B6803F00802002A48F60341DC
:101F40004AF60B404BF60F4249F6074704BF0246DC
:101F50000F4613F0040F4FF0190118BF17469B06E8
:101F600084F86E1103D547F4804747F020070AF044
:101F700037F9C7F30909002842F0D282CD4B9B798B
:101F8000002B42F09F82984664204FF0FF3A4FF0BA
:101F9000000C0C970D97ADF83CC0CDF842C0CDF8C1
:101FA00046C0CDF84AC0CDF83890ADF83E80ADF8C7
:101FB00040A08DF84E000CAF0FCFDFF808E384F897
:101FC00005C0AEE80F0097E80F00AEE807002EF856
:101FD000023B71464FF0010C1B0CFE271F20C8224C
:101FE00001F81E39A770A27184F807C0E07094F858
:101FF0007E01207180F0F10383EA0313DAB2130942
:1020000083F0E70343EA022383EAC2031BB283EAB5
:102010000312D2B2C3F3072383EA121343EA022363
:1020200083EAC2031BB283F0C80282EA0212D2B270
:10203000C3F3072383EA121343EA022383EAC203AA
:102040001BB283EA0C0787EA0717FFB2C3F3072224
:1020500082EA171242EA072200EB0C0382EAC70762
:102060000EEB0C0084F87E31278011F8013B7B4099
:1020700083EA0313DBB21A0982EA172242EA032237
:1020800082EAC3031BB29FB281422780EDD183F065
:102090007C0383EA0313DBB24FEA131E8EEA172E8A
:1020A0008EEA032E8EEAC30E0FFA8EFE1FFA8EF909
:1020B000DFF814C2A4F800905FFA8EFE4FEA1929E7
:1020C00084F8289084F827E00CF5D37804F1220AEC
:1020D000DCF80000DCF80410DCF80820DCF80C3038
:1020E00047460FC70CF1100CD445B846F0D1DCF8C8
:1020F00000003860704F9CF8043088F8043007F115
:10210000270884F8CDE184F8CE9117F8011F2868DC
:10211000FCF7E6F8B845F8D194F86F21002A41F0B1
:102120005E856649029B08781B680A2184F86F1156
:10213000002801F09A86DFF894E10128BEF800102B
:10214000059142F2EE820228BEF8028002F000827F
:10215000BEF804100491032802F0DD820428BEF8C2
:1021600006A002F0D3820528BEF8087002F0C782EC
:102170000628BEF80AC002F0BF820728BEF80C107D
:1021800001D0BEF80E2094F87EB10C938BF0300392
:1021900083EA0313DBB24FEA131E494884F804B004
:1021A0008EF07A0E4EEA032E00888EEAC303DFF823
:1021B00020E1C0EB00208EFB009E8644C0171BB2BE
:1021C000C0EB6E200690C3F3072E83EA0310059B35
:1021D000C0B24FF0000963F30F098EEA10130593A4
:1021E0004FF0000E049B68F31F4967F30F0E4FF08A
:1021F0000008002763F30F0861F30F07059BCDF874
:1022000034906CF31F4E62F31F474FF0000C9DF8A3
:102210001820CDF83CE06AF31F48CDF838801097BD
:102220008DF844C08DF8452043EA00230DF13008B5
:1022300083EAC007B8E80F003FB287F0C80989EA0F
:102240000919DFF880E084F805C05FFA89F9C7F35F
:102250000727AEE80F0087EA191747EA092398E82D
:10226000030083EAC9031BB283F023074EF8040B73
:1022700087EA0717FFB2C3F3072282EA17127046F4
:1022800042EA072282EAC70720F814190BF1010B72
:102290004FF0230CFE211622C82384F87EB127803C
:1022A00084F807C00EF1020EA170E270A37111E074
:1022B000E0620020D06200204F220020C87400207D
:1022C0008A490020B0200020AA200020FC9D002088
:1022D0000308208010F8013B7B4083EA0313DBB244
:1022E0001A0982EA172242EA032282EAC3031BB2D6
:1022F0009FB270452780EDD183F0F40383EA031386
:10230000DBB24FEA131E8EEA172E8EEA032E8EEAF8
:10231000C30E0FFA8EFE1FFA8EFCD64FA4F800C033
:102320004FEA1C295FFA8EFE84F81EE084F81F90A5
:102330007968BA683868FB6807F5D37CACE80F00A9
:1023400038697969BA6904F2C518ACE8070004F283
:10235000A71784F8C59184F8C4E117F8011F28680D
:10236000FBF7BEFFB845F8D194F87231002B41F06D
:102370004684C14F3B681922980684F8722140F1C7
:102380000E83BE4BDFF800831B78990741F18687E7
:1023900098F81430042B8CBF4FF003094FF002095A
:1023A000FBF7DCFCB8F81030B8F808200C9003EB11
:1023B00083035B00ADF84A304FF47A70D8F80030F0
:1023C0008DF84C900E93B8F80E1098F814E0D8F8E9
:1023D00004308DF84DE000FB02F24FF0000A4FF0A0
:1023E000FF300DF13009CDF834A010920F93ADF805
:1023F00048101190CC46BCE80F00DFF890E2AEE840
:102400000F009CE80F00AEE807007246182122F882
:102410001C39E17194F87E1184F805A081F07803ED
:1024200083EA0313D8B2030983F0F60343EA0023D7
:1024300083EAC0031BB283EA0310C0B2C3F30723CD
:1024400083EA101343EA002383EAC0031BB283F03C
:10245000C80080EA001C5FFA8CFCC3F3072080EA06
:102460001C1040EA0C2080EACC0000B280F0180377
:1024700083EA0313DBB2C0F3072080EA131040EABB
:10248000032080EAC30301F1010CFE204FF01E0A75
:102490004FF0C80BA0700EF1020E217184F87EC1BE
:1024A000238084F803A084F806B0184612F8011BB4
:1024B000414081EA0111C9B20B0983EA102343EAC2
:1024C000012383EAC10109B288B272452080EDD1AF
:1024D00081F0180181EA0111C9B20A0982EA1023C8
:1024E00083EA012383EAC1031BB29AB261492280C5
:1024F000DBB2120A04910692059384F8272084F82F
:1025000026308E4601F5D37B04F1220ADEF8000066
:10251000DEF80410DEF80820DEF80C30DC46ACE80B
:102520000F000EF1100ED645E346EFD1DEF80000A5
:10253000CCF800009DF81430DFF854A184F8CC31B9
:102540009DF8183084F8CD31D3461BF8011F286858
:10255000FBF7C6FE4A4B5B45F7D1FBF7FFFBD8F80C
:1025600000103B68B8F808200591D8F804100691CF
:1025700013F0140F4FF47A7101FB02F141F07485EE
:102580000F4694F87EB10C908BF06A003D4BDFF85B
:1025900004E1B3F90420109780EA0010C0B20309E7
:1025A00083F0D50343EA002383EAC0031BB283EA26
:1025B0000310C0B2C3F3072383EA101343EA0023D6
:1025C00083EAC0031BB28EFB020E05980D90D21752
:1025D0004FF00008C2EBAE0206980E9083F0C80CD4
:1025E0000F91ADF84A20ADF84480ADF84680ADF8C3
:1025F00048808CEA0C1CCE465FFA8CFCC3F307279C
:10260000BEE80F0087EA1C1747EA0C2787EACC07C9
:10261000DFF878C084F804B03FB2ACE80F0087F070
:1026200021039EE8070083EA0313DBB2C7F3072701
:1026300087EA13170BF1010E47EA03278CE807001E
:1026400087EAC30384F87EE14FF0210B4FF0FE0EC2
:102650001C27C8220CF10C0C84F8058084F807B004
:1026600084F802E0ACF11C01E7701846A2712380E7
:1026700012E000BFAA200020E06200203E6300209C
:1026800075220020EC62002050920020B020002033
:102690004F2200206766666611F8012B424082EAED
:1026A0000212D2B2130983EA102343EA022383EA17
:1026B000C20212B290B261452080EDD182F0680270
:1026C00082EA0212D2B24FEA121B8BEA102383EA8B
:1026D000022B8BEAC20B0FFA8BFB1FFA8BF3DB4F3B
:1026E00023805FFA8BFB1B0A059384F8253084F85E
:1026F00024B007F5D37C04F1220838687968BA68F9
:10270000FB68E646AEE80F0010374745F446F4D1C3
:102710003B88AEF800309DF81430CD4F84F8CAB134
:10272000D04684F8CB3118F8011F2868FBF7D8FD94
:102730004745F8D194F87EC1C64A84F804C08CF0AD
:10274000EB0383EA0313D9B20B0983F0C50343EA11
:10275000012383EAC1031BB283EA0310C0B2C3F3AF
:10276000072181EA101141EA002181EAC00109B282
:102770000CCA81F0C80787EA0717FFB24FF0000EB6
:10278000C1F307210D93CDF838E081EA17130C92BD
:1027900099E8070043EA072383EAC7030FFA83F89F
:1027A000AD4B84F805E088F0310783E8070087EA3D
:1027B0000717FFB2C8F3072383EA171343EA072377
:1027C00083EAC703277A607AA27AE17A94F80CE068
:1027D00094F811801BB25F4087EA0717FFB2C3F37A
:1027E000072383EA171343EA072383EAC7031BB2CD
:1027F000584080EA0010C0B2C3F3072383EA1013E5
:1028000043EA002383EAC0031BB25A4082EA021063
:10281000C0B2C3F3072282EA101242EA002282EA1F
:10282000C00212B2514081EA0111C9B2C2F30723BA
:1028300083EA111343EA012383EAC1031BB28EEA40
:10284000030E8EEA0E1E5FFA8EFEC3F3072383EAA1
:102850001E1343EA0E23677BA07BE17B227C83EA85
:10286000CE031BB25F4087EA0717FFB2C3F307230B
:1028700083EA171343EA072383EAC7031BB25840CE
:1028800080EA0010C0B2C3F3072383EA101343EABF
:10289000002383EAC0031BB2594081EA0111C9B287
:1028A000C3F3072383EA111343EA012383EAC10335
:1028B0001BB25A4082EA0212D2B2C3F3072383EA60
:1028C000121343EA022383EAC2031BB288EA030815
:1028D00088EA08185FFA88F8C3F3072383EA181315
:1028E00043EA082383EAC803A17CE27CDFF8748111
:1028F0001BB2594081EA0111C9B2C3F3072383EA2D
:10290000111343EA012383EAC1031BB25A4082EA4E
:102910000212D2B2C3F3072383EA121343EA02235B
:1029200083EAC2031BB283F0270787EA0712D2B2F9
:10293000C3F3072787EA121747EA022787EAC20785
:102940003FB20CF10103BAB25FFA87F94FF0310CD4
:10295000FE200C2184F87E31C8234FEA122E2280FB
:1029600084F807C0A070E170A37184F81490049FEC
:1029700084F815E07968BA68FB683868B7F810C061
:10298000A8E80F0028F803CB84F8BBE184F8BA91DB
:102990001AF8011F2868FBF7A3FCD045F8D194F87A
:1029A0007671002F41F026812C4B94F87E81B3F98B
:1029B0000010B3F90220B3F904309FED296A677162
:1029C00007EE103A029B1B680C9388F06A0383EAB7
:1029D000031306EE901AD9B20B0983F0D50343EA2C
:1029E000012383EAC1031BB283EA03115242C9B235
:1029F00007EE902AC3F3072383EA111343EA012366
:102A0000F8EEE77AF8EEE66AB8EEC77A83EAC10331
:102A10001BB267EE867A66EE866A27EE067A00209B
:102A200083F0C80ECDED0E7ACDED0D6A8DED0F7AE7
:102A30001090119012908EEA0E1C0DF130095FFA81
:102A40008CFCC3F3072EB9E80F000DE0AA2000208C
:102A500073220020E8490020B0200020EC62002012
:102A600088C3E43A502200208EEA1C1E4EEA0C2E47
:102A70008EEACC0EDFF888C40FFA8EFEACE80F00A9
:102A80008EF01E0799E8070087EA071A5FFA8AFAAC
:102A9000CEF3072787EA1A1747EA0A278CE80700C8
:102AA00087EACA071C214FF0050A4FF01E094FF0B4
:102AB000FE0EC82208F10103E17084F876A184F8C3
:102AC000079084F802E0ACF11001A2710CF10C0C3B
:102AD00084F80480278084F87E3111F8013B7B4024
:102AE00083EA0313DBB21A0982EA172242EA0322BD
:102AF00082EAC3031BB29FB261452780EDD183F008
:102B0000270383EA0313DBB21A0982EA172282EA57
:102B1000032282EAC3031BB21FFA83FCDFF8E483BB
:102B2000A4F800C05FFA83FE4FEA1C2C84F825C08D
:102B300084F824E008F5D37904F1220AD8F80000DB
:102B4000D8F80410D8F80820D8F80C304F460FC732
:102B500008F11008D045B946F0D1E04FB8F8003080
:102B6000A9F8003007F1240884F8CAE184F8CBC141
:102B700017F8011F2868FBF7B3FBB845F8D194F8A4
:102B800077A1BAF1000F41F02F80D54B1B680522C9
:102B900084F877219A0641F17281D24ADFEDD27A28
:102BA000D18907EE101AB8EEC77A13F0140F27EE8A
:102BB000277A01F0F984CD4BDFEDCB6AD3ED007AB3
:102BC000F8EEE77A67EEA67A94F87EC1C84BC94A58
:102BD000B3F90410B2F90620C74FC8488DED0D7A3D
:102BE0008CF0220383EA03135FFA83FE4FEA1E137D
:102BF00083F0590343EA0E23B2F5FA6F83EACE035A
:102C00001BB2A8BF4FF4FA6283EA0318B2F57A7FC9
:102C10005FFA88F8C3F3072EB8BF4FF47A72A2F5B3
:102C20007A728EEA181E642303FB02F34EEA082E22
:102C300087FB03278EEAC80EDA17C2EBA71280FBC8
:102C400001300FFA8EF7CB174FF0000BC3EBA00348
:102C500087F0C8080DF13009CDED0E7AADF84220AD
:102C6000ADF84030CDF830B0CDF83CB0CE4688EA73
:102C70000818BEE80F005FFA88F8C7F3072787EA4D
:102C8000181747EA082787EAC8089D4FDEF800E0D2
:102C900084F804C00FC70FFA88F888F04A0383EA63
:102CA0000310C0B2C8F3072383EA10133A460CF1AD
:102CB000010143EA002383EAC00342F810E900203F
:102CC0004FF04A084FF0FE0C4FF0140E84F87E11BE
:102CD000C82160712380043784F8078084F802C01B
:102CE00084F803E0A171184612F8011B414081EA03
:102CF0000111C9B20B0983EA102343EA012383EAD5
:102D0000C10109B288B2BA422080EDD181F014012C
:102D100081EA0111C9B24FEA111E8EEA102E8EEA25
:102D2000012E8EEAC10E774B0FFA8EFE1FFA8EFC33
:102D30001F464FEA1C2B5FFA8EFE84F81DB084F804
:102D40001CE0596838689A68DB68A4F800C007F589
:102D5000D37CACE80F0038697969B7F8188004971C
:102D6000ACE8030004F2A717ACF8008084F8C3B104
:102D7000B84684F8C2E104F2C31B18F8011F2868A2
:102D8000FBF7AEFAC345F8D15F4B604A1B78127867
:102D9000013B12F00100DBB214BFC0214021172B10
:102DA00003D85B4A134493F814A05A4B1A8893072C
:102DB0001ABF002341F01001012312F4027F18BF53
:102DC000022312F0100F18BF062312F0200F18BFB5
:102DD0001023002841F091814FF0030894F87EC140
:102DE0000C938CF0460383EA0313DAB2130983F0E1
:102DF000920343EA022383EAC2031BB283EA03106D
:102E0000C0B2C3F3072282EA101242EA002282EA29
:102E1000C00212B282F0C80E8EEA0E1E00235FFAC4
:102E20008EFE0320C2F307228DF834A08DF8378080
:102E300082EA1E128DF835308DF836108DF8380084
:102E400042EA0E2899E8070088EACE0E0FFA8EF8BB
:102E5000DFF8ACA0E37188EA0819AAE803005FFA7A
:102E600089F9C8F3072888EA191848EA092181EA8C
:102E7000C90994F808808AF800200FFA89F988EACD
:102E8000090282EA02185FFA88F8C9F3072282EA87
:102E9000181242EA0822607AA17A94F80B906371C2
:102EA00082EAC80212B2504080EA0010C0B2C2F3F7
:102EB000072282EA101242EA002282EAC00212B21B
:102EC000514081EA0111C9B2C2F3072282EA11120C
:102ED00042EA012282EAC1021EE000BF4F22002026
:102EE000E0620020509200200AD7233CE4620020D8
:102EF000EC620020FC9D0020D34D62106766666680
:102F0000B0200020AA2000201053002008750020C7
:102F10004CFF03083C63002012B289EA020989EAE7
:102F200009195FFA89F9C2F3072282EA191242EA03
:102F3000092294F80C80607BA17B84F804C082EAAB
:102F4000C90212B288EA020888EA08185FFA88F80B
:102F5000C2F3072282EA181242EA082282EAC80271
:102F600012B2504080EA0010C0B2C2F3072282EAD7
:102F7000101242EA002282EAC00212B2514081EAF3
:102F80000111C9B2C2F3072282EA111242EA0122F8
:102F900082EAC102E17B94F8109013B281EA030245
:102FA00082EA0212D2B2C3F3072383EA121343EA7E
:102FB000022383EAC2031BB289EA030282EA0212F5
:102FC000D2B2C3F3072383EA121343EA022383EA4C
:102FD000C2031BB283F0320282EA0212D2B2C3F3FE
:102FE000072383EA121343EA022383EAC2031BB2D4
:102FF0009AB24FF0FE085FFA83FE0920C8210CF157
:10300000010C84F802804FEA1228E070A17184F864
:103010007EC1228084F8128084F811E0049B186835
:1030200059689A68B3F80CB00AF5CC7CACE8070094
:103030000AF5D47A8CF80290ACF800B084F8B88124
:1030400084F8B7E117F8011F2868FBF749F9BA457A
:10305000F8D1039BC4F86831FEF706BEDFF83C8365
:10306000BF4FDFF83CA341201AF0EEFBB8F9022075
:1030700087FB0230D217C2EBA00080B21AF0C8FB67
:10308000B8F9002087FB0230D217C2EBA00080B253
:103090001AF0BEFBB8F9042087FB0230D217C2EB4E
:1030A000A00080B21AF0B4FB9AF80010D9F8000022
:1030B000FBF716F994F8608118F0010700F02885F5
:1030C000A84F3A68910640F18180A74ADFF8D48280
:1030D0001278920740F1C48798F81420042A8CBF14
:1030E00003230223039347201AF0AEFBD8F8000015
:1030F0001AF05AFBD8F804001AF056FBB8F80E2064
:103100009A49D9F80000A1FB0232C2F347121146D6
:103110000492FBF7E5F89AF800003968049A11F078
:10312000140F82EA00028AF8002040F0BA86B8F84C
:103130000820642000FB02F01AF036FB98F81470A7
:10314000039BD9F8000043EA8707FFB23946FBF733
:10315000C7F89AF80020D9F80000574039468AF895
:103160000070FBF7BDF894F86081B8F1000F2DD125
:103170007F4F4F201AF068FB38681AF015FB78680B
:103180001AF012FB40461AF00FFB0121D9F800009B
:10319000FBF7A6F8744A9AF800701278D9F8000084
:1031A00002F00108414687F001078AF80070FBF73A
:1031B00097F89AF80020D9F8000088EA0202114630
:1031C0008AF80020FBF78CF894F86081694AC4F80B
:1031D0005CB108F10103DBB2A2FB0312D20802EBDF
:1031E0008202A3EB420384F86031FEF71DBD624BFF
:1031F00062491868FBF73CF800232370FEF7BDBD59
:103200005F4F386800283EF4FCAC4FF0000ADFF84E
:1032100098815C4CAB465546FBF75EF8F8B1F5B9C2
:103220004FF00109AA463868FBF74EF883B27E2BAF
:1032300000F0518498F80120002A49D194F84C11EB
:10324000B1B11B2B84F84C2100F01E840D2B45D00E
:10325000386888F80190FBF73FF80028E3D1AA46C8
:1032600050460CAA48495D4620F0D0FBFEF7C9BC89
:103270007D2B00F0F08594F8502122B180F02003DE
:10328000DBB284F8501194F84B21062A10D8B4F818
:103290004E1138681944A4F84E11A118013281F872
:1032A000543184F84B21FBF717F80028BBD1D6E73F
:1032B000B4F84E2188F8019013449BB21A0A52FACE
:1032C00083F3FF2BA4F84E31386802D12F4DA3E7CA
:1032D0003868FBF701F80028A5D1C0E73868A4F8E2
:1032E0004E21FAF7F9FF00289DD1B8E794F8BC32D7
:1032F000C4F8B862012B40F2738594F8BD222449CA
:10330000981801EB8001013202F00102CF6A84F8C3
:10331000BD22BFB11F4D0D950DF15009123DA523E2
:1033200049F8205D802284F8103115233146484643
:1033300084F8112184F81231B847002840F0D18474
:1033400094F8BC32144A013382FB0312A2EBE372FD
:1033500002EB42029B1A84F8BC32FEF795BC00BF18
:1033600067666666E06200203E6300201F85EB51C1
:10337000E8490020CDCCCCCC7C640020A4630020A4
:103380004C630020A8200020F2210020FC21002016
:103390004CFF0308CD21002056555555EC62002006
:1033A0005C50002050920020200000209E4A9F4B3D
:1033B00092F80BE0029AD4F8381110681B889C4AE6
:1033C000401A4FF47A71DFB201FB0EF11B0A9777B6
:1033D000177588424FF00007D377537597701771B0
:1033E00080F0EA84934BDFF870C21B689249934FD8
:1033F0000868DFF8689289683F688CFB038EDB17EA
:10340000C3EB6E1303F5FA739BB293761B0AD37664
:1034100089FB00A389FB01A9C017C917C0EBA30052
:10342000C1EBA90107F5EA43DFF834E21077303346
:10343000001282F8201009121B12DFF828829EF871
:1034400000E0507782F821108CFB0790F917C1EB50
:10345000601182F823307A4B98F814A083F81AA0F0
:10346000783130371EF0020F82F8241082F8227073
:1034700000F09F84D8F800E0724AD8F80400DFF822
:10348000E8B182FB0E714FEAEE77C7EBA1510391D1
:1034900082FB0092C117C1EBA25203990BFB01E121
:1034A00001EB410149000F460BFB020B0497B946A3
:1034B0000BEB4B0B644F4FEA4B01059187FB099BCC
:1034C00087FB01194FEAA949CDF81C90B8F80E9076
:1034D0000399B8F8088002EB820209EBC90902EBF4
:1034E0008202089201EB81074FEA89020599039253
:1034F00007EB8707049A0697CF17C10F0991049825
:1035000052494FEAAB4BD2174FEADE7E83F809E00F
:10351000ABEB020E01FB1E020798069908F5FA783C
:10352000BAF1050F1FFA88FAA0EB0708059F474874
:1035300083F815A04FFA8EF909EB8109414600FB8B
:1035400018789DF8240098730898414FDFF81CE123
:1035500049B201EB80018CFB020B4FEAE27204924C
:10356000039ABEF800E08CFB08C087FB02C74FEA55
:10357000E27C049AC2EB6B120392364A1FFA89F975
:103580001288ADF8102083F80A90039A83F813E0AC
:1035900089B24FEAE8784FEA112BC8EB6010CCEB08
:1035A000A7174FEA1A284FEA192C4FEA222A9DF84A
:1035B0000C2083F810B04FEA202983F80BC0D97390
:1035C000C7F3072C4FEA1E2134BF4FF0320B4FF0E8
:1035D000330B1A739DF8102083F80DA0587483F8EC
:1035E000129083F81680DF7183F808C0197583F88C
:1035F0001BB01A77C4F83461FEF795BADFF8709003
:10360000D9F80000FAF758FE00283EF41BABD9F8B1
:1036100000000121FAF74CFE0222002387F87420F3
:1036200088F80030FEF70EBB8C4E0020844E002040
:1036300020640020E4620020B8620020E8620020DC
:103640004C6400206BCA5F6B83DE1B4340420F005B
:10365000D34D6210544A00201F85EB5167666666A1
:103660003E63002050920020806967FF486300207D
:10367000C43D00205E209047D9F8003002209847D2
:10368000FF2019F0E7FD0378FF2B00F0998490F9F3
:1036900001304FEAE3785FFA88F8D8B220F062FD93
:1036A000404620F05FFDD9F800305E209847D9F8F9
:1036B000003003209847FF2019F0CCFD0378FF2B42
:1036C00000F07984B0F90830D8B2C3F3072820F0AD
:1036D00049FD404620F046FDDA4B1B78042B7DD097
:1036E000DFF88CB3B4F82E119BF80020DFF884A328
:1036F00091FBF2F302FB13139BB2BAF80010A4F88B
:103700002E314FEA03181FFA88F8642303FB0123C4
:103710005200B3FBF2F348EA0328C3F303225E200E
:10372000D9F800301FFA88F848EA02089847D9F813
:103730000030062098475FFA88F020F013FD4FEA2A
:10374000182020F00FFDC049B4F82E214B7ABAF8AA
:1037500000A00132012BA4F82E2100F00C874A7B37
:103760000AEB8A031FFA83FA002A40F0C084D9F8D2
:1037700000305E209847D9F800303A209847B34B84
:10378000A3FB0A384FEA58181FFA88FB5FFA8BF040
:1037900020F0E8FC4FEA1B2020F0E4FCD9F80030D0
:1037A0005E209847D9F800303B209847642303FBFC
:1037B00018A39BB2A648053380FB0320DB17C3EB9D
:1037C000A000C0B220F0CEFC002020F0CBFCDFF83F
:1037D000A88298F80630002B40F051843B689F0681
:1037E00040F11282DFF894A29AF80030980700F1B5
:1037F000EA83DFF88C820027BB46D9F800305E20D0
:103800009847D9F8003001209847584620F0AAFC84
:10381000384620F0A7FCD9F800305E209847D9F848
:10382000003009209847002020F09CFC002020F068
:1038300099FCB8F8123098F814B0B3F5967F0AD90D
:1038400094F82C2102F00F02072A04D842F20F7BD1
:103850009B4528BF9B46D9F800307B4F5E20984798
:10386000D9F80030052098473B7A002B00F0668598
:10387000ABF1200307EE903A9FED767AF8EEE77A07
:10388000F6EE006A67EE877ABEEE007AF5EEC07A51
:10389000F1EE10FA58BFB0EE667A77EE877AFDEE59
:1038A000E77ACDED027ABDF908B05FFA8BF020F02F
:1038B00059FCCBF3072020F055FC9AF80020002398
:1038C00092070A930B9300F1658394F83031012B32
:1038D00000F06083B7F90030DFED5F6A07EE103A61
:1038E000B7F9023007EE903AB8EEC77AF8EEE77A09
:1038F00027EE267A67EEA67ABDEEC77AFDEEE77A66
:103900000CA88DED0C7ACDED0D7A20F04DFC94F8DD
:103910002C31D9F80020FEF7F3B85E209047D9F893
:103920000030302098474D4BD3F800805FFA88F084
:1039300020F018FCC8F3072020F014FC94F82C3178
:1039400013F003087EF4C8AA454AD4F82811454B61
:103950009142186840F28F8380EAE073A3EBE07332
:103960003A4A1BB282FB03124FEAE37ACAEB621AAD
:103970004FF0640808FB1A380FFA88F80FFA8AFA31
:103980005FFA88FB5FFA8AF2C8F30728CAF3072AAE
:10399000D9F8003002925E209847D9F80030102004
:1039A0009847029A104620F0DDFB504620F0DAFBE3
:1039B000D9F800305E209847D9F800302120984788
:1039C000584620F0CFFB404620F0CCFB3B68D9F8AE
:1039D0000020FEF78BB8DFF8AC809FED238A4FF014
:1039E000240A5E2090475046D9F8003098471F4B74
:1039F000F8EC016A9B8A07EE103AF8EEE66AB8EE38
:103A0000C77A0AF1010AC6EE877A5FFA8AFA67EE88
:103A1000887AFDEEE77ACDED027ABDF908B05FFA5B
:103A20008BF020F09FFBCBF3072020F09BFBBAF13B
:103A3000270F02D0D9F80020D3E73B68D9F800203F
:103A4000FEF750B88D4900208C4E00201F85EB51A9
:103A500067666666E4380E3F0050C347E8620020A0
:103A60003F4B4C00E462002000007A44F4620020E6
:103A70009A4E0020844E0020D06200203E63002039
:103A800050920020246300203868FAF725FC0028B3
:103A90007FF4DEAB386884F84A9188F80190FAF731
:103AA0001BFC00287FF4BFABFFF7D9BBFAF756F930
:103AB000D14B1B68A0EB030B40F6B8339B4500F2DB
:103AC000BF81CE4B1A793A2A00F04284002388F84D
:103AD0000030FEF7B7B8386884F84AA184F84BA1E3
:103AE00084F84C9188F801A0FAF7F6FB00287FF4DF
:103AF0009AABFFF7B4BB94F8481194F84931C04829
:103B00004A1CFEF76AB8013B84F86E31FEF704BB2D
:103B1000BC4A1288D30513D4D00600F1E682910680
:103B200000F11D85530600F13C85100700F1548516
:103B3000D10700F1588512F0020F0CBF04270C27A3
:103B4000B149B24A0B78D27803F001030AB143F0CD
:103B500002035320039319F077FEAD4A128802EB5B
:103B6000820202EB8202900080B219F051FE002026
:103B700019F04EFEA74AA8491288D9F80000C2EBF6
:103B8000C212520081FB023111444FEAE278C8EBC5
:103B900061285FFA88F84146FAF7A2FB9AF80020FC
:103BA000039BD9F800001F4388EA020800218AF825
:103BB0000080FAF795FB3946D9F80000FAF790FB38
:103BC0009AF80020D9F800007A40D2B211468AF85B
:103BD0000020FAF785FB94F86081FFF7C6BA013A36
:103BE00084F86F21FEF7C0BB0AF1FF3A84F877A191
:103BF000FFF72FBA013F84F87671FEF7C0BF013B93
:103C000084F87231FEF7CBBE1B077FF580AE834B85
:103C100093E803000CAB83E80300184620F0C4FAD5
:103C200075E60024DFF8108227464FF0500A02E0C4
:103C3000DBB283F3118815F804B0601C59462844A0
:103C400019F0B0FC002840F025810BF101031C4461
:103C5000EFF311838AF312882A6E9442E8DB002284
:103C6000DBB22A6683F31188FEF73EB94FF0000AF3
:103C70005E201F6884F82CA19047D9F80030DFF847
:103C8000BC8117209847504620F06CFA644BA3FB88
:103C900007239B0BA8FB03125209C2EB0212A3EBF2
:103CA0008203D8B220F05EFAD9F800305E2098473F
:103CB000D9F80030182098475A4BA3FB07239B09DB
:103CC000A8FB03125209C2EB0212A3EB8203D8B283
:103CD00020F048FA504620F045FAD9F80020FDF7C8
:103CE00014BF0C9EAE424FF000014FD941F22100AB
:103CF00015F8013B81EA03235A0013F4004F80EAD0
:103D0000020192B289B208BF11464A0080EA02035A
:103D100011F4004F99B293B218BF0B46590013F437
:103D2000004F80EA010289B292B208BF0A465300EE
:103D300012F4004F80EA03019BB289B208BF194612
:103D40004A0080EA020311F4004F99B293B218BFFF
:103D50000B465A0013F4004F80EA020192B289B276
:103D600008BF11464B0011F4004F80EA03029BB2DA
:103D700092B208BF1A46530080EA030112F4004FC2
:103D80009BB289B208BF1946B542B1D14846F5F792
:103D900083FC25490C9D25486D1A152DA8BF1525B6
:103DA0002A462AF0DBFE224A94F8BC321570FFF74F
:103DB000C9BA2D22DA761DE41E4B02991B780968D8
:103DC000C4F83811013B012B3FF60CAB1021022344
:103DD00091701371FFF706BB20F0A6F9FDF705BF40
:103DE0000E4A02EB8302D76AFFF793BA20F08CF9F0
:103DF00001233B70FDF7B6BEB43C00209C3C002084
:103E0000506300203C63002008750020904900208A
:103E1000844E00208A490020030820804CFF0308BC
:103E200073B2E745D34D6210B8210020903A0020CC
:103E3000A53A00208D490020CD4203088988888852
:103E4000C44AB2F8623100210133A2F8623188F825
:103E50000010FDF7F7BE386884F85091FAF73CFA85
:103E600000287FF4E0A9FFF7FAB901468446074627
:103E700082460490804605900246FEF784B99FED85
:103E8000B67A13F0140F08BFF0EE477A7EF493AEC3
:103E9000FEF79ABE41463A2019F0E0FA0743FFB216
:103EA000D3E6AE4A1068FFF747B9AD49AD4B009372
:103EB000A1F13F07AC4BAD4A0B9101F8404C0CA867
:103EC000AB490A97F5F7C0FC0A9F7B1C0A933C702C
:103ED0000A9B2922591C0A911A700A9BEA22591C32
:103EE0000A911A700A9BC822591C0A910CA81A70D0
:103EF00029F0F6FE00F101080CA942460A982AF0C2
:103F00002DFE0A9A02EB080301330A9302F80840D7
:103F10000A9B5A1C0A921C700A9B5A1C0A921C701B
:103F20000A9B5A1C0A921C700A9B5A1C0A921C700B
:103F30000A9B5A1C0A921C700A9B5A1C0A921C70FB
:103F40000A9B5A1C0A921C700A9B5A1C0A921C70EB
:103F50000A9B5A1C0A921C700A9B5A1C0A921C70DB
:103F60000A9B5A1C0A921C700A9B5A1C0A921C70CB
:103F70000A9B0122991814A80A911A7050F8283D3A
:103F8000DB1B3B7020F088F9724B2C70C3F8B062D9
:103F9000FDF76EBE98E80C0001210AA884F83011E4
:103FA0000A920B9320F000F9B1E4C4F83C6187F861
:103FB0000080FDF7D7BD4FF000084046FFF787BBF4
:103FC0004046FFF76BBBDFF8C081D9F80030694F7E
:103FD0005E209847D9F8003011209847B8F80E2095
:103FE0004FF4F36B0BFB02F287FB0237D217C2EBE5
:103FF0006737F8B220F0B6F8C7F3072020F0B2F820
:10400000D9F800305E2098471920D9F80030984739
:10401000B8F80E30584A0BFB03F382FB0301DB17A1
:10402000C3EB611382FB0321DA17C2EB6112642137
:1040300001FB1233D8B220F095F8002020F092F85E
:104040009AF80030B8F8087099077FF5D4AB5FFA9A
:1040500087FB3F0AFFF7D1BBFAF72AF9FDF797BDB7
:1040600001230393FFF73FB83C4B1F6807EB87071B
:104070007F00FEF786BAC346C246424688E4D9F8B6
:104080000030DFF808B1DFF808A15E209847D9F8C2
:10409000003028209847DBF800308AFB032ADB1722
:1040A000C3EBAA0A5FFA8AF020F05CF8CAF3072093
:1040B00020F058F8D9F800305E209847D9F8003041
:1040C00004209847B8F80830002B40F04B82DBF80A
:1040D000083083F310085FFA88F020F043F8C8F343
:1040E000072020F03FF8FFF779BB342728E59BF83D
:1040F00000309AFBF3FAFFF73ABB204AD278002A45
:104100000CBF4FF004084FF00508FEF767BE01230F
:10411000D9F800003B70FAF7D7F80746D9F8000045
:10412000FAF7D2F87F067DF41DAD8A2800F04382AD
:104130008E287DF417AD9AF80030002B7DF42EAD5B
:104140000F48104B03602D2384F840310768FDF7BA
:104150000DBD00BFA820002000000000E462002088
:10416000A4630020BE430020A4350408AC35040835
:10417000B835040889B5F8141F85EB519049002023
:10418000586300202064002050920020B862002074
:1041900067666666CF4AD04B0D920DF15008A2F1CA
:1041A0003D0048F8200D1988DFF85493A2F1400330
:1041B00000204FF00A0E02F8400C082283F801E0BC
:1041C00040469A70F5F742FAD9F80030C349DA1739
:1041D00081FB0313C2EBA30399B24046F5F736FA0D
:1041E00008F00CF8D9F808900C9B4FEA1942591CBA
:1041F0000C911A700C9B4FEA1922591C0C911A70E1
:104200000C9B5A1C0C9283F800900C9B5A1C0C922D
:104210001870404620F040F8FDF7D3BDAD4B0D932C
:10422000A3F1400900222121A3F13D0A03F8402C0B
:1042300089F8021089F80120CDF830A012F0AAFF09
:10424000A74BA84A1B88A84900280ABF11464FF06F
:1042500003084FF004085A0500F19F81D80700F1C8
:10426000BE8103F00203A14A002B1CBF4FF00308DC
:10427000114642469E482AF071FC0AEB080314A836
:104280009C4A013340F8203D9B1A00220AF808207E
:1042900089F8013020F000F8FDF796BD4FF00109D4
:1042A000FEF77EB8DFF86C929FED938AB9F9023081
:1042B000884A0D9207EE903AF8EEE77A0DF1500831
:1042C00067EE887AA2F14003FDEEE77AA2F13D01A4
:1042D00048F8201D02F8400C0822CDED027A5A70F1
:1042E0001E229A70BDF808104046F5F7AFF9B9F9EB
:1042F000003007EE903AF8EEE77A404667EE887AAB
:10430000FDEEE77ACDED027ABDF80810F5F79EF9DB
:10431000B9F9043007EE903AF8EEE77A404667EED6
:10432000887AFDEEE77ACDED027ABDF80810F5F750
:104330008DF940461FF0B0FFFDF740BD5FFA8BF0EE
:104340001FF010FF4FEA1B201FF00CFFFFF7B5BA5C
:104350009978039318460FF021FE00287FF4B6AB3E
:104360005D49664F664A09886648674CF961DFF81F
:10437000A891116803689268F962B4F86211C7F8ED
:104380006CB0FB63FA64D9F80000F965F7F7EEFF4B
:10439000834600287DF451AC5146D9F80000F9F766
:1043A00087FF039B94F86421DB780493642A4FF021
:1043B000040387F8743040F0198194F86531072BB5
:1043C00008BF84F865B194F86521504B079207EB5C
:1043D000021A0393DAF804100691084629F080FCCB
:1043E000DAF8083005935FFA80FA184629F078FC6D
:1043F0005FFA80FB454B079A06990AEB0B000830E1
:10440000D87122F00F00987202F00F020BEBCA0075
:104410005A739873524603F10F002AF09FFB059BD5
:1044200019463B4B0AF1090018445A462AF096FBFC
:104430003648C37903F1010ACBB1013B5FFA83FC33
:104440000CF1080CDFF8D4E084440023073010F8A6
:10445000012B5A409300D10883EA420301F018016E
:1044600053404EFA01F253408445DBB2EFD1284A63
:1044700004980AF802302AF04DFB94F865310022C6
:10448000013384F8653184F86421039BDDF80CA0C6
:104490009B785BB11AF80510D9F80000F9F720FFF6
:1044A00001359AF80230EDB2AB42F3D894F864319A
:1044B0000322013384F8643187F8742088F80020DF
:1044C000FFF79EB80E4B8046B3F900A06420FDF7BD
:1044D0005EBD00BFA4630020844E00206766666650
:1044E0003C6300208835040890350408A035040892
:1044F000676300206563002058A08B4120000020E6
:10450000B8620020E4620020A82000206892002009
:104510006E920020EC620020C43D00200007090ECE
:10452000854B864A1B88927903EB830303EB830355
:104530004FEA83081FFA88F8002A40F0FA804FF00B
:10454000FF330FFA83FA07F059FE40B2FDF71FBDA3
:1045500011469446174692460492FDF714BE24274E
:10456000FFF7EEBA07F04AFE1FF0FCFD00201FF037
:10457000F9FDFFF733B9D9F800305E209847D9F834
:104580000030392098475FFA8AF01FF0EBFD4FEAC0
:104590001A201FF0E7FDFFF71AB94FF0030868492A
:1045A00067E61027FFF7CCBA138907EE903AF8EECA
:1045B000677AFEF709BB634B1B6898067DF5D2AAA4
:1045C0009AF80030002B7DF4E9AA5F485F4B036046
:1045D0002D2384F84031B9E52027FFF7B1BA5C49B3
:1045E0004FF0040845E60827FFF7AABA97F8753098
:1045F00058481A0704BF0133DBB2072B28BF012339
:104600004FEA031B07EB0B025FFA8BFA92F810E0FC
:10461000514A039200EB0E010022087A4E498A7239
:1046200001F10D0207EB0B014AEA0E0E012882F898
:1046300000E0C96802F1010C0DD90238C0B200F1E6
:10464000020E9644624602F8011B72454FEA1121A0
:10465000F9D101308444BB4421F0600201339BF85E
:104660001110DBB20A43082B8CF800200CF1010278
:1046700049D04FEA031B07EB0B00384990F810E0D4
:1046800034487044511A007A01EB000C0AF1100A08
:10469000BCF1130F5FFA8AFAC4DDC9B28A1DD2B227
:1046A000039842F0400E80F807E002F1010ADFF8BB
:1046B000B8E0CAB105315FFA81FB0BF1080B834406
:1046C0000EF1010C00221CF8010B5040820082EA1E
:1046D0004002C1084240224801F0180140FA01F1AD
:1046E0004A40E345D2B2EED104980AF80E2087F88A
:1046F00075302AF00FFAC8E61146FDF744BD1146A1
:104700009446FDF740BD1549511AC6E71146944637
:104710001746FDF738BD1146944617469246FDF7F9
:1047200032BD114694461746924604929046FDF7D4
:104730002ABD0C4B1B6804E7844E0020D062002089
:1047400094350408E0620020586300204C64002087
:10475000983504084CFF03086892002075920020E9
:104760000007090EB86200206E9200202DE9F04F7C
:1047700095B0B0F908500D81EDB2442D00AF0C4654
:10478000904600F04684064643D9812D00F07F8391
:1047900000F29880542D00F0CC8040F2D6806E2D2F
:1047A00000F00584802D40F0D380764B93F800A074
:1047B0000AF1020A1AF0FF0A00F09780724BDFF844
:1047C000F481724EDFF8F0B19A4403F101090A2531
:1047D00016E0322D01F06083A5F13C00C0B2132831
:1047E00041F2648300232268511C21601570226805
:1047F000CA4502F101012160137076D019F8015BFE
:104800000A2DE6D1BBF80030FF2BA8BFFF23DBB297
:10481000E9E7052D00F0EB8320D8022D00F0818020
:1048200040F21483032D00F0B983042D40F09080F2
:10483000574920462A46F4F7E7FE00212046F4F7C0
:104840002BFF22680021531C0125236028462B469C
:10485000543711706381BD46BDE8F08F242D5ED0C2
:1048600040F2AA82282D00F05B83382D70D10A68AF
:10487000484B0125511C21601570226805215019F3
:104880002060117022680A2150192060117022687E
:104890000021501920601170226819785019206089
:1048A0001170226859785019206011702268997827
:1048B000531923602B461170284654376381BD4637
:1048C000BDE8F08FA02D18D040F29582B82D00F0F1
:1048D0006383FE2D3CD1304D05F1080635F8021BEF
:1048E0002046F4F7D9FEB542F8D101252B462846DB
:1048F00054376381BD46BDE8F08F284B08461968E0
:10490000F4F7B2FE264B20461968F4F7ADFE254BAE
:10491000196820460125F4F7A7FE2B46E7E7224B4E
:10492000F6E70422214920460125F4F76DFE2B46C7
:10493000C2E70B6800215A1C226019702268012509
:10494000531923602B461170B6E7522D3FF479AF0F
:104950002146284608F066FC03460028C5D1742D80
:1049600000F08782772D29D13268716891421EBF8D
:10497000531C336011780E4A08BF194620461EF0BA
:1049800045FEB2E7614D002088FF03084426002061
:10499000BE430020AB3E0020844D0020107AFF1F54
:1049A000147AFF1F187AFF1FF43F002024360408F2
:1049B00025270308676666666C260020F52D01F042
:1049C000C183762D00F02D83472D01F0EE82292D35
:1049D000326801F0D182392D01F09B82212D01F046
:1049E000AB8270680B3D811AEF2D00F229840FF223
:1049F000080E5EF825F000BF155901084152010864
:104A00004152010841520108415201084152010836
:104A10004152010841520108415201084152010826
:104A20004152010841520108415201084152010816
:104A30004152010841520108415201084152010806
:104A400041520108415201084152010841520108F6
:104A500041520108415201084D59010841520108D3
:104A6000F358010841520108C95801084152010890
:104A70004152010841520108A15801084152010860
:104A80002B58010841520108F95701084152010809
:104A90008B5701084152010879570108415201081A
:104AA0002157010841520108875601084152010867
:104AB000415201084152010841520108EB480108E6
:104AC00041520108B55B01084152010841520108F9
:104AD0009B5B010841520108415B010841520108FA
:104AE000415201084152010841520108FD5A010892
:104AF000415201084152010841520108BD5A0108C2
:104B0000415201086F5A01084152010841520108FF
:104B10002F5A01084152010841520108415201082F
:104B20004152010841520108415201084152010815
:104B3000C159010841520108715D01084152010843
:104B4000B75C010841520108095C010841520108A3
:104B5000E15B01080F5E0108F35D010841520108A5
:104B600041520108415201084152010841520108D5
:104B700041520108415201084152010841520108C5
:104B800041520108415201084152010841520108B5
:104B900041520108415201084152010841520108A5
:104BA0004152010841520108415201084152010895
:104BB0004152010841520108415201084152010885
:104BC0004152010841520108415201084152010875
:104BD0004152010841520108415201084152010865
:104BE0004152010841520108415201084152010855
:104BF0004152010841520108415201084152010845
:104C00004152010841520108415201084152010834
:104C10004152010841520108415201084152010824
:104C20004152010841520108415201084152010814
:104C30004152010841520108415201084152010804
:104C400041520108415201084152010841520108F4
:104C500041520108415201084152010841520108E4
:104C600041520108415201084152010841520108D4
:104C700041520108415201084152010841520108C4
:104C800041520108415201084152010841520108B4
:104C900041520108415201084152010841520108A4
:104CA00041520108415201082D5E0108415201089C
:104CB0006B56010841560108415201084152010852
:104CC0004152010841520108415201084152010874
:104CD0004152010841520108415201084152010864
:104CE000415201084152010841520108E3550108AF
:104CF000915501085955010841520108B75401085E
:104D00009D5401082B540108415201081154010817
:104D1000A55301087D5301086B5301080F53010887
:104D200041520108DF520108415201084152010875
:104D3000B552010887520108735201084B5201080D
:104D400023520108F9510108CD510108B55101085C
:104D500041520108415201084152010841520108E3
:104D600041520108415201084152010841520108D3
:104D700041520108415201084152010841520108C3
:104D80004152010841520108955101084152010860
:104D9000415201083D5101084152010841520108A8
:104DA00041520108D95001084152010841520108FD
:104DB000415201086F500108202D7FF4C9AD0B68E6
:104DC000B14D591C6A7821601A7023682A78591CE1
:104DD00021601A702368AA78591C21601A702989E9
:104DE0002046F4F759FC23686A79591C21601A702F
:104DF0002268A97927E5822D7FF4AAAD0B68A34A22
:104E0000A34D1178A04A581C2060197011892046C2
:104E1000F4F742FC9F4B22681B88FF2B02F1010133
:104E2000A8BFFF2321601370A96881F3100189B224
:104E30002046F4F731FC296801F30F0189B22046BE
:104E4000F4F72AFC944B22681978FCE4012D7FF4D6
:104E50007FAD0B680022591C21601A7023685A1C10
:104E600022601D7022682521531C23602B4611707F
:104E700022E53268716891421EBF531C336011787D
:104E8000864A08BF194620461EF0C0FB2DE5844B1C
:104E90001E78033616F0FF063FF427AD814BDFF88E
:104EA00030821E4403F1010A4FF00A0920E0B9F1F3
:104EB000500F00F0F887B9F1320F01F00D80A9F121
:104EC0003C00C0B2132841F20B800025294623681C
:104ED0005A1C2260204683F80090F4F7DDFB294637
:104EE0002046F4F7D9FBB2453FF4FFAC1AF8019B1A
:104EF000B9F10A0FDBD16C4B9D68196805EB85058C
:104F00004FF6FF736D009D42A8BF1D469942A8BF92
:104F1000194625EAE57521EAE171ADB289B2D6E715
:104F20000B68DFF8B091614E591C022221601A70A3
:104F300023684FF006085A1C226083F8008023681B
:104F40000A22591C21601A70236801255A1922600F
:104F50001D70B9F800102046F4F79EFBB9F8021056
:104F60002046F4F799FB23685A19226083F80080E1
:104F700023685022591921601A7023680022591998
:104F800021601A7031882046F4F786FB718820462C
:104F9000F4F782FB2B468FE4454BB9E40B685A1CAF
:104FA0000A601D700B685A1C0A601D7049E4394B79
:104FB0000A681B88364DFF2BA8BFFF23511C2160B8
:104FC0001370A96881F3100189B22046F4F764FBDD
:104FD000384B20461988F4F75FFB296801F30F016D
:104FE00089B220460125F4F757FB2B4664E40B22D7
:104FF00031492046F4F708FB082230492046F4F7EF
:1050000003FB012507222E492046F4F7FDFA2B4623
:1050100052E4002A3FF469AC2A4B136001252B4669
:105020004AE43268511C31601278002A01F04A814A
:10503000102A01F07E811E46194625686B1C2360EC
:1050400020462A70F4F710FB31462046F4F70CFB9B
:105050001D4B20461968F4F707FB20460021F4F7A2
:105060001BFB00212046F4F717FBFFF7EABB174BA9
:105070001B78DB0700F1E4800125FCF74DFAF7F718
:10508000EBFC2B4618E400BFD06200209A4E0020B3
:10509000B8620020844E00208D4900208527030837
:1050A000614D002098FF0308F82500202C260020E1
:1050B000703700208A4900202C360408383604084E
:1050C0004436040805D201086C250020087500202C
:1050D0003C260020D05200203046F4F783FA336893
:1050E000B8851A46591C316012F8021B326087F8E5
:1050F0002E105A7887F82F20DA1C32609A7887F8B9
:1051000030201A1D3260DA7887F831205A1D32605B
:105110001B7987F8323007F12C000023BB86F4F7A7
:10512000BBF9C94AC94B1268801A4FF0010561F1F9
:105130000001C3E906012B46FFF7BEBB531C3360D9
:1051400013780F2B7CD8911C3160C3EBC303C0498B
:105150005078C854D01C30600B4491785970111DA0
:105160003160D1789970511D31601179D970911DDC
:10517000316051791971D11D31609179597102F104
:1051800008013160D2799A71012524F031F92B465A
:10519000FFF792BB3046F4F725FADFF8C482A8F88F
:1051A0000E003046F4F71EFA0125A8F80C002B4635
:1051B000FFF782BB3046F4F715FAA64A00EB8000F1
:1051C0004300012513802B46FFF776BB1146531C85
:1051D0003360A14B11F8020B18703160517859708F
:1051E000D11C316091789970111D3160D278DA70DC
:1051F00001252B46FFF760BB3046F4F7F3F9DFF8E3
:105200008C82A8F810003046F4F7ECF9A8F81200E8
:105210003046F4F7E7F90125A8F814002B46FFF70C
:105220004BBB1346511C316013F8020B3360D31C87
:105230005178336092781FF029FC00287FF455AB39
:105240004FF0FF352B46FFF737BB1346511C31603B
:10525000824913F8020B08703360814953788B70D0
:10526000D31C33607B4B92789A7001252B46FFF755
:1052700023BB7C4B7C4918684E22012529F06EFC2B
:105280002B46FFF719BB1146531C3360774B11F8BF
:10529000020B1870316051785970D11C31609278CE
:1052A0009A703046F4F79EF9714B0125D8802B4651
:1052B000FFF702BB3046F4F795F9DFF8B481A8F8A0
:1052C00000003046F4F78EF9A8F802003046F4F7F3
:1052D00089F90125A8F804002B46FFF7EDBADFF89D
:1052E000B09199F80030002B3FF4FFAADFF8A481B9
:1052F00000253046F4F776F911F0BAF999F8003044
:10530000A8EC010A01359D42F3DBFFF7EEBA0D2947
:1053100096D1531C33601578072D91D8DFF878911A
:1053200030464FF00C08F4F75DF908FB05F809EB7F
:105330000805A8803046F4F755F9E8803046F4F7C0
:1053400051F9336828811A46591C316012F8021B42
:10535000A97232605B78EB723046F4F72BF90125C5
:1053600049F808002B46FFF7A7BA3046F4F73AF998
:10537000404B012518802B46FFF79EBA531C336023
:105380001078060601F149803B4B1B78DD073FF59D
:10539000ACAA032828BF00200125FCF76DF82B4696
:1053A000FFF78ABA531C3360304692F800A0F4F736
:1053B00001F981463046F4F7FDF805463046F4F72A
:1053C000F9F880463046F4F70DF93046F4F70AF95B
:1053D0003046F4F713F9BAF1000F00F0EC87BAF198
:1053E000100F7FF482AA194BC3F804909D60B8F1A6
:1053F000000F02D0214BC3F800802149214B02222B
:10540000081F01251A7020F05DF82B46FFF754BAEB
:10541000194B1B78D8073FF568AA0125FCF770F8EF
:10542000F7F71AFB2B46FFF747BA134B1B78DA073F
:105430003FF55BAA144A1378012543F00403137067
:105440002B46FFF739BA00BF98A90020702300202F
:1054500084360020F0520020344B002028750020B4
:10546000E052002040630020901F0408D852002022
:10547000384300201C4B0020087500206C250020BC
:1054800078230020124A00203E630020287F00205D
:10549000614D002098380020C4350020C44B1B7893
:1054A000D9073FF522AAC34B4FF4C87201251A80D1
:1054B0002B46FFF701BA09297FF7C2AEDFF8308328
:1054C0001346511CD8F80050316013F8021B2970A4
:1054D00033605378AB70D31C33609378642B02F144
:1054E0000401A8BF64236B713160D378642B02F18F
:1054F0000501A8BF6423AB7131601379EB71931D73
:1055000033605379642B02F10701A8BF64232B7227
:1055100031609379EB7002F108033360D3792B711A
:105520003046F4F75FF8726833686881D11A002951
:105530000CDD591CD8F800003160521A002A197885
:10554000417203DD9A1C32605B784370012511F0D3
:1055500093FE2B46FFF7B0B9974B1868D31C014652
:1055600021329D1E356013F8035C0D705D1E3560A1
:1055700013F8025C4D70336013F8015C8D700333D7
:10558000934201F10301ECD124F096FBFFF7ADB992
:10559000531C336013788949002B00F007870B7880
:1055A00043F00203901C0B70854D306053782B75CF
:1055B0003046F3F7FFFF28603046F3F7FBFF6860E3
:1055C0003046F4F70FF828813046F4F70BF87D4A9F
:1055D000E8811378012543F0020313702B46FFF78F
:1055E0006BB9C1F34705122D3FF62AAEC5B107F1DD
:1055F000500307F12A0903EB450AC846AAF1260A17
:105600003046F3F7EFFF28F8020FD045F8D16E4B84
:1056100039F8022F23F8022FC845F9D1112D09D8E6
:105620006A4A6B00023B13440021223223F8021F16
:105630009A42FBD1664A01231D461370FFF73CB91D
:10564000531C6448336001781378002940F0898640
:1056500004220270604A9B001380F8F77FFB5F4BC7
:10566000012518622B46FFF727B9DFF88881002350
:105670003046C8F80030F3F79DFF0125C8F8000058
:105680002B46FFF719B90723B1FBF3F3C3EBC305AF
:10569000491B7FF4D5ADDBB203F1FF395FFA89F91D
:1056A000002B3FF422A9DFF838A109F101090D46CA
:1056B000531C336092F90010494B4FF0000805E08D
:1056C00008F10108B8F1060F3FF4BAAD93F90220D2
:1056D0008A4203F10803F3D10AEBC80B30468BF87A
:1056E0000210F3F77FFF33682AF838001A46591C76
:1056F000316012F8021B8BF8031032605A788BF875
:105700000420DA1C32609A788BF806201A1D326069
:105710000135DB788BF805304D45C9D1FFF7E5B889
:10572000531C336013780E2B3FF68AAD911C316009
:105730005578032D3FF684AD2A48062101FB03F17D
:10574000431802F1030E5D71C6F800E095784554E8
:10575000111D3160D1785970511D316011799970E6
:10576000911D31605179D970D11D316092791A71D2
:1057700001252B46FFF7A0B8531C33601A4B127853
:105780005A7501252B46FFF797B8531C33601578DF
:105790001F2D3FF655AD05297FF452AD3046F3F786
:1057A00009FF124B43F8250015F00EFDFFF79DB8D9
:1057B0000875002078430020406300203E630020ED
:1057C00050920020104A0020863B0020883B002099
:1057D000AC3B0020AC4800208A4900207023002008
:1057E000905B00207C370020645B0020F464002084
:1057F0004463002070370020C34D05F14008304657
:10580000F3F7F0FE3368A5F88000591C1A463160A2
:1058100012F8021B85F8821032605B7885F88330BD
:105820000435A845EBD1FFF760B8531CB74D336082
:1058300013782B723046F3F7D5FEA8833046F3F782
:10584000D1FE28833046F3F7CDFE32686883531CBF
:1058500033601278EA747268D31A032B00F38685DA
:105860003368D11A05290EDD5A1C32601B78EB72A1
:105870003046F3F79FFE3368E8605A1C32601B78AD
:105880002B7433687268D21A002A7FF72EA85A1C2C
:1058900032601B7885F8213001252B46FFF70CB8C4
:1058A000531C33609A4915780D70C01A00287FF791
:1058B0001CA8931C33605378003318BF01230125C3
:1058C0004B702B46FEF7F8BF3046F3F78BFEDFF840
:1058D0006082C8F800003046F3F784FEC8F8040080
:1058E0003046F3F77FFE0125C8F808002B46FEF787
:1058F000E3BFDFF840820023C8F800303046F3F7FA
:1059000059FED8F8003001250343C8F800302B4673
:10591000FEF7D2BF7F4810294FF000020B4628BF88
:105920001023026042608260C2600274002B3EF469
:10593000DCAF3268411E13440132326012F8010CB0
:1059400001F8010F9A42F7D1FEF7CFBF511C316029
:1059500015783B62132D3FF673AC911C3160507883
:105960007A621DF08DFE00283FF46AAC7A6A6A49BB
:10597000007801F82500D01C306001EB8505907897
:105980006870101D3060D078A870501D306012799A
:10599000EA7001F150003B6A02E00431884207D00E
:1059A0000A78002AF9D18D78CA789542F5D2012378
:1059B0005A4A83F00103012513702B46FEF77CBF82
:1059C000574B1B68002B3EF490AF1FF073FEFF286F
:1059D0003EF48BAF3046F3F705FE3F2840F260857A
:1059E000DFF85481002588F8005033687268A8F801
:1059F0000400D21A012A7EF778AF1A46591C31608A
:105A000012F8021B88F8021007F1500032600022E1
:105A10005D7800F8242D1FF01FFE97F82C30AB4264
:105A20003EF463AF28461FF03BFEFEF75EBF3D4BE2
:105A30001B78012B3EF659AF531C11463360DFF83B
:105A4000FC8011F8023B88F80230D31CC01A316088
:105A5000012892F801E0336040F332853046F3F7D5
:105A6000C1FD0125A8F800002B46FEF725BF531CF9
:105A7000336092F80080B8F1110F3FF6E1AB931C50
:105A80003360294D537805F818303046F3F7AAFDF6
:105A900040F6CA039842A8BF184640F2EE23984247
:105AA00005EB4801B8BF18460125A0F2EE222B46AF
:105AB000192092FBF0F24A70FEF7FEBE1346511C0D
:105AC0001A4D316013F8021B2971336053786B71E2
:105AD0003046F3F787FD336828805A1C32601B7804
:105AE000AB713046F3F77EFD336868805A1C326034
:105AF0001B78EB7101252B46FEF7DEBE0125F4F77E
:105B00001BFD2B46FEF7D8BEF4640020645B00202A
:105B100010530020BC520020283D0020A00F002080
:105B20000C750020DE3F0020343E0020544300204E
:105B300018350020F43F002010750020E03F0020C1
:105B4000531C3360C44B1278DFF844831A7000236F
:105B5000C8F800303046F3F72DFD3368D8F8002040
:105B6000BE49BF4D10435A1CC8F8000032601B7874
:105B70000B723046F3F736FD28603046F3F732FDFE
:105B800068603046F3F72EFDA8603046F3F72AFD33
:105B90003046F3F727FDFEF7A8BEB24B02F108012D
:105BA0000132326012F8010C03F8010F9142F7D173
:105BB000FEF79BBE1346511C3160AB4913F8025BE4
:105BC0008D70336055784D7083423EF48EAED31C99
:105BD0003360A64B92781A7401252B46FEF76CBEF3
:105BE0001346511C3160A24913F8020BC870336090
:105BF000A04953784B71D31C33609F4B9278DA7075
:105C000001252B46FEF758BE3046F3F7EBFC304635
:105C1000F3F7E8FC3046F3F7E5FC3046F3F7EEFC2B
:105C20003368964D1946581C2A68306011F8020BEB
:105C300082F82C003160597882F83610D91C316016
:105C40009B7882F837303046F3F7D8FC3046F3F7CC
:105C5000D5FC3046F3F7D2FC3046D5F80080F3F798
:105C6000C1FCA8F83A003046D5F80080F3F7BAFC3A
:105C700033687268A8F83800D11A01290ADD591C66
:105C80002A6831601B7882F82E303046F3F7B6FC74
:105C900033687268D31A032B0BDD3046D5F80080C9
:105CA000F3F7A0FCA8F8320030462E68F3F79AFC10
:105CB000B086286868E4531C3360704DDFF8D481E7
:105CC000137888F805303046D5F80090F3F78AFC51
:105CD000A9F820003046D5F80090F3F783FC7268ED
:105CE0003368A9F81E00D11A072919DD3046F3F7E9
:105CF00079FCA8F80A003046F3F774FCA8F80C0009
:105D00003046D5F80090F3F76DFCA9F82200304634
:105D1000D5F80090F3F766FC33687268A9F82400A0
:105D2000D11A03290BDD3046F3F75CFCA8F80E000E
:105D30003046F3F757FC33687268A8F81000D21A9F
:105D4000002A05DD591C2A6831601B7882F826304C
:105D5000F6F7DAFD21F01EF9494B1B68002B00F025
:105D600048832868012523F0D7FB2B46FEF7A4BD06
:105D70001346511C3160DFF81C8113F8021B88F8B0
:105D8000021033603F4953780B70D31C33603E4D93
:105D900093782B71131D3360D378092BA8BF092387
:105DA0003046AB70F3F71EFC336872682880D11A56
:105DB000012905DD3046F3F715FC33687268E88188
:105DC0009A4207D05A1C32601B78003318BF012357
:105DD00088F80730F6F798FD336872689A423EF407
:105DE00084AD5A1C32601B78EB7001252B46FEF700
:105DF00063BD531C33601378002B00F005834FF410
:105E00000040012508F0DCFA2B46FEF755BD1F4B7C
:105E10001B7813F001017FF413AA531C3360107830
:105E2000012506F0EFF82B46FEF746BD1346511C40
:105E3000316013F8025B3360D31C50783360917883
:105E4000002D00F0F582012D7EF44FAD06F098F99B
:105E50002B46FEF731BD00BF10530020645B0020CD
:105E600018350020635B00200053002070230020C1
:105E7000E052002018740020F052002040630020FF
:105E800008530020D4520020287F002008750020ED
:105E9000F43F0020287500203388FF2BA8BFFF2384
:105EA000DBB2FEF7A0BCA24BFFF726B817F0D2F981
:105EB00000283EF497AC03780A2B28D8B0F90230BA
:105EC00088FB0312DB17C3EBA2039BB2FF2BA8BF17
:105ED000FF23DBB2FEF787BC98E82200FFF70EB87D
:105EE00017F0B8F900283EF4F0AF03780A2B3EF61D
:105EF000ECAFB0F90430B0F9061003EB830383F381
:105F0000500521EAE171ADB289B2FEF7E0BF00238E
:105F1000DFE7531C336013780A2B00F0C48130464E
:105F2000F3F76CFB3046F3F769FB01253046F3F7D6
:105F300065FB2B46FEF7C0BC1346511C31607D4DFE
:105F400013F8021B6970336053782B70D31C3360D5
:105F50009378AB703046F3F745FB33682881591CC2
:105F60001A46316012F8021B697132605B78AB71BE
:105F700001252B46FEF7A0BC531C336013780A2B77
:105F800000F08B81502B7FF400AE3046F3F72AFBF4
:105F9000DFF8A881A8F800003046F3F723FB0125BD
:105FA000A8F802002B46FEF787BC726835687B6252
:105FB0003046551BF3F7FEFA052D38627B6A00F276
:105FC00060818026B346012594E80600521A103AF3
:105FD000B242B8BF1FFA82FB574A396A92683A61E7
:105FE000521A9345396A7B622046FA6088BF1FFACD
:105FF00082FBF3F739FB7B6A002B00F02181002D37
:1060000040F0FD802368C7F800D05D71C0B0053353
:10601000C7F808D0FB61BBF1000F00F0E6813B6AD6
:106020003A69934280F0DE81AA463E6A7D627C60D6
:1060300080255446FB681C1B3F4BB4F5807F28BF6E
:106040004FF480749B6832199A4288BF9C1BF4F706
:10605000E7F92246BC6830462146F4F7A7F8F9690B
:10606000B86104EB000C0B787B6164452ED2DFF83D
:10607000D0900CF1FF3C04F1FF3E1EF8013F09EB0C
:10608000830219F823405688ECB100234FF40042F4
:1060900004F1FF3816424FEA520202D00878284332
:1060A00008706D0806D10AF1010A4D701FFA8AFACC
:1060B00001318025D34503D8F44533D8434531DB3E
:1060C00001339C42E6D1F445D7D1F9617B6ABA69C4
:1060D00013449BB2D3457B6206D97B6A3A6A1C465D
:1060E000D6183B699E42A5D37C68802D1CBF0AF15F
:1060F00001031FFA83FA0AF1020189B22046F3F77D
:10610000CBFA2368796A01255A19226020461D704E
:10611000F3F7C2FA2368534423602B46D7F800D024
:10612000FEF7CABBFB697C681A463B7D1370DCE74F
:1061300030260020D0620020041000202C260020F1
:10614000A8FF0308336872689A4240F0C080C24BCF
:10615000FF221A704FF0000AC04D19F0AFFB5146F4
:106160002022BF4885F800A029F0F3FD87F82CA075
:1061700097F82C30072B00F2F280DFF81C93B84E12
:10618000524697F82C3003EB430309EBC3035B7CC7
:10619000E3B197F82C3003EB430309EBC303202151
:1061A0005B699BB197F82C3003EB430309EBC30306
:1061B000586946F82200F8F70DFA2B7856F82300B4
:1061C000F8F7C6FA2A780132D2B22A7097F82C3042
:1061D0000133DBB287F82C3097F82C30072BD0D95D
:1061E0002368591C21601A70B8F1000F3EF47DAB92
:1061F0009C4BC8F8003001252B46FEF75DBB9A4B3F
:106200003A6A9B68D4F800905A449A4200F2968009
:10621000F4F706F95A464946386AF3F7C7FF236888
:1062200003442360B042BEF660AB002100E0236867
:1062300001305A1CB04222601970F8D1FEF755BBEC
:10624000002DDCD159462046F3F726FA23685A1C64
:1062500022601D70844B26689D683B6A0BEB03022D
:10626000AA4240F2EB803B6AED1AF4F7D9F82A46CD
:106270003146386AF3F79AFF236803442360FEF738
:1062800034BB3046F3F7AEF9326871687B6A9142ED
:10629000834645D106461D4696E63046F3F7A2F9F9
:1062A000DFF8F88176E6931C3360704B51781970F3
:1062B000D11C316091785970111D3160D2789A707B
:1062C000FEF713BB6A4B93E84200FEF7B6BE5A1CBA
:1062D00019463260604811F8022B027031605B7819
:1062E0004370042A03D9FF2A7EF4ABAA32E761493E
:1062F0000978994205D8022A7EF4A3AAFF2B7EF4DE
:10630000A0AA236801255A1922601D70B8F1000F58
:106310003EF4EBAA584BC8F800302B46FEF7CCBA37
:10632000511C316012781D46131C064618BF01230C
:106330004AE6494B59689E68FEF77FBE3A6AA3EB6E
:106340000208F4F76DF842464946386AF3F72EFF23
:10635000236803442360002D3EF4C7AA62E7524637
:106360003EE704297EF4C1AAFFF774B93046F3F77B
:1063700039F9A8843046F3F735F933687268E88450
:10638000D11A03297FF76DAA1A46591C316012F8F9
:10639000021BA97732605B7885F820303046F3F72E
:1063A00021F9336872686884FFF75BBA0B7803F0F1
:1063B000FD03FFF7F7B82E4B1020C3F800905D6087
:1063C00007F0CEFF2D4A137843F001031370B8F1A4
:1063D000000F3EF48AAA2A4B0125C3F800802B4601
:1063E000FEF76ABA7D62AA4685E6DA46C7F824B0A7
:1063F00081E624482449254A254B036001250B608A
:1064000013602B46FEF758BA224A1368012523F47D
:10641000004313602B46FEF74FBA00F07F000328BD
:1064200028BF0020012505F0C7FE2B46FEF744BA21
:10643000012523F0C4FA2B46FEF73EBAF3F7F0FF2E
:106440005A463146386AF3F7B1FE23680125034402
:1064500023602B46FEF730BA702300205BA7002094
:106460001CA7002079C2030804100020AB3E0020C6
:10647000E8490020614D002011D201083E63002050
:106480006C250020F08400204485002044890020F1
:10649000D583000838630020687E0020D052002099
:1064A000C50800F0070301350133EDB2DFF8308095
:1064B0002846194688F8013016F036FEFFF793BAE1
:1064C000064B91781A88012512FB0EF22B4692FB9F
:1064D000F1F2A8F80020FEF7EFB900BF3A51002012
:1064E000107500202DE9F04F2DED0C8B364C97B038
:1064F0006368069020469847002800F07D82B4F833
:10650000A870002284F85120002F67D1656AB4F981
:106510003860206AB4F93A20A16AB4F93C30521BC1
:10652000301A2A4DE0625B1A04F12C0094F85210E4
:1065300063630795226313F02FFE2B68990042F1E5
:106540005981D4ED0B7ADFF88CB0DFF88C909BED9D
:10655000405ADBED415A9BED426ADBF80C31D9F829
:106560000020F8EEE76AD4ED0C7AB8EEE77AD4EDC5
:106570000D7AF8EEE77A013376EE856A37EE257A02
:1065800077EE867A9342CBED406A8BED417ACBED84
:10659000427ACBF80C3101F0D1840D4B049393F87F
:1065A00000C0BCF1140F03F06785DBF8142100254F
:1065B000062A01F2A685DFE812F0F71863181D1706
:1065C000761891170F18850D3C750020287D002046
:1065D000804D0020A023002094450020D44BD549B5
:1065E000079391F801901B68D348DFF8A0830490CB
:1065F0004FF47A71B1FBF3F3C3EB431603EB86035D
:10660000DE00B6B2B7420578B8F9060003F01F8283
:10661000D4F87CE0B4F93820236E0EF1010107EEC6
:10662000902A13440129E1672366F8EEE77A03F024
:106630001882D4ED1B5AD4ED1D6A07EE101A37EEFE
:10664000E56AB8EEC75A012F86EE057A37EE257A4D
:1066500077EEC77A84ED1C7AE7EE866A84ED1B7AC2
:10666000F0EE667AC4ED1E6AC4ED1D6A03F076860C
:10667000D4F890E0B4F93A20636E0EF1010107EE10
:10668000902A13440129C4F890106366F8EEE77A63
:1066900003F0FF81D4ED205AD4ED226A07EE101AE0
:1066A00037EEE56AB8EEC75A012F86EE057A37EE67
:1066B000257A77EEC77A84ED217AE7EE866A84ED53
:1066C000207AF0EE667AC4ED236AC4ED226A03F004
:1066D0001D86D4F8A4E0B4F93C20A36E0EF10101AC
:1066E00007EE902A13440129C4F8A410A366F8EE1B
:1066F000E77A03F0E781D4ED255AD4ED276A07EE57
:10670000101A37EEE56AB8EEC75A012F86EE057A01
:1067100037EE257A77EEC77A84ED267AE6EE276A99
:1067200084ED257AF0EE667AC4ED286AC4ED276A16
:1067300003F0DF85DFF858B2A8F80600B4F8A830F7
:10674000049A013B1578A4F8A83007990023072D77
:106750004B608B60CB6040F05781F7F7FFFA049BEA
:10676000DFF828821D78069BC01A9BF82131A8F813
:1067700000000993002B40F04D816E4B5B79002B9C
:1067800001F009836D4B1B78013BDBB2072D8BF8C1
:10679000213102F0E58300230A93694ADBF82C31AA
:1067A000D2ED006A674A9FED686AD2F800A0604A9D
:1067B0000792069ADBED4AAADFF8D8819BED499A49
:1067C0009FED62AADFED62BA9FED62CA9FED62BAE9
:1067D000DFF8C491614FCBF82C21D31A07EE903A21
:1067E000F8EE677AB7EE007AC6EE279A08F11C0336
:1067F000002508935A4B05932E4677EE6A8A68EE79
:10680000A68AF4EEC78AF1EE10FA88BFF0EE478A46
:10681000544B98ED008A2B44D3ED007AF5EE407A84
:10682000F1EE10FA17D0504B2B4493ED007A78EE2E
:10683000476AB0EEE66AF4EEC67AF1EE10FA08D5D1
:10684000F5EEC06AF1EE10FACCBF37EE878A37EE6C
:10685000678A83ED008A454B1A8893073FD0022E42
:106860003DD0434B9AF82E1033F9163007EE103A0C
:10687000089B07EE901A2B44F8EEE76AB8EEC77A49
:10688000D3ED007A4B42A6EEA77A700007EE903A5D
:10689000F8EEE77AB4EEE77AF1EE10FA0AD407EEF2
:1068A000901AF8EE677AF4EEC77AF1EE10FA88BF24
:1068B000F0EE477A2F4B30490344085EB3F90C30B1
:1068C000C01A07EE100AB8EEC77AD007E7EE4A7A88
:1068D00041F1F781294B93ED008A27EE888A079BC7
:1068E0009BF864212B4493ED01DA78EE4DCA002A1F
:1068F00000F0E780224BDBF8682106991B688A1AB2
:106900009A4240F3DE809AF84830022B02F08A83E4
:10691000022E04F045871B4B1B68990700F19280FB
:10692000194B87ED00CA1B689342C0F2C48035E062
:10693000187D002028750020804D0020D4520020B2
:10694000988900204063002000247449CDCCCC3DC0
:10695000AE47813F000000000000C8428C5000207C
:10696000805000208C890020DC2400203C63002023
:10697000E8240020E0520020EC620020748900200E
:10698000A0890020E06200209C890020844D002026
:10699000A0230020D024002098500020F7EE007A99
:1069A000F4EEE7AAF1EE10FA40F18B8007991F4B45
:1069B000D1ED017A93ED007AF0EEE77AF4EEC77A42
:1069C000F1EE10FA7DD5D1ED027AF0EEE77AB4EE71
:1069D000E77AF1EE10FA74DDD1ED037AF0EEE77AA2
:1069E000B4EEE77AF1EE10FA6BDD114B1B689A07F3
:1069F00061D51049104B45E0104BDFF844B01D78CD
:106A00000493072D3FF4A9AE9BF821310993002B85
:106A10003FF4B3AE581E8BF82101012D01F0C28363
:106A200017B0BDEC0C8BBDE8F08F00BFA88900202B
:106A3000E0620020EC620020E0520020804D002047
:106A4000A0230020D64BD749DFF8C8E331F916C0A0
:106A50009EED008ADFF8C0E387ED00CA03EB460035
:106A600028EE0A8AB0F90C00A0EB0C0007EE900AA1
:106A7000F8EEE77ADEF8000027EE888A904278EE9A
:106A80004DCA8BDAB3F90C20B1F900E0C648AEEB81
:106A9000020E00688EEAEE72A2EBEE72824210DA0B
:106AA000B3F90E30B1F90220D21A82EAE273A3EBF5
:106AB000E273984205DD002318468BF86431F7F73E
:106AC00055FEBA4B2B4493ED000A059B29EE000AB4
:106AD000022E20EE2C0AA3EC010A059304F01D8679
:106AE000B34BD7ED006A93ED007AB24BD3ED007A49
:106AF000B14B93ED006AB14B67EE277A2B4427EE3A
:106B0000A87AD3ED007A67EE277AF0EE665AECEEBB
:106B1000A75AB1EE467AF4EEC75AF1EE10FA08D44D
:106B2000B4EEE56AF1EE10FA8CBFB0EE657AB0EE25
:106B3000467A9BED4A6AF7EE007AB4EEE76AF1EE28
:106B400010FAACBF0123002343B1F0EEE66AF0EE89
:106B5000C77AF4EEE67AF1EE10FA01D587ED007A05
:106B6000022E04F00485964A964B52F826001B68C4
:106B7000B0EE4D0A9847944A944B52F826001B6891
:106B800098479AF8373023B1914B1B88002B01F0BE
:106B90000581B0EE4C8A8F4B38EE400A2B4493EDC2
:106BA000008A83ED000A9AF8483030EE480A20EE59
:106BB000298A53B3884B1B78DB0741F17580F7EEC8
:106BC000007AF4EEE7AAF1EE10FA9BF86431C1F214
:106BD000D586002B01F08781DBF86831069AD31A3D
:106BE0007E4A12689A4210DD7D4BD3ED007AF0EEBA
:106BF000ECCAF4EEE7CAF1EE10FA42F11C8200236F
:106C000018468BF86431F7F7B1FD764B9BF8742189
:106C10002B4493ED000A29EE000A20EE088A89ED44
:106C2000008A32B9059B87ED00CA03ED01CA89EDE0
:106C300000CA0136032E08F1040809F1040907F11E
:106C4000040705F104057FF4E3AD049B1B78072BD3
:106C500001F09986012B02F08881002308939BF8AC
:106C60007C31002B41F0AB825F4B604A07931B687D
:106C70001668D80496F82C7001F1AB80DFF89CA15F
:106C80005B4ABAF81A105B4B5B4D92ED006AD3ED8C
:106C9000004A5A4A5A4BD5ED036AD3ED005AD2ED59
:106CA000007A92ED014A92ED025A8BED636A07EE8B
:106CB000101AB8EEC77A74EEC63A012336EEC77AD8
:106CC0008BED616ACBED603ACBED644A8BF8943181
:106CD000C7EE258A338D5A4206EE102A494ADFED67
:106CE0004A6AD2ED005A494AD2ED004AB7EE007A1C
:106CF000F4EEC78A75EEA45AF1EE10FA88BFF0EEF2
:106D0000478A75EEA75AB8EEC66AF4EEE68AF1EE47
:106D100010FA07EE903AF4EEC65AB8BFF0EE668A63
:106D2000F1EE10FACBED678AB8EE677A01F13E8496
:106D3000F4EEC75AF1EE10FA88BFF0EE475A314B25
:106D4000DFED336AD3ED017A304BD3ED014A77EEB4
:106D5000A47A65EEA65A77EE847AB4EEE76AF1EE8D
:106D600010FA08DCB4EEE77AF1EE10FA8CBFB0EE60
:106D7000676AB0EE476A234A738DD2ED027A9FEDBF
:106D8000247A5A4204EE902A75EE277AF8EEE44A05
:106D900026EE076AF4EEE47AF1EE10FA4BD43FE007
:106DA000E0520020EC620020A489002048890020E5
:106DB000EC84002098000020BC8900205489002029
:106DC000F4840020F08400204885002044850020C1
:106DD0003C6300200C25002008750020A0890020BD
:106DE000AC89002060890020287D002040630020BD
:106DF00040510020B05200209C4E00208C500020BA
:106E000040430020805000200000000098500020E7
:106E10006F12833A748900209C890020645B0020F3
:106E200007EE103AF8EE474AF4EEE74AF1EE10FAB0
:106E300088BFF0EE674AE94BDFEDE97A5B7864EEF4
:106E4000A74A0BB9F1EE644A002F41F0F287F7EE42
:106E5000003AE44F3E78002E03F0E280E24BDFED93
:106E6000E37A93ED025AD3ED016A93ED037A26EEAD
:106E7000055AA5EEA65AA4EE875A23EE855AB4EE1B
:106E8000E75AF1EE10FAB4BFB0EE674AB0EE454AE9
:106E900098BFF0EE457A012E8DED0E5A03F0FF807B
:106EA00093ED067A93ED053AD3ED076A26EE077A5D
:106EB000A5EE837AA4EEA67A23EE877AB4EEE77A7B
:106EC000F1EE10FAB4EEC47A8CBFF0EE676AF0EE21
:106ED000476AF1EE10FA88BFF0EE676AB4BFF0EED1
:106EE000447AF0EE477A022E8DED0F7A00F0DE80C4
:106EF00093ED0A7A93ED093A93ED0B4A26EE077A61
:106F0000A5EE837AA4EE847A23EE877AB4EEE67A4D
:106F1000F1EE10FAB4EEE77A8CBFB0EE664AB0EE4E
:106F2000474AF1EE10FA98BFF0EE446AA8BFF0EEBF
:106F3000477A032E8DED107A00F0B88093ED0E7A2B
:106F400093ED0D3A93ED0F4A26EE077AA5EE837A7C
:106F5000A4EE847A23EE877AB4EEE67AF1EE10FAA4
:106F6000B4EEE77A8CBFB0EE664AB0EE474AF1EE77
:106F700010FA98BFF0EE446AA8BFF0EE477A042EEC
:106F80008DED117A00F0928093ED124A93ED113A53
:106F900093ED137A26EE044AA5EE834AA4EE874ABF
:106FA00023EE844AB4EEE64AF1EE10FAB4EEE74A74
:106FB0008CBFB0EE667AB0EE447AF1EE10FA98BF6C
:106FC000F0EE476AA8BFF0EE447A052E8DED124A26
:106FD0006CD093ED164A93ED153A93ED177A26EEA1
:106FE000044AA5EE834AA4EE874A23EE844AB4EE0F
:106FF000E64AF1EE10FAB4EEE74A8CBFB0EE667ADC
:10700000B0EE447AF1EE10FA98BFF0EE476AA8BFEE
:10701000F0EE447A062E8DED134A47D093ED1A4ACE
:1070200093ED193A93ED1B7A26EE044AA5EE834AB6
:10703000A4EE874A23EE844AB4EEE64AF1EE10FA53
:10704000B4EEE74A8CBFB0EE667AB0EE447AF1EE69
:1070500010FA98BFF0EE476AA8BFF0EE447A072E08
:107060008DED144A22D093ED1E7A93ED1D3A93EDE7
:107070001F4A26EE077AA5EE837AA4EE247A27EE3D
:10708000237AB4EEE67AF1EE10FAB4EEE77A8CBF2A
:10709000B0EE666AB0EE476AF1EE10FA8DED157A41
:1070A00098BFF0EE466AA8BFF0EE477A77EEE67A30
:1070B000F7EE006AF4EEE67AF1EE10FACBED4A7ADA
:1070C00043F3FD8786EEA77A022EDDED0F7A27EED9
:1070D000055A67EE877A8DED0E5ACDED0F7A2DD0D9
:1070E000DDED107A67EE877A032ECDED107A25D08C
:1070F000DDED117A67EE877A042ECDED117A1DD081
:10710000DDED127A67EE877A052ECDED127A15D075
:10711000DDED137A67EE877A062ECDED137A0DD06A
:10712000DDED147A67EE877A072ECDED147A05D05F
:10713000DDED157A27EE877A8DED157A2C4B1B68DD
:10714000DA0041F1D283F6EE008ACBED678A002E99
:1071500002F08A87264A274B1068D978264A9BF97D
:1071600094319BED646A0A9107EE103A1178DFF8CA
:1071700090E0224A079BDFF88CC0DBED635A1B6866
:107180000592BDEEC66A9EED005AB2F906E0BAF865
:107190001A209CF800900B9216EE10CA00F0805254
:1071A00001F00108BDEEE56A0A990C9203F01000A7
:1071B00003F4805203F480030D93DBED606ADBED92
:1071C000617AB8EEC77A16EE103A002941F0BA801B
:1071D0000549DDED0E5A91ED006A15E010530020CF
:1071E0006F12833A614D0020B04200200000000081
:1071F000285100209049002008750020FC9D0020A7
:10720000AC4200204C7F0020002841F0DE8428EEB4
:10721000866AC34AA5EE876AF0EE675AE6EE265AFA
:10722000BDEEE56A16EE10EA16EE100AE645A8BFB6
:1072300060467345C8BF184606EE100AB8EEC66A27
:10724000012E82ED006A00F0DC8091ED046ADDED34
:107250000F5A28EE866AA5EE876AF0EE675AE6EEC8
:10726000265ABDEEE56A16EE10EA16EE100AE6455D
:10727000A8BF60467345C8BF184606EE100AB8EEB0
:10728000C66A022E82ED016A00F0BB8091ED086AA9
:10729000DDED105A28EE866AA5EE876AF0EE675A91
:1072A000E6EE265ABDEEE56A16EE10EA16EE100A74
:1072B000E645A8BF60467345C8BF184606EE100AEB
:1072C000B8EEC66A032E82ED026A00F09A8091ED54
:1072D0000C6ADDED115A28EE866AA5EE876AF0EE9B
:1072E000675AE6EE265ABDEEE56A16EE10EA16EE8D
:1072F000100AE645A8BF60467345C8BF184606EEAB
:10730000100AB8EEC66A042E82ED036A79D091EDB8
:10731000106ADDED125A28EE866AA5EE876AF0EE55
:10732000675AE6EE265ABDEEE56A16EE10EA16EE4C
:10733000100AE645A8BF60467345C8BF184606EE6A
:10734000100AB8EEC66A052E82ED046A59D091ED96
:10735000146ADDED135A28EE866AA5EE876AF0EE10
:10736000675AE6EE265ABDEEE56A16EE10EA16EE0C
:10737000100AE645A8BF60467345C8BF184606EE2A
:10738000100AB8EEC66A062E82ED056A39D091ED74
:10739000186ADDED145A28EE866AA5EE876AF0EECB
:1073A000675AE6EE265ABDEEE56A16EE10EA16EECC
:1073B000100AE645A8BF60467345C8BF184606EEEA
:1073C000100AB8EEC66A072E82ED066A19D091ED52
:1073D0001C6ADDED155A68EE868AE7EE258AE6EE30
:1073E000A87AFDEEE77A17EE901A8C45A8BF8C4676
:1073F0008B42D8BF634607EE903AF8EEE77AC2EDCB
:10740000077AB8F1000F01F0AB80464B1B68002BE8
:1074100041F0B380444B1B789BB1387870B1DFF8F2
:107420000081DFF81C910026F0B2D9F80030B8ECEA
:10743000010A9847387801368642F5DB3B4B1B68DA
:107440009847049B1B78072B01F0B28200230B9313
:10745000079B1B680A935E0501F1BF81344B1F68CF
:107460003C0701F15C81334BB3F80090324B089339
:10747000324B059A1C68B2F906806289904580F209
:1074800006864FF07E53CBF82431089A059992F97D
:107490000430B1F90000BAF81860117892F801E0F0
:1074A000002BA0EB060383EAE37CACEBE37C14BF88
:1074B00001224FF0FF32BCF5FA7FA8BF4FF4FA7CEF
:1074C000614580F2E085ACEB010307EE903AF8EEFF
:1074D000E77A8642C5ED007A03DDF1EE677AC5ED05
:1074E000007A059BB3F90200831B83EAE37CACEBD3
:1074F000E37CBCF5FA7FA8BF4FF4FA7C614580F2CB
:10750000BE85ACEB010307EE903AF8EEE77AB042A5
:10751000C5ED017A16DAF1EE677AC5ED017A11E070
:10752000E0500020E884002078820020487F00207E
:10753000E06200203C630020D85200204463002019
:10754000407F0020059BB3F904108B1B83EAE37096
:10755000A0EBE370B0F5FA7FA8BF4FF4FA70704566
:10756000CCBFA0EB0E0E4FF0000E02FB0EFE07EE9E
:1075700090EAF8EEE77AB1420A9BC5ED027ABCBF09
:10758000F1EE677AC5ED027A13F48053059300F0AB
:107590005185B8F5FA6F4246A8BF4FF4FA62B2F5CA
:1075A0007A7F9BF8A431B8BF4FF47A72A2F57A7251
